:020000040800F2
:1000000000500020719C0008695D00086F5D0008C9
:10001000755D00087B5D0008815D00080000000040
:10002000000000000000000000000000875D0008E4
:10003000895D0008000000008B5D00088D5D0008F0
:10004000B99C0008B99C0008B99C0008B99C00083C
:10005000B99C0008B99C0008B99C0008B99C00082C
:10006000B99C0008B99C0008B99C0008B99C00081C
:10007000458D0008B99C0008B99C0008B99C00088F
:10008000B99C0008B99C0008B99C0008B99C0008FC
:10009000A15D0008B99C0008B99C0008B99C000843
:1000A000B99C0008158E0008B99C0008B99C00088E
:1000B000B99C0008998E0008B99C0008B99C0008FA
:1000C000B99C0008B99C0008B99C0008B99C0008BC
:1000D000B99C000899960008B5960008B99C0008DC
:1000E000B99C0008B99C0008B99C000800000000F9
:1000F0000000000000000000000000000000000000
:0C01000000000000000000005FF808F1A3
:1001100010B5054C237833B9044B13B10448AFF341
:1001200000800123237010BDF801002000000000B2
:100130008CC0000808B5034B1BB103490348AFF35B
:10014000008008BD00000000FC0100208CC00008F9
:1001500081F0004102E000BF83F0004330B54FEA78
:1001600041044FEA430594EA050F08BF90EA020FE5
:100170001FBF54EA000C55EA020C7FEA645C7FEA78
:10018000655C00F0E2804FEA5454D4EB5555B8BF9B
:100190006D420CDD2C4480EA020281EA030382EA0C
:1001A000000083EA010180EA020281EA0303362D9E
:1001B00088BF30BD11F0004F4FEA01314FF4801C71
:1001C0004CEA113102D0404261EB410113F0004F83
:1001D0004FEA03334CEA133302D0524263EB43033A
:1001E00094EA050F00F0A780A4F10104D5F1200ED8
:1001F0000DDB02FA0EFC22FA05F2801841F1000133
:1002000003FA0EF2801843FA05F359410EE0A5F106
:1002100020050EF1200E012A03FA0EFC28BF4CF037
:10022000020C43FA05F3C01851EBE37101F00045ED
:1002300007D54FF0000EDCF1000C7EEB00006EEBFA
:100240000101B1F5801F1BD3B1F5001F0CD3490884
:100250005FEA30004FEA3C0C04F101044FEA4452DB
:1002600012F5800F80F09A80BCF1004F08BF5FEA62
:10027000500C50F1000041EB045141EA050130BD42
:100280005FEA4C0C404141EB010111F4801FA4F1E5
:100290000104E9D191F0000F04BF01460020B1FA3A
:1002A00081F308BF2033A3F10B03B3F120020CDA72
:1002B0000C3208DD02F1140CC2F10C0201FA0CF050
:1002C00021FA02F10CE002F11402D8BFC2F1200CB5
:1002D00001FA02F120FA0CFCDCBF41EA0C0190406B
:1002E000E41AA2BF01EB0451294330BD6FEA0404B4
:1002F0001F3C1CDA0C340EDC04F11404C4F120029F
:1003000020FA04F001FA02F340EA030021FA04F3B0
:1003100045EA030130BDC4F10C04C4F1200220FA07
:1003200002F001FA04F340EA0300294630BD21FA45
:1003300004F0294630BD94F0000F83F4801306BF0B
:1003400081F480110134013D4EE77FEA645C18BFFF
:100350007FEA655C29D094EA050F08BF90EA020F96
:1003600005D054EA000C04BF1946104630BD91EA8E
:10037000030F1EBF0021002030BD5FEA545C05D191
:100380004000494128BF41F0004130BD14F58004D0
:100390003CBF01F5801130BD01F0004545F0FE4144
:1003A00041F470014FF0000030BD7FEA645C1ABF79
:1003B000194610467FEA655C1CBF0B46024650EAB0
:1003C000013406BF52EA033591EA030F41F40021DC
:1003D00030BD00BF90F0000F04BF0021704730B562
:1003E0004FF4806404F132044FF000054FF0000137
:1003F00050E700BF90F0000F04BF0021704730B5F8
:100400004FF4806404F1320410F0004548BF4042CC
:100410004FF000013EE700BF42004FEAE2014FEA21
:1004200031014FEA02701FBF12F07F4393F07F4FFC
:1004300081F06051704732F07F4208BF704793F0FF
:100440007F4F04BF41F40021704730B54FF4607412
:1004500001F0004521F000411CE700BF50EA010215
:1004600008BF704730B54FF000050AE050EA0102BE
:1004700008BF704730B511F0004502D5404261EB2E
:1004800041014FF4806404F132045FEA915C3FF46F
:10049000D8AE4FF003025FEADC0C18BF03325FEA0C
:1004A000DC0C18BF033202EBDC02C2F1200300FABD
:1004B00003FC20FA02F001FA03FE40EA0E0021FAE2
:1004C00002F11444BDE600BF70B54FF0FF0C4CF4D0
:1004D000E06C1CEA11541DBF1CEA135594EA0C0F82
:1004E00095EA0C0F00F0DEF82C4481EA030621EABD
:1004F0004C5123EA4C5350EA013518BF52EA0335F8
:1005000041F4801143F4801338D0A0FB02CE4FF0A9
:100510000005E1FB02E506F00042E0FB03E54FF0D9
:100520000006E1FB03569CF0000F18BF4EF0010ED1
:10053000A4F1FF04B6F5007F64F5407404D25FEACD
:100540004E0E6D4146EB060642EAC62141EA555180
:100550004FEAC52040EA5E504FEACE2EB4F1FD0CC2
:1005600088BFBCF5E06F1ED8BEF1004F08BF5FEA40
:10057000500E50F1000041EB045170BD06F00046F2
:1005800046EA010140EA020081EA0301B4EB5C049F
:10059000C2BFD4EB0C0541EA045170BD41F4801197
:1005A0004FF0000E013C00F3AB8014F1360FDEBFBC
:1005B000002001F0004170BDC4F10004203C35DA98
:1005C0000C341BDC04F11404C4F1200500FA05F31B
:1005D00020FA04F001FA05F240EA020001F00042BC
:1005E00021F0004110EBD37021FA04F642EB060132
:1005F0005EEA430E08BF20EAD37070BDC4F10C045C
:10060000C4F1200500FA04F320FA05F001FA04F21F
:1006100040EA020001F0004110EBD37041F100010B
:100620005EEA430E08BF20EAD37070BDC4F1200516
:1006300000FA05F24EEA020E20FA04F301FA05F27E
:1006400043EA020321FA04F001F0004121FA04F226
:1006500020EA020000EBD3705EEA430E08BF20EAF6
:10066000D37070BD94F0000F0FD101F00046400030
:1006700041EB010111F4801F08BF013CF7D041EAB2
:10068000060195F0000F18BF704703F000465200B6
:1006900043EB030313F4801F08BF013DF7D043EA87
:1006A0000603704794EA0C0F0CEA135518BF95EA3D
:1006B0000C0F0CD050EA410618BF52EA4306D1D1C4
:1006C00081EA030101F000414FF0000070BD50EAE3
:1006D000410606BF1046194652EA430619D094EA6D
:1006E0000C0F02D150EA013613D195EA0C0F05D157
:1006F00052EA03361CBF104619460AD181EA0301AB
:1007000001F0004141F0FE4141F470014FF0000062
:1007100070BD41F0FE4141F4780170BD70B54FF0FD
:10072000FF0C4CF4E06C1CEA11541DBF1CEA13557D
:1007300094EA0C0F95EA0C0F00F0A7F8A4EB05045F
:1007400081EA030E52EA03354FEA013100F0888056
:100750004FEA03334FF0805545EA131343EA12631F
:100760004FEA022245EA111545EA10654FEA0026D4
:100770000EF000419D4208BF964244F1FD0404F58D
:10078000407402D25B084FEA3202B61A65EB0305E9
:100790005B084FEA32024FF480104FF4002CB6EBA6
:1007A000020E75EB030E22BFB61A754640EA0C0026
:1007B0005B084FEA3202B6EB020E75EB030E22BF66
:1007C000B61A754640EA5C005B084FEA3202B6EBA7
:1007D000020E75EB030E22BFB61A754640EA9C0066
:1007E0005B084FEA3202B6EB020E75EB030E22BF36
:1007F000B61A754640EADC0055EA060E18D04FEAF4
:10080000051545EA16754FEA06164FEAC30343EA93
:1008100052734FEAC2025FEA1C1CC0D111F4801F60
:100820000BD141EA00014FF000004FF0004CB6E759
:1008300011F4801F04BF01430020B4F1FD0C88BFF8
:10084000BCF5E06F3FF6AFAEB5EB030C04BFB6EB03
:10085000020C5FEA500C50F1000041EB045170BDF6
:100860000EF0004E4EEA113114EB5C04C2BFD4EB23
:100870000C0541EA045170BD41F480114FF0000EA7
:10088000013C90E645EA060E8DE60CEA135594EA23
:100890000C0F08BF95EA0C0F3FF43BAF94EA0C0F26
:1008A0000AD150EA01347FF434AF95EA0C0F7FF49B
:1008B00025AF104619462CE795EA0C0F06D152EAEF
:1008C00003353FF4FDAE1046194622E750EA4106D3
:1008D00018BF52EA43067FF4C5AE50EA41047FF4E4
:1008E0000DAF52EA43057FF4EBAE12E74FF0FF3C49
:1008F00006E000BF4FF0010C02E000BF4FF0010C1A
:100900004DF804CD4FEA410C7FEA6C5C4FEA430C92
:1009100018BF7FEA6C5C1BD001B050EA410C0CBFE1
:1009200052EA430C91EA030F02BF90EA020F002043
:10093000704710F1000F91EA030F58BF994208BFAA
:1009400090422CBFD8176FEAE37040F00100704767
:100950004FEA410C7FEA6C5C02D150EA013C07D1BE
:100960004FEA430C7FEA6C5CD6D152EA033CD3D009
:100970005DF8040B704700BF8446104662468C4603
:100980001946634600E000BF01B5FFF7B7FF002836
:1009900048BF10F1000F01BD4DF808EDFFF7F4FF5F
:1009A0000CBF012000205DF808FB00BF4DF808EDEA
:1009B000FFF7EAFF34BF012000205DF808FB00BF0D
:1009C0004DF808EDFFF7E0FF94BF012000205DF82F
:1009D00008FB00BF4DF808EDFFF7CEFF94BF0120E4
:1009E00000205DF808FB00BF4DF808EDFFF7C4FFDD
:1009F00034BF012000205DF808FB00BF4FEA410C26
:100A00007FEA6C5C02D150EA013C0AD14FEA430C08
:100A10007FEA6C5C02D152EA033C02D14FF0000045
:100A200070474FF0010070474FEA410212F5001283
:100A300015D211D56FF47873B3EB625212D94FEA25
:100A4000C12343F0004343EA505311F0004F23FA0F
:100A500002F018BF404270474FF00000704750EA64
:100A6000013005D111F0004008BF6FF00040704721
:100A70004FF00000704700BF4FEA4102B2F1E0437F
:100A800024BFB3F5001CDCF1FE5C0DD901F0004C75
:100A90004FEAC0024CEA5070B2F1004F40EB8300C5
:100AA00008BF20F00100704711F0804F21D113F1F1
:100AB0003872BCBF01F00040704741F480114FEA2A
:100AC0005252C2F11802C2F1200C10FA0CF320FAB3
:100AD00002F018BF40F001004FEAC1234FEAD323D0
:100AE00003FA0CFC40EA0C0023FA02F34FEA43033A
:100AF000CCE77FEA625307D150EA01331EBF4FF0C3
:100B0000FE4040F44000704701F0004040F0FE40DD
:100B100040F40000704700BF80F0004002E000BFDA
:100B200081F0004142001FBF5FEA410392EA030FD8
:100B30007FEA226C7FEA236C6AD04FEA1262D2EB22
:100B40001363C1BFD218414048404140B8BF5B4227
:100B5000192B88BF704710F0004F40F4000020F0C0
:100B60007F4018BF404211F0004F41F4000121F0D6
:100B70007F4118BF494292EA030F3FD0A2F1010220
:100B800041FA03FC10EB0C00C3F1200301FA03F15E
:100B900000F0004302D5494260EB4000B0F5000F81
:100BA00013D3B0F1807F06D340084FEA310102F140
:100BB0000102FE2A51D2B1F1004F40EBC25008BFF2
:100BC00020F0010040EA03007047490040EB0000BC
:100BD00010F4000FA2F10102EDD1B0FA80FCACF1EB
:100BE000080CB2EB0C0200FA0CF0AABF00EBC250EA
:100BF00052421843BCBFD0401843704792F0000FD8
:100C000081F4000106BF80F400000132013BB5E72A
:100C10004FEA41037FEA226C18BF7FEA236C21D0A0
:100C200092EA030F04D092F0000F08BF0846704705
:100C300090EA010F1CBF0020704712F07F4F04D1D3
:100C4000400028BF40F00040704712F100723CBFE6
:100C500000F50000704700F0004343F0FE4040F410
:100C6000000070477FEA226216BF08467FEA2363CE
:100C70000146420206BF5FEA412390EA010F40F4B9
:100C8000800070474FF0000304E000BF10F0004305
:100C900048BF40425FEA000C08BF704743F09643EC
:100CA00001464FF000001CE050EA010208BF704707
:100CB0004FF000030AE000BF50EA010208BF70478E
:100CC00011F0004302D5404261EB41015FEA010CA3
:100CD00002BF84460146002043F0B64308BFA3F19B
:100CE0008053A3F50003BCFA8CF2083AA3EBC2537D
:100CF00010DB01FA02FC634400FA02FCC2F120029C
:100D0000BCF1004F20FA02F243EB020008BF20F0D2
:100D10000100704702F1200201FA02FCC2F1200238
:100D200050EA4C0021FA02F243EB020008BF20EA2D
:100D3000DC7070474FF0FF0C1CEAD0521EBF1CEA5B
:100D4000D15392EA0C0F93EA0C0F6FD01A4480EA49
:100D5000010C400218BF5FEA41211ED04FF0006332
:100D600043EA501043EA5111A0FB01310CF000405E
:100D7000B1F5000F3EBF490041EAD3715B0040EA84
:100D8000010062F17F02FD2A1DD8B3F1004F40EB54
:100D9000C25008BF20F00100704790F0000F0CF027
:100DA000004C08BF49024CEA502040EA51207F3AEB
:100DB000C2BFD2F1FF0340EAC250704740F40000C6
:100DC0004FF00003013A5DDC12F1190FDCBF00F0B7
:100DD00000407047C2F10002410021FA02F1C2F165
:100DE000200200FA02FC5FEA310040F1000053EA01
:100DF0004C0308BF20EADC70704792F0000F00F04F
:100E0000004C02BF400010F4000F013AF9D040EA54
:100E10000C0093F0000F01F0004C02BF490011F4E8
:100E2000000F013BF9D041EA0C018FE70CEAD153E6
:100E300092EA0C0F18BF93EA0C0F0AD030F0004C66
:100E400018BF31F0004CD8D180EA010000F000401A
:100E5000704790F0000F17BF90F0004F084691F0D8
:100E6000000F91F0004F14D092EA0C0F01D1420212
:100E70000FD193EA0C0F03D14B0218BF084608D1DB
:100E800080EA010000F0004040F0FE4040F4000025
:100E9000704740F0FE4040F4400070474FF0FF0CB8
:100EA0001CEAD0521EBF1CEAD15392EA0C0F93EAFF
:100EB0000C0F69D0A2EB030280EA010C49024FEA51
:100EC000402037D04FF0805343EA111143EA10130A
:100ED0000CF000408B4238BF5B0042F17D024FF4C2
:100EE000000C8B4224BF5B1A40EA0C00B3EB510F9D
:100EF00024BFA3EB510340EA5C00B3EB910F24BF86
:100F0000A3EB910340EA9C00B3EBD10F24BFA3EB0A
:100F1000D10340EADC001B0118BF5FEA1C1CE0D1D2
:100F2000FD2A3FF650AF8B4240EBC25008BF20F085
:100F3000010070470CF0004C4CEA50207F32C2BFD9
:100F4000D2F1FF0340EAC250704740F400004FF076
:100F50000003013A37E792F0000F00F0004C02BFA7
:100F6000400010F4000F013AF9D040EA0C0093F071
:100F7000000F01F0004C02BF490011F4000F013BCB
:100F8000F9D041EA0C0195E70CEAD15392EA0C0F33
:100F900008D142027FF47DAF93EA0C0F7FF470AF6B
:100FA000084676E793EA0C0F04D14B023FF44CAFAE
:100FB00008466EE730F0004C18BF31F0004CCAD143
:100FC00030F000427FF45CAF31F000437FF43CAF7F
:100FD0005FE700BF4FF0FF3C06E000BF4FF0010CA1
:100FE00002E000BF4FF0010C4DF804CD4FEA400283
:100FF0004FEA41037FEA226C18BF7FEA236C11D0CD
:1010000001B052EA530C18BF90EA010F58BFB2EB7F
:10101000030088BFC81738BF6FEAE17018BF40F0FF
:10102000010070477FEA226C02D15FEA402C05D1B3
:101030007FEA236CE4D15FEA412CE1D05DF8040B38
:10104000704700BF844608466146FFE70FB5FFF7CB
:10105000C9FF002848BF10F1000F0FBD4DF808ED83
:10106000FFF7F4FF0CBF012000205DF808FB00BF74
:101070004DF808EDFFF7EAFF34BF012000205DF8CE
:1010800008FB00BF4DF808EDFFF7E0FF94BF01201B
:1010900000205DF808FB00BF4DF808EDFFF7D2FF18
:1010A00094BF012000205DF808FB00BF4DF808ED5B
:1010B000FFF7C8FF34BF012000205DF808FB00BF28
:1010C0004FEA40024FEA41037FEA226C02D15FEA15
:1010D000402C08D17FEA236C02D15FEA412C02D177
:1010E0004FF0000070474FF0010070474FEA400298
:1010F000B2F1FE4F0FD34FF09E03B3EB12620DD946
:101100004FEA002343F0004310F0004F23FA02F0AF
:1011100018BF404270474FF00000704712F1610F56
:1011200001D1420205D110F0004008BF6FF000402D
:1011300070474FF00000704742000ED2B2F1FE4FF0
:101140000BD34FF09E03B3EB126209D44FEA002396
:1011500043F0004323FA02F070474FF0000070475D
:1011600012F1610F01D1420202D14FF0FF307047FE
:101170004FF00000704700BFF8B50022002307467B
:101180000E46FFF713FC28B938463146BDE8F84053
:1011900000F00AB8384606F1004100F005F8404278
:1011A00061EB4101F8BD00BFD0B500220D4B0646F2
:1011B0000F46FFF789F900F019F80446FFF70AF91E
:1011C0000022094BFFF780F902460B4630463946AC
:1011D000FEF7C2FF00F00AF800222346104319462A
:1011E000D0BD00BF0000F03D0000F0414A0011D228
:1011F00012F5001211D20DD56FF47873B3EB625271
:101200000ED44FEAC12343F0004343EA505323FA7C
:1012100002F070474FF00000704750EA013002D1F1
:101220004FF0FF3070474FF000007047034613F84F
:10123000012B002AFBD1181A0138704710B504465B
:101240000E4B18784FF47A73B3FBF0F30C4A106826
:10125000B0FBF3F000F08EF868B90F2C01D9012033
:101260000AE0002221464FF0FF3000F041F8034B26
:101270005C60002000E0012010BD00BF00000020E5
:101280002C01002008B5074A136843F010031360CF
:10129000032000F01BF80020FFF7D0FF04F030FD22
:1012A000002008BD00200240034A1168034B1B7850
:1012B0000B441360704700BF900400200000002022
:1012C000014B1868704700BF90040020074AD3689C
:1012D00023F4E0631B041B0C000200F4E0601843DD
:1012E00040F0BF6040F40030D060704700ED00E097
:1012F00030B4174BDB68C3F30223C3F10704042C9B
:1013000028BF04241D1D062D18D9033B4FF0FF35BF
:1013100005FA04F421EA0401994005FA03F322EAEC
:101320000303194300280BDB0901C9B200F1604037
:1013300000F5614080F8001330BC70470023E5E7FA
:1013400000F00F000901C9B2024B1954F4E700BFC5
:1013500000ED00E014ED00E0002807DB00F01F02C4
:10136000400901239340024A42F82030704700BFF1
:1013700000E100E00138B0F1807F0AD2064B5860EE
:10138000064AF02182F823100020986007221A6094
:1013900070470120704700BF10E000E000ED00E062
:1013A000F0B587B0002873D0044690F82932D3B145
:1013B000032384F82932206800F0DBFF254655F826
:1013C000107B6E460FCD0FC62B683360231D0ECBEE
:1013D000384600F0BFFF58B1022384F829320125B6
:1013E000284607B0F0BD80F8283207F0C9F8DFE7DB
:1013F0000021206800F0C7FF002311E004EB431236
:10140000012182F8291082F82830D386002182F841
:101410002B109163D1639A1C5201A1500133DBB2AE
:1014200060688342EAD3002312E004EB43110022F8
:1014300081F8292181F8283181F82B21C1F8382140
:10144000C1F83C2103F10A01490162500133DBB2CA
:101450009842EAD8254655F8107B6E460FCD0FC648
:101460002B683360231D0ECB384600F08EFF0546F7
:1014700020B1022384F829320125B1E7002384F842
:101480002430012384F82932206801F0B0FAA7E75C
:101490000125A5E790F82832012B10D010B504469D
:1014A000012180F8281207F076F9206801F09DFAF2
:1014B000206800F056FF002084F8280210BD0220AA
:1014C000704790F82832012B0DD010B50446012347
:1014D00080F8283280F82410006801F080FA00209B
:1014E00084F8280210BD0220704770B511F0800FFB
:1014F00023D101F007056D0105F5947404440544FA
:10150000002685F8296101F0070121702261E3704E
:10151000627802B1E181022B1AD090F82832012BB7
:1015200019D00546012380F828322146006800F0D2
:1015300042FF002085F8280270BD01F007056D010B
:1015400005F1280404440544012685F82960DAE7FA
:1015500000232371E1E70220EEE710B511F0800FC0
:101560001CD101F007035B0103F5947202440344AC
:10157000002483F8294101F00703137090F8283202
:10158000012B16D00446012380F82832114600684A
:1015900001F0C5F8002084F8280210BD01F007030F
:1015A0005B0103F1280202440344012483F829402B
:1015B000E1E70220F1E770B501F007056C0104F5E1
:1015C000947101440444C4F83C2105F10A0252011B
:1015D000861883500023736084F8293184F82851D9
:1015E00025B1006801F01FFA002070BD006801F00D
:1015F0001AFAF9E701F007010A3100EB41114868D6
:10160000704770B501F007056C0104F12801014431
:101610000444E263AA1C52018618835000237360BD
:10162000012384F8293084F8285025B1006801F09E
:10163000FAF9002070BD006801F0F5F9F9E7F8B596
:1016400004462068B0F8443013F4004F00F0AD8138
:10165000B0F844309BB213F00F0540F0CD8013F08A
:10166000100F58D003889BB213F4006F40F08980AC
:1016700013F4004FE5D0038823F070031B051B0D06
:1016800043F0800303802068B0F8503094F828219C
:1016900003EBC203063300EB4303B3F80034C3F398
:1016A0000903C4F844318BB1D4F83C1171B1B4F8DA
:1016B0002E2101F048FBD4F84421D4F83C311344E6
:1016C000C4F83C310021204606F082FF2368B3F8BD
:1016D00050201344D4F83821002A74D1B3F80C24D4
:1016E00092B222F4F84292B2A3F80C24B3F80C247C
:1016F00042F40042A3F80C24226813889BB223F41E
:10170000804323F0700383F4405343F4004343F0D9
:101710008003138095E703889BB223F4E14323F011
:1017200070036FEA43436FEA53439BB2038022681E
:10173000B2F8503094F8281003EBC103023302EBE7
:101740004303B3F80034C3F309036364E26B134447
:10175000E3630021204606F045FF94F82430002B77
:101760003FF46FAF236C002B7FF46BAF94F8243001
:10177000226843F08003A2F84C30002384F8243020
:101780005FE7B0F8503094F8282103EBC20306332A
:1017900000EB4303B3F80034C3F30903C4F8443146
:1017A000B4F82E2104F50C7101F0CDFA22681388EB
:1017B00023F070031B051B0D43F0800313802046AC
:1017C00006F0FEFE3DE73E2A09D8510812F0010F4F
:1017D00000D00131890289B2A3F80C148CE75109B9
:1017E00012F01F0F00D101396FEAC1626FEA524255
:1017F00092B2A3F80C247FE730F82560B6B216F455
:10180000004F33D116F0800F3FF41BAF226832F83F
:1018100025309BB223F4E14323F070036FEA434386
:101820006FEA53439BB222F825302268B2F8503059
:1018300004EB451090F8281003EBC103023302EBD0
:101840004303B3F80024C2F30902AB1C5B01E118A7
:101850004A60C16B0A44C263E358002B40F09D808C
:1018600090F82810204606F0BDFEEAE630F8253054
:1018700023F070031B051B0D43F0800320F8253077
:1018800004EB451393F83431D3B92068B0F85030E5
:1018900004EB451292F8282103EBC203063300EB58
:1018A0004303B3F80074C7F309078FB304EB451182
:1018B0003B46B1F82E21D1F83C1101F044FA27E063
:1018C000206804EB451393F8282130F8223013F4F4
:1018D000804F43D0B0F8503003EBC203023300EB2B
:1018E0004303B3F80074C7F309076FBB226804EB26
:1018F000451393F8281132F821309BB223F4E043CA
:1019000023F0700343F4004343F0C00322F8213076
:1019100005F10A035B01E1184A683A444A6004EBA6
:101920004511D1F83C213A44C1F83C21E3581BB1A0
:10193000D1F838118F4228D204EB451393F82811BF
:10194000204606F045FE5DE704EB45113B46B1F845
:101950003021D1F83C1101F0F6F9C7E7B0F850306A
:1019600003EBC203063300EB4303B3F80074C7F381
:101970000907002FBAD004EB45113B46B1F83221DC
:10198000D1F83C1101F0DFF9B0E704EB451191F813
:1019900028112046FFF70FFE34E704EB451595F8B4
:1019A00028102046FFF72DFE4BE60020F8BD10B5AD
:1019B0000446006801F01DF810F4004F45D120687E
:1019C00001F017F810F4806F43D1206801F011F88E
:1019D00010F4804F08D02268B2F844309BB223F450
:1019E00080439BB2A2F84430206801F002F810F462
:1019F000005F08D02268B2F844309BB223F4005351
:101A00009BB2A2F84430206800F0F3FF10F4805F2E
:101A100030D1206800F0EDFF10F4006F49D120684C
:101A200000F0E7FF10F4007F6DD1206800F0E1FFC7
:101A300010F4807F08D02268B2F844309BB223F4BF
:101A400080739BB2A2F8443010BD2046FFF7F7FD2B
:101A5000B5E72268B2F844309BB223F480639BB2AE
:101A6000A2F84430204606F0CCFD00212046FFF7C6
:101A700028FDAAE72268B2F840309BB223F00403A5
:101A80009BB2A2F840302268B2F840309BB223F0FB
:101A900008039BB2A2F84030204606F0D3FD22682E
:101AA000B2F844309BB223F480539BB2A2F8443086
:101AB000AFE72268B2F8403043F00803A2F84030A4
:101AC0002268B2F844309BB223F400639BB2A2F8C0
:101AD00044302268B2F8403043F00403A2F84030AA
:101AE000206800F086FF10F4805F08D02268B2F80A
:101AF00044309BB223F480539BB2A2F8443020467A
:101B000006F090FD8BE72268B2F844309BB223F4D4
:101B100000739BB2A2F84430204606F06CFD84E7C7
:101B200038B501F0070543689D422CD811F0800FAD
:101B30001AD14B0103F5947101440344002283F848
:101B4000292101238B700D7090F82832012B1CD0B5
:101B50000446012380F82832006800F0CAFE65B10F
:101B6000002084F828020FE06B0103F128010144F2
:101B70000344012283F82920E3E704F50C7120686F
:101B800000F03AFFECE7012038BD0220FCE701F04D
:101B90000F0243689A422DD810B511F0800F1ED164
:101BA00001F007035B0103F594720244034400242F
:101BB00083F829410023937001F00703137090F814
:101BC0002832012B18D00446012380F82832114610
:101BD000006800F0B3FE002084F8280210BD01F078
:101BE00007035B0103F1280202440344012483F844
:101BF0002940DFE7012070470220EFE711F0800F56
:101C00000CD001F007014901283101445AB10122E9
:101C10000A730B811B0C4B8100207047490101F5B1
:101C200094710144F2E70A73CB80F5E782B0084B68
:101C30001B68084AA2FB03235B0A00FB03F0019028
:101C400000BF019B5A1E0192002BF9D102B07047D0
:101C50002C010020D34D6210002800F0F58170B5F2
:101C600082B00446036813F0010F2CD0AB4B5B68C5
:101C700003F00C03042B1DD0A84B5B6803F00C038E
:101C8000082B12D06368B3F5803F41D0002B55D1AB
:101C900003F1804303F504331A6822F480321A609A
:101CA0001A6822F480221A6037E09C4B5B6813F4B8
:101CB000803FE7D0994B1B6813F4003F03D0636863
:101CC000002B00F0C381236813F0020F76D0934BF2
:101CD0005B6813F00C0F5FD0904B5B6803F00C0354
:101CE000082B54D02369002B00F08A808C4B0122F2
:101CF0001A60FFF7E5FA0546884B1B6813F0020FE0
:101D000075D1FFF7DDFA401B0228F5D90320A0E1C9
:101D1000824A136843F480331360636843B3FFF768
:101D2000CFFA05467D4B1B6813F4003FCBD1FFF77C
:101D3000C7FA401B6428F5D903208AE1B3F5A02F28
:101D400009D0764B1A6822F480321A601A6822F49D
:101D500080221A60E1E703F18043A3F53C331A685F
:101D600042F480221A601A6842F480321A60D4E782
:101D7000FFF7A6FA0546694B1B6813F4003FA2D093
:101D8000FFF79EFA401B6428F5D9032061E1634BFD
:101D90005B6813F4803FA5D1604B1B6813F0020F02
:101DA00004D02369012B01D0012052E15B4A136862
:101DB00023F0F803616943EAC1031360236813F059
:101DC000080F32D0A369002B5BD0564B01221A605A
:101DD000FFF776FA0546514B5B6A13F0020F21D1EB
:101DE000FFF76EFA401B0228F5D9032031E14B4A78
:101DF000136823F0F803616943EAC1031360DDE768
:101E0000474B00221A60FFF75BFA0546434B1B68FD
:101E100013F0020FD2D0FFF753FA401B0228F5D976
:101E2000032016E10120FFF701FF236813F0040FE0
:101E300000F09880394BDB6913F0805F33D1374B6A
:101E4000DA6942F08052DA61DB6903F08053019372
:101E5000019B0125344B1B6813F4807F25D0E36878
:101E6000012B36D0002B4CD103F1804303F5043312
:101E70001A6A22F001021A621A6A22F004021A6235
:101E80002CE0284B00221A60FFF71AFA0546234B74
:101E90005B6A13F0020FC8D0FFF712FA401B02284A
:101EA000F5D90320D5E00025D4E71F4A136843F491
:101EB00080731360FFF704FA06461B4B1B6813F48C
:101EC000807FCCD1FFF7FCF9801B6428F5D9032073
:101ED000BFE0124A136A43F001031362E3687BB365
:101EE000FFF7EEF906460D4B1B6A13F0020F38D1CF
:101EF000FFF7E6F9801B41F288339842F3D90320BB
:101F0000A7E0052B12D0054B1A6A22F001021A62D3
:101F10001A6A22F004021A62E0E700BF00100240D1
:101F20000000424280044242007000404C4B1A6A5A
:101F300042F004021A621A6A42F001021A62CDE704
:101F4000FFF7BEF90646464B1B6A13F0020F08D096
:101F5000FFF7B6F9801B41F288339842F3D903208A
:101F600077E0E5B9E369002B72D03D4A526802F090
:101F70000C02082A56D0022B17D03A4B00221A60C6
:101F8000FFF79EF90446364B1B6813F0007F47D0DD
:101F9000FFF796F9001B0228F5D9032059E0304AD3
:101FA000D36923F08053D361DCE72E4B00221A6003
:101FB000FFF786F905462A4B1B6813F0007F06D011
:101FC000FFF77EF9401B0228F5D9032041E0236A80
:101FD000B3F5803F1AD022494B6823F47413226A68
:101FE000606A024313434B601E4B01221A60FFF7E5
:101FF00067F904461A4B1B6813F0007F0ED1FFF7F8
:102000005FF9001B0228F5D9032022E0144A536827
:1020100023F40033A1680B435360DCE7002018E091
:10202000002016E0012B16D00D4B5B6803F48031C5
:10203000226A914201D001200BE003F47013626A1E
:1020400093420AD0012004E001207047012000E003
:10205000002002B070BD0120FBE70020F9E700BFBF
:10206000001002406000424210B487B0164C94E861
:102070000F000DF1180C0CE90F00238AADF80430A5
:10208000124B5B6803F00C02082A1AD1C3F3834297
:10209000624412F8102C13F4803F05D10C4800FB69
:1020A00002F007B010BC7047084B5B68C3F34043B5
:1020B000634413F8143C074800FB02F0B0FBF3F054
:1020C000EFE70448EDE700BFA8C000080010024099
:1020D00000093D0000127A00002800F0A38070B5CE
:1020E0000446524B1B6803F007038B420CD24F4A45
:1020F000136823F007030B431360136803F007030F
:102100008B4201D0012070BD236813F0020F17D05D
:1021100013F0040F04D0464A536843F4E06353605D
:10212000236813F0080F04D0414A536843F4605306
:1021300053603F4A536823F0F003A06803435360A1
:102140000D46236813F0010F31D06368012B20D0B6
:10215000022B25D0364A126812F0020F64D034499F
:102160004A6822F0030213434B60FFF7A9F80646C2
:102170002F4B5B6803F00C036268B3EB820F16D041
:10218000FFF79EF8801B41F288339842F0D9032074
:10219000B9E7274A126812F4003FE0D10120B2E704
:1021A000234A126812F0007FD9D10120ABE71F4B00
:1021B0001B6803F00703AB420CD91C4A136823F0D9
:1021C00007032B431360136803F00703AB4201D0EE
:1021D000012098E7236813F0040F06D0144A5368CF
:1021E00023F4E063E1680B435360236813F0080FA6
:1021F00007D00F4A536823F46053216943EAC103AF
:102200005360FFF731FF0A4B5B68C3F30313094ABE
:10221000D35CD840084B1860084B1868FFF70EF8DD
:10222000002070E70120704701206CE70020024089
:1022300000100240BCC000082C0100200400002057
:1022400070B582B00446036813F0010F34D03E4BE2
:10225000DB6913F0805F48D13B4BDA6942F0805272
:10226000DA61DB6903F080530193019B0125374B51
:102270001B6813F4807F3AD0334B1B6A13F440730E
:1022800011D0626802F440729A420CD02E4A136A4E
:1022900023F440702E4901260E6000260E60106265
:1022A00013F0010F37D1284A136A23F44073616891
:1022B0000B431362002D3FD1236813F0020F06D0A9
:1022C000214A536823F44043A1680B4353602368B9
:1022D00013F0100F35D01C4A536823F48003E168D3
:1022E0000B435360002002B070BD0025BFE7174AC2
:1022F000136843F480731360FEF7E2FF0646134B46
:102300001B6813F4807FB7D1FEF7DAFF801B6428C7
:10231000F5D90320E7E7FEF7D3FF06460A4B1B6A11
:1023200013F0020FBFD1FEF7CBFF801B41F28833C1
:102330009842F3D90320D6E7D36923F08053D361C1
:10234000BAE70020CFE700BF001002400070004055
:102350004004424284B001A880E80E00002004B08E
:102360007047B0F8403043F43F43A0F840300020BD
:102370007047B0F8403023F47C535B045B0CA0F84A
:102380004030002070470020704784B038B505AC5D
:1023900084E80E000123A0F840300024A0F840405B
:1023A000A0F84440A0F85040FFF7DBFF2046BDE80E
:1023B000384004B0704730B403460C7830F824201D
:1023C00092B222F4EC4222F0700292B2C878032852
:1023D0005AD8DFE800F04D550251002048F2800540
:1023E0002A4323F824200C7833F8242092B222F4D4
:1023F000E04222F0700222432A4323F824200A7B81
:10240000002A40F0B1804A78002A4ED0B3F850201C
:102410001A440C7802EB0412CC8864086400A2F819
:1024200000440C7833F8242012F0400F0CD033F81D
:10243000242092B222F4E04222F0700242F40042E0
:1024400042F0C00223F82420CA78012A1ED009785D
:1024500033F8212092B222F4E04222F0400282F0CE
:10246000200242F4004242F0800223F8212060E082
:1024700042F400720020B1E742F4C0620020ADE7F0
:1024800042F480620020A9E70120A7E7097833F829
:10249000212092B222F4E04222F0400242F40042B3
:1024A00042F0800223F8212043E0B3F850201A4480
:1024B0000C7802EB0412CC8864086400A2F808448B
:1024C000B3F850201A440C7802EB04120C6994BB48
:1024D000B2F80C44A4B224F4F844A4B2A2F80C4418
:1024E000B2F80C4444F40044A2F80C440C7833F8DD
:1024F000242012F4804F0CD033F8242092B222F41E
:10250000E04222F0700242F4404242F0800223F89E
:102510002420097833F8212092B222F4804222F05C
:10252000700282F4405242F4004242F0800223F8EA
:10253000212030BC70473E2C09D8650814F0010FEB
:1025400000D00135AD02ADB2A2F80C54CEE765095A
:1025500014F01F0F00D1013D6FEAC5646FEA5444C7
:10256000A4B2A2F80C44C1E70C7833F8242092B24C
:1025700022F4E04222F0700242F4014242F0800272
:1025800023F82420B3F850201A440C7802EB0412EC
:102590000C8964086400A2F80044B3F850201A447F
:1025A0000C7802EB04124C8964086400A2F8084419
:1025B0004A78002A4ED10C7833F8242012F4804F48
:1025C0000CD033F8242092B222F4E04222F07002C0
:1025D00042F4404242F0800223F824200C7833F881
:1025E000242012F0400F0CD033F8242092B222F4B1
:1025F000E04222F0700242F4004242F0C00223F8AE
:1026000024200C7833F8242092B222F4E04222F005
:10261000700242F4004242F0C00223F824200D78F8
:1026200033F8252092B222F4804222F0700282F424
:10263000405248F28004224323F82520097833F8D9
:10264000212092B222F4E04222F04002224323F8F9
:1026500021206EE70C7833F8242012F4804F0CD040
:1026600033F8242092B222F4E04222F0700242F4C5
:10267000404242F0800223F824200C7833F82420D2
:1026800012F0400F0CD033F8242092B222F4E04232
:1026900022F0700242F4004242F0C00223F82420EB
:1026A0000C7833F8242092B222F4E04222F0700237
:1026B00042F4404242F0800223F82420CA78012AE2
:1026C0001ED00C7833F8242092B222F4E04222F09B
:1026D000400282F0200242F4004242F0800223F8DD
:1026E0002420097833F8212092B222F4804222F08B
:1026F000700242F4004242F0800223F8212018E7E1
:102700000C7833F8242092B222F4E04222F0400206
:1027100042F4004242F0800223F82420E1E70B7BE0
:10272000002B46D14B7813B30A7830F8223013F0DF
:10273000400F0CD030F822309BB223F4E04323F05A
:10274000700343F4004343F0C00320F822300A78BA
:1027500030F822309BB223F4E04323F0400343F4EB
:10276000004343F0800320F82230002070470A78AD
:1027700030F8223013F4804F0CD030F822309BB266
:1027800023F4E04323F0700343F4404343F0800319
:1027900020F822300A7830F822309BB223F48043AC
:1027A00023F0700343F4004343F0800320F8223009
:1027B000DBE710B44B78002B4ED10A7830F822308A
:1027C00013F4804F0CD030F822309BB223F4E04356
:1027D00023F0700343F4404343F0800320F8223099
:1027E0000A7830F8223013F0400F0CD030F8223045
:1027F0009BB223F4E04323F0700343F4004343F01F
:10280000C00320F822300A7830F822309BB223F43B
:10281000E04323F0700343F4004343F0C00320F887
:1028200022300B7830F8232092B222F4804222F03A
:10283000700248F28004224320F823200A7830F8FE
:1028400022309BB223F4E04323F04003234320F8DB
:102850002230002010BC70470A7830F8223013F480
:10286000804F0CD030F822309BB223F4E04323F0A9
:10287000700343F4404343F0800320F822300A7889
:1028800030F8223013F0400F0CD030F822309BB2D9
:1028900023F4E04323F0700343F4004343F0C00308
:1028A00020F822300A7830F822309BB223F4E0433B
:1028B00023F0700343F4404343F0800320F82230B8
:1028C0000B7830F8232092B222F4E04222F040024A
:1028D00048F28004224320F823200A7830F822307E
:1028E0009BB223F4804323F07003234320F822306B
:1028F000AFE74B788BB90A7830F822309BB223F4DB
:10290000804323F0700383F4805343F4004343F087
:10291000800320F82230002070470A7830F82230F7
:102920009BB223F4E04323F0400383F0100343F40D
:10293000004343F0800320F82230ECE70B7B002BB0
:102940004BD14B7833B30A7830F8223013F0400F74
:102950000CD030F822309BB223F4E04323F0700314
:1029600043F4004343F0C00320F82230CB78012B1E
:1029700033D00A7830F822309BB223F4E04323F0BE
:10298000400383F0200343F4004343F0800320F826
:10299000223022E00A7830F8223013F4804F0CD035
:1029A00030F822309BB223F4E04323F0700343F469
:1029B000404343F0800320F822300A7830F8223078
:1029C0009BB223F4804323F0700383F4405343F419
:1029D000004343F0800320F822300020704711B9F3
:1029E0008023A0F84C300020704700207047002062
:1029F0007047B0F8440070470020704701335B080F
:102A000000EB420202F5806263B110B40C784878A2
:102A100044EA002422F8044B0231013B002BF5D19B
:102A200010BC7047704770B54E78012E33D08A695C
:102A30000B699A4240F2FC80D21A8A610A7B002A12
:102A400040F01381B0F8502002440C7802EB0412DD
:102A5000002B40F0F180B2F80C349BB223F4F84321
:102A60009BB2A2F80C34B2F80C3443F40043A2F841
:102A70000C340A7830F822309BB223F4804323F0E0
:102A8000700383F4405343F4004343F0800320F881
:102A90002230002070BD8A690B699A4222D9D21A6D
:102AA0008A610C4605460A7B02B30A7830F8221088
:102AB00011F0400F72D0002E40D1B0F850100144F8
:102AC00001EB02120BBBB2F80C1489B221F4F841ED
:102AD00089B2A2F80C14B2F80C1441F40041A2F827
:102AE0000C1433E000238B611346DAE79EB23346C1
:102AF000CA884969FFF782FFB5F850302B44227825
:102B000003EB0213A3F8046437E03E2B09D85908FD
:102B100013F0010F00D00131890289B2A2F80C1420
:102B200014E0590913F01F0F00D101396FEAC16198
:102B30006FEA514189B2A2F80C1407E0B0F85010C6
:102B4000014401EB021299B2A2F80C1462899BB203
:102B500061692846FFF752FF6378002B57D122782E
:102B600035F822309BB223F4E04323F0700343F4A2
:102B7000004343F0C00325F82230227835F8223094
:102B80009BB223F4E04323F0400383F0300343F48B
:102B9000004343F0800325F822307AE76EBBB0F89B
:102BA0005010014401EB021273B9B2F8041489B257
:102BB00021F4F84189B2A2F80414B2F8041441F4E3
:102BC0000041A2F8041420E03E2B09D8590813F064
:102BD000010F00D00131890289B2A2F8041414E077
:102BE000590913F01F0F00D101396FEAC1616FEA73
:102BF000514189B2A2F8041407E0B0F85010014422
:102C000001EB021299B2A2F8041422899FE7012B6A
:102C1000B3D1227835F822309BB223F4E04323F07D
:102C2000700343F4404343F0800325F82230A4E7C7
:102C300000238B61134601E73E2B09D85C0813F093
:102C4000010F00D00134A402A4B2A2F80C4410E792
:102C50005C0913F01F0F00D1013C6FEAC4646FEAF6
:102C60005444A4B2A2F80C4403E7A6B9B0F850202B
:102C700002440C7802EB041233BBB2F80444A4B251
:102C800024F4F844A4B2A2F80444B2F8044444F48E
:102C90000044A2F804444A78002A47D1B0F85020F2
:102CA00002440C7802EB04123BBBB2F80C349BB22A
:102CB00023F4F8439BB2A2F80C34B2F80C3443F47A
:102CC0000043A2F80C34D4E63E2B09D85C0813F07C
:102CD000010F00D00134A402A4B2A2F80444DAE740
:102CE0005C0913F01F0F00D1013C6FEAC4646FEA66
:102CF0005444A4B2A2F80444CDE73E2B09D85C08A2
:102D000013F0010F00D00134A402A4B2A2F80C44C5
:102D1000AFE65C0913F01F0F00D1013C6FEAC463FA
:102D20006FEA53439BB2A2F80C34A2E6012A7FF467
:102D3000A0AEB0F8502002440C7802EB04129BB213
:102D4000A2F80C3495E630B45D0800EB420202F5BF
:102D5000806207E032F8044BA4B20C70240A4C7075
:102D60000231013D002DF5D113F0010F01D0138880
:102D70000B7030BC704710B5D0F8B842D0F8BC32F8
:102D80005BB194F80002FF2807D09B6894F80122F9
:102D900021469847FF2384F80032002010BD000030
:102DA000432303800048704708000020432303802A
:102DB000004870474C0000204323038000487047C0
:102DC000900000200A23038000487047D4000020B0
:102DD00038B50446D0F8B85205F0D2FCC5F80C025C
:102DE000D4F8B8324BB1D4F8BC32DB6805F50371C6
:102DF000D5F804029847002038BD0220FCE738B51A
:102E0000D0F8B822D0F8C052EAB101EB8104A30097
:102E10000344DB693BB105EB4115AD6BB3FBF5F446
:102E200005FB14331BB10020C2F8140238BD01EBBE
:102E30008102930003440024DC612346224605F00E
:102E40008FFC2046F2E70220F0E770B582B005461D
:102E50000C46D0F8B86200238DF80730ADF8043086
:102E60000B7813F0600227D0202A56D1CA883AB9CD
:102E7000D0F8BC329B6800224878984700204FE089
:102E800013F0800F0CD0D0F8BC329B6831466078CC
:102E90009847E2883146284600F0AEFD00203FE02A
:102EA0004B7886F800328B7986F80132CA88314631
:102EB00000F0B7FD002033E04B780A2B14D00B2B29
:102EC00021D01BB100F077FA022029E090F89C3263
:102ED000032B05D1022201A900F08EFD00201FE086
:102EE00000F069FA02201BE090F89C32032B06D117
:102EF00001220DF1070100F07FFD002010E000F03D
:102F00005AFA02200CE090F89C32032B01D10020E9
:102F100006E000F050FA022002E000F04CFA022035
:102F200002B070BD38B50446812105F0E6FB0025EE
:102F3000E5620121204605F0E0FBC4F86C518221D6
:102F4000204605F0DAFB2564D4F8B8324BB1D4F84A
:102F5000BC325B689847D4F8B80205F01BFCC4F893
:102F6000B852002038BD38B50446037CA3BB4FF4EB
:102F700000730222812105F0B5FB0125E5624FF4C3
:102F8000007302222946204605F0ACFBC4F86C51C0
:102F9000082303228221204605F0A4FB0123236499
:102FA0004FF4077005F0F2FB0546C4F8B80268B3A9
:102FB000D4F8BC321B6898470023C5F81432C5F812
:102FC0001832237CC3B14023D5F8042201212046C6
:102FD00005F0CEFB002038BD40230222812105F000
:102FE00081FB0125E562402302222946204605F0A7
:102FF00079FBC4F86C51CBE74FF40073D5F8042289
:103000000121204605F0B4FB0020E4E70120E2E7BF
:1030100019B1C0F8BC120020704702207047D0F8E8
:10302000B832C3F80812C3F8102200207047D0F855
:10303000B832C3F8041200207047D0F8B822A2B109
:1030400008B5D2F814320BB1012008BD0123C2F833
:103050001432D2F810320363B2F81032D2F80822D8
:10306000812105F07DFB0020EFE702207047D0F8BA
:10307000B8229AB108B5037C3BB14023D2F80422B0
:10308000012105F075FB002008BD4FF40073D2F854
:103090000422012105F06CFB0020F5E702207047B7
:1030A00098B108B50346D0F8B40210B10020C3F8B7
:1030B000B40209B1C3F8B0121846012380F89C325B
:1030C000027005F0C5FA002008BD0220704719B152
:1030D000C0F8B412002070470220704708B505F010
:1030E000F9FA002008BD08B5D0F8B43233B11B6836
:1030F000984708B9002008BD0220FCE70220FAE743
:1031000008B5D0F8B4325B689847002008BD38B5E0
:10311000044600F52A75284600F039F90123C4F861
:103120009432B4F8AE32C4F8983294F8A81201F090
:103130001F03012B0ED03BB1022B10D001F08001F8
:10314000204605F0E2FA03E02946204600F0CDFAD9
:10315000002038BD2946204600F0FBFAF8E7294652
:10316000204600F026FBF3E738B50446A1BB104625
:10317000D4F89432032B03D0052B24D0002037E061
:10318000D4F86031D4F8642193420DD99B1AC4F865
:1031900060319A4206D99AB20146204600F050FCAE
:1031A000002025E092B2F7E7D4F8B4321B692BB1C6
:1031B00094F89C22032A01D120469847204600F02B
:1031C00047FC002014E00025C4F89452294620460C
:1031D00005F09BFA28460BE00A46D0F8B4329B690A
:1031E0003BB190F89C12032905D111469847002065
:1031F00038BD0220FCE70220FAE710B5044600299A
:1032000053D11046D4F89432022B0CD0042B00D0AA
:103210001BB98021204605F078FA94F8A032012BE2
:103220003FD000204DE0236A626A93421DD8E169D5
:10323000B1FBF2F302FB13132BB98A4203D8D4F883
:10324000983299421FD3D4F8B432DB682BB194F88A
:103250009C22032A01D1204698478021204605F070
:1032600054FA204600F0FFFBD7E79A1A226292B286
:103270000146204600F0CDFB00231A4619462046A1
:1032800005F076FAC9E700221146204600F0C1FB9E
:103290000021C4F898120B460A46204605F068FA49
:1032A000BBE7002084F8A0020BE00A46D0F8B43255
:1032B0005B693BB190F89C12032905D111469847F0
:1032C000002010BD0220FCE70220FAE770B504469A
:1032D00040230022114605F005FA0125C4F8585193
:1032E0004026C4F86461334600228021204605F060
:1032F000F9F9A561666284F89C520023C4F89432FF
:103300006360C4F8A432D4F8B8322BB1D4F8B43224
:103310005B68002120469847002070BD01740020A2
:10332000704790F89C3280F89D32042380F89C32DC
:103330000020704790F89C32042B01D00020704789
:1033400090F89D3280F89C32F8E708B590F89C32EE
:10335000032B01D0002008BDD0F8B432DB69002B6C
:10336000F8D09847F6E7002302E00133DBB20130E2
:103370000278002AF9D11846704708B54B88012B0E
:1033800000D008BDC0F8A43200F062FBF9E70B786A
:1033900003704B7843708B78CA7803EB0223438029
:1033A0000B794A7903EB022383808B79CA7903EB8B
:1033B0000223C380704710B50446802105F0A5F9AB
:1033C0000021204605F0A1F910BD30B583B00546B7
:1033D0000C460023ADF806304A88130A013B062B41
:1033E00000F2A480DFE803F004182CA2A286930068
:1033F000D0F8B0321B680DF10601007C9847BDF88B
:1034000006201AB1E388002B40F09480E388002B5B
:1034100000F09A8003B030BD037C43B9D0F8B432D9
:103420009B6A0DF10600984702234370E7E7D0F846
:10343000B432DB6A0DF10600984702234370DEE7E1
:10344000D2B2052A52D8DFE802F003101D2A374411
:10345000D0F8B0325B6823B10DF10601007C9847CB
:10346000CDE72146FFF7A7FFD4E7D0F8B0329B683D
:1034700023B10DF10601007C9847C0E72146FFF714
:103480009AFFC7E7D0F8B032DB6823B10DF106012F
:10349000007C9847B3E72146FFF78DFFBAE7D0F8E5
:1034A000B0321B6923B10DF10601007C9847A6E7F5
:1034B0002146FFF780FFADE7D0F8B0325B6923B15A
:1034C0000DF10601007C984799E72146FFF773FF4D
:1034D000A0E7D0F8B0329B6923B10DF10601007C62
:1034E00098478CE72146FFF766FF93E72146FFF7F1
:1034F00062FF8FE7037C33B9D0F8B4325B6B0DF118
:10350000060098477BE72146FFF755FF82E7037CDB
:1035100043B9D0F8B4321B6B0DF10600984707236E
:1035200043706CE72146FFF746FF73E72146FFF73C
:1035300042FF6FE79A4228BF1A46ADF806200146BF
:10354000284600F059FA61E7284600F081FA61E761
:1035500038B504468B88F3B9CB88E3B94B887F2B09
:1035600019D803F07F0590F89C32032B0CD080F81B
:103570009E52294605F0ECF8204600F069FA35B174
:10358000022384F89C3209E0FFF715FF06E00123CF
:1035900084F89C3202E02046FFF70DFF38BD0000A2
:1035A00038B504460D468978284B197001290ED884
:1035B00090F89C32022B0ED0032B21D02946FFF726
:1035C000FAFE224B19782046FFF79AFD02E02946C1
:1035D000FFF7F1FE38BD81B14160032380F89C32D2
:1035E000FFF781FD022803D0204600F031FAF1E711
:1035F00029462046FFF7DFFEECE700F029FAE9E76D
:1036000089B1436899421DD0D9B2FFF779FD0F4BBC
:10361000197861602046FFF766FD02280DD020462C
:1036200000F016FAD6E7022380F89C324160FFF7DB
:1036300067FD204600F00CFACCE729462046FFF74C
:10364000BAFEC7E700F004FAC4E700BF1402002086
:1036500008B5CB88012B0BD190F89C329BB1022B83
:1036600009D9032B0FD10122011D00F0C5F901E09A
:10367000FFF7A1FE08BD0146002341F8083F0122E3
:1036800000F0BAF9F6E7FFF796FEF3E708B590F811
:103690009C32013B022B12D8CB88022B0CD1012388
:1036A000C360D0F8A4320BB10323C360022200F13F
:1036B0000C0100F0A1F908BDFFF77DFEFBE7FFF765
:1036C0007AFEF8E708B590F89C32013B022B09D846
:1036D0004B88012B00D008BD0023C0F8A43200F0B5
:1036E000B7F9F8E7FFF767FEF5E708B50B7803F0E1
:1036F0006003202B05D0402B03D043B1FFF75BFEC6
:1037000003E0D0F8B4329B689847002008BD4B789E
:10371000092B1BD8DFE803F011171A141A08051A31
:103720000E0BFFF752FEF0E7FFF712FFEDE7FFF792
:1037300037FFEAE7FFF78CFFE7E7FFF7A7FFE4E7CC
:10374000FFF71BFEE1E7FFF7BDFFDEE7FFF733FE04
:10375000DBE738B505460C460B7803F06003202BF9
:1037600006D0402B04D01BB1FFF725FE002038BD4A
:1037700095F89C32013B022B16D82379012B0ED8E9
:10378000D5F8B4329B68214628469847E388002B39
:10379000ECD10028EAD1284600F05AF9E6E72146A4
:1037A0002846FFF708FEE1E721462846FFF703FE1B
:1037B000DCE738B504468A880B7803F06003202BD9
:1037C00008D0D0B2402B05D05BB12046FFF7F3FD07
:1037D000002005E0D4F8B4329B68204698470020CA
:1037E00038BD202B05D1D4F8B4329B6820469847C9
:1037F000F6E74B78012B32D0002B5ED0032B40F044
:10380000D88094F89C32022B06D0032B16D0204689
:10381000FFF7D1FD0020E3E708B1802804D120465E
:10382000FFF7C9FD0020DBE70146204604F06DFFED
:103830008021204604F069FF0020D1E74B8823B99E
:1038400018B1802801D0CB8823B1204600F000F9C0
:103850000020C5E70146204604F057FFF5E794F83D
:103860009C32022B06D0032B16D02046FFF7A3FD77
:103870000020B5E708B1802804D12046FFF79BFD62
:103880000020ADE70146204604F03FFF802120469E
:1038900004F03BFF0020A3E74B88002B40F08E8014
:1038A00010F07F0F04D1204600F0D2F8002097E7F7
:1038B0000146204604F031FFF5E794F89C32022BD4
:1038C00006D0032B2AD02046FFF775FD002087E79E
:1038D00008B1802813D112F0800F15D100F07F00BD
:1038E00000EB8000830003F5A8712144043100251A
:1038F0000D600222204600F07FF8284670E720463F
:10390000FFF759FD00206BE700F07F0000EB80001F
:10391000830003F1100121440431E8E752B2002A88
:103920001FDB00F00F0303EB83039D002544D5F854
:10393000583123B3002A27DB00F07F0202EB82021A
:10394000930003F5A8752544043508B1802825D1D6
:1039500000232B6002222946204600F04DF800206B
:103960003EE700F00F0303EB83039D002544AB69A2
:10397000002BDFD12046FFF71EFD002030E7204658
:10398000FFF719FD00202BE700F07F0202EB820217
:10399000930003F1100525440435D6E7014620467F
:1039A00004F0C3FE10B101232B60D3E700232B608A
:1039B000D0E72046FFF7FFFC002011E700200FE7CB
:1039C000C8B170B50D4616460446FFF7CCFC013071
:1039D00040003080287003236B70022307E001341D
:1039E0005A1CD2B2E9540233DBB20021A954217827
:1039F0000029F4D170BD704710B513460222C0F8FB
:103A00009422C36103620A46002104F0A9FE00204B
:103A100010BD08B513460A46002104F0A1FE00209F
:103A200008BD10B513460322C0F89422C0F85C31DB
:103A3000C0F860310A46002104F09AFE002010BD53
:103A400008B513460A46002104F092FE002008BD86
:103A500008B50423C0F8943200231A46194604F02E
:103A60007FFE002008BD08B50523C0F8943200236E
:103A70001A46194604F07CFE002008BD0B88584009
:103A80005B080B8010F0010F04D083F4044383F033
:103A900008030B807047000008B5064B4FF6FF7215
:103AA0001A8201229A7600221A705A7005F0BCFA26
:103AB00008BD00BF9C04002020B1054B93F89D0079
:103AC000C0B27047034B93F89D00C0B2704700BF6F
:103AD000B804002058050020F8B50D46A04B1B88FF
:103AE000D3B19F4A538801339BB25380042B13D91F
:103AF000134600221A805A809A4B93F89E309B1AE4
:103B000018BF0123984A92F89E20002A3CD0022236
:103B10001343964A82F8B834012D37D0914C94F86B
:103B20009C305B00DBB200280CBF184643F001005C
:103B300084F89C007E282BD000F07F037F2B00F0C0
:103B4000C78094F89D30DBB300F03F033E2B37D0A5
:103B500010F0010F05D094F89A3063F07F0384F8D9
:103B60009A3094F89B300133DBB284F89B30072BFA
:103B700040F2EF80B4F89830962B00F2B980012B18
:103B800040F2D5800025D0E00022C1E7764CC6E7A0
:103B900094F89D30022B03D1B4F898200F2A10D846
:103BA000012384F89D30002384F89A3084F89B30F8
:103BB000A4F898304FF6FF732380284605F07CF870
:103BC000F8BD00231E461746911E8B4207DAE01807
:103BD000807810F0010F02D101339BB2F2E7731C21
:103BE00023449B78032B0AD0002384F89A3084F86E
:103BF0009B30A4F898304FF6FF732380E0E702363D
:103C00002644B378F02BEFD1214489782288D3431E
:103C1000DBB2994207D17B1E234499786FEA1223C5
:103C2000DBB2994203D0284605F046F8B8E70123F5
:103C300084F89E304A4B1B889A42B1D0484B1A8078
:103C4000284605F051F8494BA3F8B604B3F85822BA
:103C5000B3F85A329A420BD99B1A9BB203F25523FE
:103C60009BB2B4F89820023A9A4299DC00221AE0FA
:103C70009B1A9BB2033B9BB2F3E73C48B0F85862F7
:103C8000731C99B2A0F85812A3189B788355384B2F
:103C9000A3FB01639B094FF4167606FB1313A0F8F0
:103CA0005832013292B2B4F89830023B9A42E4DBC7
:103CB0002E4AB2F858124B1C9BB2FF2050544FF4BE
:103CC0001670B3FBF0F100FB1133A2F8583267E72E
:103CD000284604F0F1FF002384F89D3084F89A30E0
:103CE00084F89B30A4F898304FF6FF73238067E781
:103CF000002384F89D3084F89A3084F89B30A4F82F
:103D000098304FF6FF732380284604F0D5FF57E71D
:103D1000B4F89830023B234498782841214600F0BB
:103D20000100FFF7ABFE0135EDB2072DF0D90223FC
:103D300084F89D30B4F898305A1CA4F8982094F870
:103D40009A2023449A70002384F89A3084F89B3098
:103D500036E794F89A305B0884F89A3030E700BF71
:103D60001602002058050020B8040020FC050020A1
:103D7000B5814E1B10B5A24B5B785BB2082B19D0F6
:103D80009F4B9B7EDBB2032B00F00A819C4B9B7EFA
:103D9000DBB2042B00F00481994A147804F001048A
:103DA00013785B08137053785BB201335BB25370C6
:103DB000204610BD924B00225A709B7EDBB2012B35
:103DC0002DD08F4B9B7EDBB2022B3DD08C4B9B7E4C
:103DD000DBB2032B4BD08A4B9B7EDBB2042B75D01E
:103DE000874B9B7EDBB2052B00F08C80844B9B7E47
:103DF000DBB2062BC4D1834B0022A3F8B424804B42
:103E00005A8992B2DB899BB29A4280F0BC807C4A8C
:103E10007E231370538901339BB25381B0E7784BF3
:103E20005A8892B29B899BB29A4207D2744A7E23E7
:103E30001370538801339BB25380C2E7704B00224A
:103E40005A8002229A76BCE76D4B1B79DBB2032BBA
:103E500007D86B4A7E23137013790133DBB21371D9
:103E6000B4E7674B00221A7103229A76AEE7654BDE
:103E7000B3F8B4340A2B20D9614AD28892B2934263
:103E80001BD95F4BDA885F4B134493F85C32FF2BEE
:103E90000BD05B4AD1885B4B0B4493F85C321370B8
:103EA000D38801339BB2D38095E7554A0423937698
:103EB000D38801339BB2D3808DE70022514BA3F806
:103EC000B4244F4BDA8006229A7684E74C4B1B7A57
:103ED000DBB2012B08D94A4B4FF6FF721A8205223A
:103EE0009A7600221A727BE7454A138A9BB2117AAE
:103EF000C9000B41DB43DBB21370137A0133DBB231
:103F000013726DE73E4B1B79DBB2072B07D83C4A97
:103F10007E23137013790133DBB2137166E7384BDC
:103F200000221A7103229A76364BB3F8B4340A2B66
:103F300020D9334AD28892B293421BD9304BDA88C7
:103F4000304B134493F85C32FF2B0BD02C4AD188B2
:103F50002C4B0B4493F85C321370D38801339BB223
:103F6000D38043E7264A04239376D38801339BB258
:103F7000D3803BE70022234BA3F8B424204BDA8004
:103F800006229A7632E71E4B00225A819A764FF625
:103F9000FF7119825A721A705A7605F07DF8EFE6B1
:103FA000174B5B7ADBB2052B19D0154B1B7813F03E
:103FB000010F18D0124A537A0133DBB25372012435
:103FC0000F4B9B7EDBB2032B11D00D4A13785B089D
:103FD000137053785BB201335BB25370E8E6002490
:103FE000074B5C72E4E60024054B5C72E8E7044989
:103FF00011F8100B00F00100FFF740FDE5E700BFEE
:104000009C040020FC050020144B5B7EDBB2012BDE
:1040100022D0124B5B7EDBB2022B1DD0104BB3F8CB
:10402000B4340A2B04D80E4B0022A3F8B4247047F2
:1040300010B50C4B9C880C48A0FB04300B4B1C6843
:1040400004EBD0041421002000F050FA2044034B6C
:10405000586101225A7610BD704700BF9C040020B1
:10406000FC05002094040020CDCCCCCC80040020A2
:1040700008B5214B5B7E6BB11F4B5B7EDBB2022B25
:1040800008D01E4BB3F8B434092B04D81B4B0022C4
:10409000A3F8B42408BD04F005FE0028FAD1164B9D
:1040A0005A69174B1B689A42F4D204F0F5FD90B19F
:1040B000114B1B7EDBB2082B15D032210A2000F0F9
:1040C00015FA0F4B1B6803440B4A5361137E0133EF
:1040D000DBB21376DEE7084B02225A7600221A760C
:1040E000FFF7DAFCD6E7044B02225A7600221A7652
:1040F000FFF7D2FCCEE700BF9C040020FC050020A7
:104100008004002038B5144C4FF6FF712182134B08
:104110000022A3F85822A3F85A22A3F8B42483F863
:10412000B8240F4B19800F4B19800F4D2888FCF7CE
:10413000A9FD0E49FCF7B2FEFCF7FEFF80B2A0819C
:104140006888FCF79FFD0949FCF7A8FEFCF7F4FF1F
:1041500080B2E08138BD00BF9C040020FC05002037
:1041600058050020B8040020940400205C55D54078
:1041700000EB40129300764AD35C002B00F0E780FE
:1041800070B5D8B004469622002132A807F08AFE06
:104190000022134609E0591C6E48805C58AD2B4440
:1041A00003F8980C0132D2B28BB2062AF3D900225E
:1041B00009E0591C6848805C58AD2B4403F8980C02
:1041C0000132D2B28BB2052AF3D9644A1278520076
:1041D000D2B25D1CADB2603258A90B4403F8982CE2
:1041E00004EB44139A005A4B134493F87130F3B91B
:1041F0006B1E58AA134413F8982C42F0010203F8DE
:10420000982C6B1C9BB258AA2A44032102F8981CD4
:104210000235ADB258AA1344F02203F8982C0026B8
:1042200034E058A90844603200F8982C1AE00023C2
:104230000D2BDDD804EB44129100454A0A441A4480
:1042400092F871201AB9062B01D00D2BD0D1284637
:104250005200D2B258A9294401F8982C062BE0D07C
:104260000D2BDED00135ADB20133DBB2E0E7691CC6
:1042700004EB44139A00364B134433441B7B58AA77
:10428000154405F8983C0136F6B28DB204EB4412A1
:10429000930008332E4818440430FCF7C7FF8642C9
:1042A000E5D32F4BB3F8B464C6F51672AB1C9A4233
:1042B00043DD00230EE02A4AB2F8B414481CA2F8E9
:1042C000B40458A8184410F8980C0A4482F85C0208
:1042D0000133DBB29AB2AA42EDD3224B1B7873BBF7
:1042E0001F4DB5F8B4345A1CA5F8B4242B44FF2252
:1042F00083F85C22304601F045FAB5F8B414891B06
:1043000089B2013906F5167028446A4689B204302C
:1043100000F002F90021144801F06CFE204601F083
:10432000A1FE0021114801F065FE0021684601F060
:1043300061FE00210E4801F05DFE58B070BD0848D6
:10434000B0F8B41400F5177000F0BAF9C8E7704778
:10435000940E00201C0100202401002045020020B2
:10436000FC0500203C02002014C1000898D0000881
:1043700054C9000810B5002419E01D4A52F8210064
:104380001C4A1268904232D81A4A1268134401EB50
:1043900041129000184A0244C2F88030144B0022A7
:1043A00043F821202046FFF7E3FE0134E4B2072C56
:1043B0001DD8214604EB441293000F4AD35C002B16
:1043C000F3D004EB44139A000B4B13445B68002BAF
:1043D000EBD004EB44129000074A0244D2F880204C
:1043E000044800688242C8D9002ADED1C5E710BD62
:1043F0001C02002080040020940E00200023072BC4
:104400001CD830B40E485A01D418A1000144896860
:104410000C4C2468642505FB014101F6B8310A4CB7
:1044200044F823101A44910008440022C0F8802068
:104430000133DBB2072BE5D930BC7047704700BFB2
:10444000940E0020800400201C0200202DE9F84F6B
:1044500082460D4679B91AF80530303BDBB2092B9C
:1044600009D80135EDB2632DF5D900260027304675
:104470003946BDE8F88F6C1E24B20026002726E0DE
:104480001AF804B0ABF1300B681E001BFBF7B2FF4B
:1044900002460B460020144905F08AFC80468946F6
:1044A0005846FBF7A7FF42464B46FCF70DF88046FF
:1044B000894630463946FBF7D9FF42464B46FBF763
:1044C0004DFEFCF759FE06460F46013C24B2002C77
:1044D000CDDB002CD4D11AF804302D2BD0D176426C
:1044E00067EB4707F1E700BF0000244038B5814281
:1044F00005DB091A0DB204462DB9204638BD401A15
:1045000005B20C46F8E707F07BFD90FBF5F105FBE3
:10451000110121440CB2F0E7F0B4002301E00133B3
:10452000DBB2052B07D8DC1D045D6408202CF6D017
:1045300014700132F3E7437BC3F3430393B1561C7A
:104540002D241470092B02D9961C31245470721C2E
:10455000424CA4FB0354E408A5002C4465005B1BFB
:1045600030333370551C3E231370002301E00133B8
:10457000DBB2052B06D8C25C5208202AF7D02A707D
:104580000135F4E78379C3F3430393B16E1C2D2205
:104590002A70092B02D9AE1C31226A70751C2F4A71
:1045A000A2FB0342D2089400224454001B1B303368
:1045B0003370437B13F0010F3ED10E2233E0013301
:1045C000DBB2052B07D8D418045D6408202CF6D084
:1045D0002C700135F3E7971DC35DC3F34303B3B1FB
:1045E00005F1010C2D242C70092B03D905F1020CC7
:1045F00031246C700CF10105184CA4FB0364E40831
:10460000A600344466009B1B30338CF80030C3573F
:10461000002B0DDB073292B2382A0ED8531EC35C32
:1046200013F0010F09D12C232B7001350023C8E7AB
:104630002A232B700135EDE70E226B1C3A242C70D7
:10464000023292B28A4205D2845C1C70013292B26C
:104650000133F7E700221A70F0BC7047CDCCCCCC08
:104660002DE9D00316461F46C0434FF000084FF017
:10467000000918E052080133DBB2072B0FD882EA99
:10468000000414F0010F4FEA5000F3D080F06D40A9
:1046900080F4380080F4034080F02000EAE718F14D
:1046A000010849F10009B94508BFB04504D201EB42
:1046B00008031A780023E0E7C043BDE8D003704741
:1046C0002DE9F04182B007460E460025DFF89480C0
:1046D00012E0395D404605F017F80134A4B2B44247
:1046E000F7D3C021404605F00FF8404604F0F0FF34
:1046F0000135EDB2DFF87080012D0DD898F8043245
:10470000002BF5D1C021404604F0FEFF00214046B9
:1047100004F0FAFF0024E2E7114B1B7813B102B05A
:10472000BDE8F081C0238DF8043000248DF80540E9
:10473000012101A803F0F0FE01210DF1050003F0B5
:10474000EBFE05E00121381903F0E6FE0134A4B2C6
:10475000B442F7D3012101A803F0DEFEDFE700BF7A
:1047600085040020840C0020B41200200F4A136935
:1047700043F00103136100F1006000F57040018017
:104780000A4BDB6813F0010FFAD1084BDB6813F01A
:10479000200F05D0054AD36843F02003D36070474B
:1047A000024A136923F0010313617047002002409D
:1047B000F8B507460D46164600240BE0600015F8D4
:1047C0001430421CA95C43EA01213844FFF7CEFFB4
:1047D0000134A4B2B4EB560FF0D316F0010F00D1A0
:1047E000F8BD15F8141007EB4400FFF7BFFFF7E71B
:1047F00000F1006000F57040008870472DE9F84333
:1048000081460F46904600240EE0650005EB090640
:104810003046FFF7EDFF07F81400701CFFF7E8FFC4
:10482000013578550134A4B2B4EB580FEDD318F02C
:10483000010F01D1BDE8F88309EB4400FFF7D8FF71
:1048400007F81400F6E700001D4B1E4A5A6002F1FB
:1048500088325A601A4BDB6813F0010FFAD1184AFC
:10486000136943F0020313610022012A21D802F5E3
:1048700000333C339B0212494B610B6943F0400308
:104880000B610F4BDB6813F0010FFAD10C4BDB68A7
:1048900013F0200F07D00A49CB6843F02003CB6008
:1048A0000132D2B2E1E7064A136923F00203136131
:1048B0007047034A136923F002031361704700BF76
:1048C000002002402301674510B5FFF7BDFF062217
:1048D0003E490220FFF76CFF3D4B19780820FFF797
:1048E00045FF06223B4940F2BA40FFF761FF3A4CD0
:1048F00021880A20FFF73AFF61880C20FFF736FF76
:10490000A1880E20FFF732FF032234491020FFF761
:104910004FFF032232491420FFF74AFF314A137830
:10492000003318BF012392F8842052B302221343AC
:104930002C4A92F8082132B304221343294A92F8F0
:104940008C2112B308221343264A92F81022F2B1A6
:1049500010210B43234A92F89422D2B120210B4319
:10496000204A92F81823B2B140210B431D4A92F815
:104970009C2392B1802119431820FFF7F7FE0024F1
:104980001FE00022D3E70022D7E70022DBE7002167
:10499000DFE70021E3E70021E7E70021EBE704F18F
:1049A0000D0004EB44139A000E4B134459680E4B50
:1049B000A3FB0131C1F3CF114000FFF7D7FE013453
:1049C000E4B2072CEBD9002422E000BF2401002030
:1049D000450200201C01002094040020880C0020C7
:1049E000B8120020940E0020F119760504F115008C
:1049F00004EB44139A00AD4B13449968AC4BA3FBF2
:104A00000131C1F34F114000FFF7B0FE0134E4B2B1
:104A1000072CEBD9A74C642221463A20FFF7C8FEA9
:104A2000642204F184019E20FFF7C2FE642204F593
:104A300084714FF48170FFF7BBFE642204F5C671E8
:104A40004FF4B370FFF7B4FE642204F504714FF421
:104A5000E570FFF7ADFE642204F5257140F22E20CB
:104A6000FFF7A6FE642204F5467140F29220FFF79C
:104A70009FFE642204F5677140F2F620FFF798FE6E
:104A80000E2204F1650140F25A30FFF791FE0E222A
:104A900004F1E9014FF45A70FFF78AFE0E2204F286
:104AA0006D1140F27630FFF783FE0E2204F2F11111
:104AB0004FF46170FFF77CFE0E2204F2752140F284
:104AC0009230FFF775FE0E2204F2F9214FF4687060
:104AD000FFF76EFE0E2204F27D3140F2AE30FFF79A
:104AE00067FE0E2204F201414FF46F70FFF760FE83
:104AF000714C94F83E1001F0010140F2CA30FFF70A
:104B000035FE94F83D104FF47370FFF72FFE94F8C4
:104B10003F1094F8403043EA012140F2CE30FFF7D5
:104B200025FE052221464FF47470FFF741FE052251
:104B3000A11D40F2D630FFF73BFE052204F10C0127
:104B40004FF47770FFF734FE052204F1120140F2B2
:104B5000E230FFF72DFE062204F118014FF47A70BF
:104B6000FFF726FE062204F11E014FF47C70FFF7CA
:104B70001FFE062204F124014FF47E70FFF718FE99
:104B8000062204F12A014FF48060FFF711FE94F829
:104B9000301040F2AE40FFF7E9FD94F831104FF4C9
:104BA0009660FFF7E3FD94F8321040F2B240FFF751
:104BB000DDFD94F8331040F2B440FFF7D7FD94F8D0
:104BC00034104FF48160FFF7D1FD94F8351040F2B6
:104BD0000A40FFF7CBFD94F8361040F20C40FFF787
:104BE000C5FD94F8371040F20E40FFF7BFFD94F872
:104BF00038104FF48260FFF7B9FD94F8391040F295
:104C00001240FFF7B3FD94F83A1040F21440FFF75A
:104C1000ADFD94F83B1040F21640FFF7A7FD94F865
:104C20003C104FF48360FFF7A1FD94F8411040F26F
:104C30001A40FFF79BFD94F8CE1040F21C40FFF79E
:104C400095FD94F8CF1001F0010140F2AA40FFF762
:104C50008DFD8C2204F1420140F21E40FFF7A8FDB9
:104C6000164B197840F2AC40FFF780FD144B1B78CF
:104C700003F00101C3F3400341EA430140F2B640AF
:104C8000FFF774FD0F4B19784FF49760FFF76EFD37
:104C90006B210020FFF76AFD0B4B1A6922F001021D
:104CA0001A611A6942F080021A6110BD940E002048
:104CB00089888888A00E0020B40B002044020020C0
:104CC000F80500203C0200200020024030B583B0EF
:104CD0000020FFF78DFD6B2802D0002003B030BD0F
:104CE0000622C5490220FFF789FD0820FFF780FD55
:104CF000C24B18700622694640F2BA40FFF77EFDAB
:104D00009DF8002002F17E03DBB2322B08D812F0AE
:104D1000010F05D1BA4B00981860BDF804209A80A5
:104D20000A20FFF765FDB74C20800C20FFF760FDDF
:104D300060800E20FFF75CFDA0800024B24941F89E
:104D4000044FB24D45F8044F03221020FFF756FDE3
:104D5000032229461420FFF751FD1820FFF748FDD4
:104D6000C0B200F00102AA4B1A70C0F3400283F8EF
:104D70008420C0F3800283F80821C0F3C00283F8C6
:104D80008C21C0F3001283F81022C0F3401283F884
:104D90009422C0F3801283F81823C00983F89C037F
:104DA00010E004F10D004000FFF722FD41F27073A6
:104DB00003FB00F004EB4412954B03EB82035860B5
:104DC0000134E4B2072CECD900240FE004F1150003
:104DD0004000FFF70DFDC0EB0010800004EB441213
:104DE0008B4B03EB820398600134E4B2072CEDD9BE
:104DF00000240EE0642202FB04F004EB441189005D
:104E00000831834B194404313A30FFF7F7FC013481
:104E1000E4B2072CEED9002410E0C4EBC40040003B
:104E200004EB441189007031794B19440E22013191
:104E300000F25A30FFF7E2FC0134E4B2072CECD95F
:104E400040F2CA30FFF7D4FC724C94F83E3060F365
:104E5000000384F83E304FF47370FFF7C9FC84F808
:104E60003D0040F2CE30FFF7C3FCC0F30F2384F8BF
:104E70003F3084F84000052221464FF47470FFF75C
:104E8000BDFC0522A11D40F2D630FFF7B7FC05227C
:104E900004F10C014FF47770FFF7B0FC052204F128
:104EA000120140F2E230FFF7A9FC062204F11801DA
:104EB0004FF47A70FFF7A2FC062204F11E014FF4B2
:104EC0007C70FFF79BFC062204F124014FF47E70F6
:104ED000FFF794FC062204F12A014FF48060FFF7EB
:104EE0008DFC40F2AE40FFF783FC84F830004FF4B5
:104EF0009660FFF77DFC84F8310040F2B240FFF786
:104F000077FC84F8320040F2B440FFF771FC84F87B
:104F100033004FF48160FFF76BFC84F8340040F2FB
:104F20000A40FFF765FC84F8350040F20C40FFF7BB
:104F30005FFC84F8360040F20E40FFF759FC84F81D
:104F400037004FF48260FFF753FC84F8380040F2DA
:104F50001240FFF74DFC84F8390040F21440FFF78F
:104F600047FC84F83A0040F21640FFF741FC84F811
:104F70003B004FF48360FFF73BFC84F83C0040F2B9
:104F80001A40FFF735FC84F8410040F21C40FFF75F
:104F90002FFC84F8CE0040F2AA40FFF729FC94F8D9
:104FA000CF3060F3000384F8CF308C2204F142014B
:104FB00040F21E40FFF722FC40F2AC40FFF718FC25
:104FC000154B187040F2B640FFF712FC134A1378E5
:104FD00060F30003C0F3400060F3410313704FF42B
:104FE0009760FFF705FC012814BF002001200C4B3F
:104FF0001870012072E600BF240100204502002045
:105000001C01002094040020840C0020B412002015
:10501000940E0020B40B002044020020F80500206C
:105020003C02002030B400231D4601E00133DBB216
:10503000052B0ED8C1EBC1040E4A22441A4492F843
:105040004220FF2AF2D0C45CB2EB540FEED001250F
:10505000ECE7C1EBC101074B194491F84820FF2A46
:1050600004D08379603B934200D00125284630BCB0
:10507000704700BFB40B002038B5154B93F8CE3005
:1050800043FA01F111F0010F0CD005460024132C56
:1050900013D821462846FFF7C5FF034628B101343F
:1050A000E4B2F4E70023184638BD094A92F8CF204D
:1050B00012F0010FF7D10123F5E7054B93F8CF303C
:1050C00013F0010F01D00123EDE70023EBE700BF50
:1050D000B40B00200023052B18D810B51C460C4A31
:1050E00052F83320824205D00133DBB2052BF5D9CB
:1050F000002010BD064B002143F8341003EBC4041C
:105100006160044800F076FF0120F2E7002070475C
:10511000481800208CC100082DE9F04F83B00646E6
:105120008846924601939DF830709DF834909DF822
:1051300038B0072F06D8AB4B93F83F303B4113F004
:10514000010F43D1962006F09DFE0546002800F091
:1051500042810024072F06D83946F01DFFF78CFF47
:10516000002840F0388108F10601735C5B08303B91
:10517000D8B2072F16D89B4B93F83F303B4113F022
:10518000010F06D1974B93F840303B4113F0010FCC
:1051900008D0B8F10E0F40F01E81032F02D85845F9
:1051A00040F01981B9F1000F25D10023434580F06B
:1051B0008280F25CEA5401339BB2952BF6D9002D24
:1051C00000F00981284606F065FE04E10024052C64
:1051D00006D8854B53F834301BB10134E4B2F6E7FE
:1051E00000240AF10703962B00F3F58096257F4BE8
:1051F00005FB0435AEE7002353450CD2F25CEA54BC
:1052000001339BB2952BF7D9002D00F0E48028469E
:1052100006F040FEDFE0082F06D0724A92F83C20EC
:105220003A4112F0010F44D16A5C803A6A54072F68
:1052300008D86C4A92F83F2042FA07F717F0010F9E
:1052400040F082806A4AB2F8B444C4F516719A1CE0
:10525000914240F3BD80674802786749A1FB026133
:10526000490901EB8101CE00921BD2B26349019E34
:1052700041F83260624E366801EBC2014E60013285
:10528000027000227BE008EB02005E4EB65C2E54FA
:105290000132D2B2052AF6D96A5C02F001006854E4
:1052A000594A12785200D2B2203A52B202436A549A
:1052B000BDE70022EEE74B4A92F83C203A4112F05B
:1052C000010F08D1584501D000221BE0B8F10E0FA4
:1052D00001D0002216E0B9F1050F0AD85A1C49493D
:1052E00011F80910E95409F101095FFA89F993B23B
:1052F000F1E7454A12785200D2B2591C203AEA54DA
:105300008BB207220AEB02018B420CDA991A715C0C
:10531000E95401339BB2952BF4D9002D5BD028467C
:1053200006F0B8FD57E0904408F1060815F808208B
:10533000023AD2B205F8082012F01E0F7FF477AFC0
:10534000803A05F8082072E70021E954264B019ABB
:1053500043F834202A4A126803EBC40462602B48E5
:1053600000F048FE37E02249B1F8B404461CA1F829
:10537000B464AE5C014481F85C62013292B2934243
:10538000F1D81B4BB3F8B4144A1CA3F8B4240B4453
:10539000FF2283F85C221E4B1B78FBB91448B0F83F
:1053A000B414091B89B2013904F5167420442A4645
:1053B00089B20430FFF7B0F80021164800F01AFE59
:1053C0000021284600F016FE0021134800F012FECE
:1053D000284606F05FFD03B0BDE8F08F0F48FFF7E9
:1053E0006FF9DBE7B40B002048180020C41400203C
:1053F000FC05002046020020CDCCCCCC7818002043
:10540000800400202401002045020020D8C10008AB
:105410003C02002008C2000854C9000858080020B7
:105420003C4B93F83F30002B72D0F0B5B3B0002462
:1054300043E03949B1F8B4243848962707FB0507FB
:1054400017F803C08F1887F85CC20132A1F8B424A2
:105450000133DBB27345ECD32F4BB3F8B4145A18B5
:10546000FF2082F85C024A1CA3F8B4242C4B1B7862
:10547000002B47D12848B0F8B414891B89B20139F0
:1054800006F5167630446A4689B20430FFF744F8D0
:105490000021244800F0AEFD0021684600F0AAFD7E
:1054A0000021214800F0A6FD204B002243F83520C2
:1054B00003EBC5056A600134E4B2052C26D8254605
:1054C0001A4B53F83430002BF5D0194B1B68174A90
:1054D00002EBC40252689B1AB3F5FA7FEBD996200F
:1054E0000E4B00FB0430FBF7A1FE5FFA80FE0EF1CD
:1054F0000202094BB3F8B464C6F516739A4205DC90
:105500000023A7E70B48FFF7DBF8B3E733B0F0BDA4
:10551000704700BFB40B0020FC050020C41400201D
:105520003C02002024C2000854C90008481800208A
:1055300080040020580800202DE9F04F87B00D248A
:10554000035D13F0010F06D10734A4B2962CF7D9EE
:1055500007B0BDE8F08F0F46049106460E220023E7
:1055600001464FF0FF30FFF77BF8611C3A1B013A10
:10557000D3173144FFF774F880467D4B93F83F30E2
:105580000BB9002306E0FFF7A5FD0028F9D0DFE7FF
:105590000133DBB2272B14D8764A52F83320424528
:1055A000F6D1754A1168734A02EBC3025268891A30
:1055B0006F4A92F84100642202FB00F29142E7D860
:1055C000C6E70D2CC4D03357002B04DB0D2C02D0C2
:1055D000073CA4B2F7E70134A4B233199B795B0806
:1055E0000593A3F1300B5FFA8BFB0023184601E013
:1055F0000133DBB2052B07D8E218B15C5F4AD25CFD
:105600009142F5D00120F3E75D4B1B785B4501D05B
:10561000002128E008B1002125E0002302930123A6
:105620000193082300934346049A21463046FFF72E
:1056300073FD8DE70132D2B2052A0CD8A318F05CB5
:105640000B1D03EB43035F00494B3B449B5C9842BB
:10565000F0D00125EEE7464B0B4493F830305B4524
:1056600006D00131C9B2032912D800221546E3E75A
:10567000002DF6D100230293012301930B1DDBB211
:1056800000934346049A21463046FFF745FD5FE705
:10569000002741E00135EDB2B94607EB4702530060
:1056A00033481844FBF7C2FD85420CD26319F15C04
:1056B00007EB47035A002E4B13445B5D9942E9D038
:1056C0004FF0010AE6E7BAF1000F23D12544735DDC
:1056D0005B08303BDBB2059A313AD2B2062A3FF67C
:1056E00037AF002B3FF434AF072B3FF631AF9B456C
:1056F0003FF62EAF1E4A3A4492F834209A421CD309
:105700005A451AD31A4A92F83D2042FA07F919F07D
:10571000010F07D10137FFB2032F3FF619AF002564
:10572000AA46B9E702930023019300974346049ADF
:1057300021463046FFF7F0FCECE70D4A4A4492F868
:105740003820002AE6D09A42E4D8094A92F83D204F
:1057500042FA09F919F0010FDCD0029301230193F9
:1057600000974346049A21463046FFF7D5FCD1E71F
:10577000B40B0020781800208004002024010020B1
:105780004502002010B500F516701F4901440E2295
:10579000002304314FF0FF30FEF762FF0D2401E0DB
:1057A0000134A4B2184B234493F85C3213F0010F78
:1057B000F6D00134A4B20AE00134A4B201F51671A6
:1057C000114B1944012200230431FEF749FF214601
:1057D0000D4B234493F85C32FF2BEDD10B490B7832
:1057E0000B4AA2FB0342520902EB8202D4001B1BAC
:1057F000DBB2084A42F833000748006802EBC302F4
:10580000506001330B7010BDFC05002046020020E3
:10581000CDCCCCCC781800208004002084B00F4B75
:105820009A6942F020029A619A6902F0200201927C
:10583000019A9A6942F004029A619A6902F004029C
:105840000292029A9A6942F008029A619B6903F0F7
:1058500008030393039B04B0704700BF001002408D
:1058600030B5D5B0544B93F8B844002583F8B854FC
:10587000B3F85A32504AB2F858229A4215D04E49DB
:10588000C95CFF2911D05A1C92B2691C4A48C05CFD
:1058900001AB5855494BA3FB02039B094FF416700B
:1058A00000FB13239BB28DB2E4E7434BA3F85A22CB
:1058B00000239D4207D901AAD25C12F0010F02D148
:1058C00001339BB2F5E7294601A8FEF7F9FE3C4BF0
:1058D0001B78022B09D03B4B93F80432022B04D0E7
:1058E000394B93F80432022B58D127AA294601A834
:1058F000FEF712FE304AB2F8B6343449A1FB031366
:105900005B08A2F8B634642B1AD82B4BB3F8B63424
:10591000092B1AD900212E4800F06CFB14F0010F5E
:1059200018D046238DF8003014F0020F1AD0294BFE
:105930001B7813F0020F11D044238DF8013014E0CE
:105940000021254800F056FBDFE70021234800F046
:1059500051FBDFE75F238DF80030E5E750238DF83A
:10596000013002E05F238DF801300221684600F02B
:1059700041FB00211A4800F03DFB0F4BB3F8B60481
:1059800000F070FB0021174800F034FB002127A82D
:1059900000F030FB0021144800F02CFB134B93F86F
:1059A0003E3013F0010F01D155B030BD294601A89A
:1059B000FFF7C2FDF8E700BFFC050020B5814E1BD4
:1059C00085040020840C0020B4120020398EE338B6
:1059D000F0C20008F805002054C20008A0C2000868
:1059E0000CC3000820C3000854C90008B40B0020F1
:1059F00030B595B000240C940D940F941094059438
:105A000006940794089409940194029403940494CE
:105A100001220A924FF480330B930E9202251195C6
:105A200012934FF4E01313930AA8FCF715F90F2310
:105A30000593069507944FF48063089309942946CB
:105A400005A8FCF749FB10230193049401A8FCF777
:105A5000F7FB15B030BD000030B583B0FBF712FC8A
:105A6000FFF7C6FF03F00EFD8E4A936943F004036F
:105A700093618D4B5A6842F400325A605A6822F49E
:105A800040225A604FF080521A61884B1B680A33DB
:105A9000864A12689A42FBD3834B5A6822F44032FA
:105AA0005A605A6842F480225A60FFF7B7FE02F04B
:105AB000C3FC04F0C5F87E4D4FF416536B607D4C6B
:105AC00063607D4A137803F0FE036FF341031370A4
:105AD0007A4B4FF496729A801A801E225A80784B25
:105AE00083F84120FFF7F2F8FEF70CFB6A6875496E
:105AF000284603F0E3FF62687349204603F0DEFFA7
:105B00000121284603F0FCFF0121204603F0F8FFA5
:105B100003F0F4FAFEF772FC6C4B1A786C4B03FB43
:105B200002F36C4A136036E0FFF79AFE3AE06A4BE4
:105B30001B88013B694AD35CC02B50D10023684AC3
:105B40001370684A13604AE0654B01221A70654B76
:105B500000221A60634B1B681BB1544A12689342BF
:105B600047D95F4B1B78022B4ED1514B1B7A022B2E
:105B70005ED1504B1B7A022B70D1FEF7FBFB554BCD
:105B80001B681BB1494A126893427DD3474B1B687F
:105B900013F5E45F78D804F063F8534B93F8B83406
:105BA000002BC1D1FFF73CFCFEF72EFAFEF760FA9E
:105BB0004E4B1B78002BCDD04C4B00221A704C4B17
:105BC0001B782BB9394B1B6803F5FA73454A1360F0
:105BD000012000F057F9414B1B78C02BA7D03E4B5A
:105BE0001B88013B3D4AD35C0D2BADD00A2BB1D1B4
:105BF000AAE70024384B1C80FA222146374806F0D9
:105C000051F9384B1C60ACE7334D2988334C384A86
:105C1000127800920122204600F08CFB304B0222C9
:105C20001A7000212980FA22204606F03BF99CE7F1
:105C30001F4CB4F8041104F10A0594F804220092F0
:105C40000222284600F076FB022323720021A4F8EA
:105C50000411FA22284606F025F98AE7154CB4F813
:105C6000041104F10A0594F8042200920322284644
:105C700000F060FB022323720021A4F80411FA2231
:105C8000284606F00FF978E7BFF34F8F1949CA6825
:105C900002F4E062184B1343CB60BFF34F8F00BF99
:105CA000FDE700BF00100240000801408004002012
:105CB000840C0020B4120020F80500209404002079
:105CC000B40B002000380140004400404402002092
:105CD000407E050040020020900E0020B80A0020FF
:105CE0009001002048020020FC05002084040020D0
:105CF0008504002000ED00E00400FA057047000074
:105D000082B00E4B9A6942F001029A619A6902F0E0
:105D100001020092009ADA6942F08052DA61DB698E
:105D200003F080530193019B054A536823F0E0631D
:105D300043F08073536002B0704700BF0010024010
:105D400000000140BFF34F8F0549CA6802F4E062CA
:105D5000044B1343CB60BFF34F8F00BFFDE700BF81
:105D600000ED00E00400FA0508B5FFF7EBFF08B509
:105D7000FFF7E8FF08B5FFF7E5FF08B5FFF7E2FF1B
:105D800008B5FFF7DFFF70477047704708B5FBF7AE
:105D90008BFA024A13680133136008BD80040020A7
:105DA00008B50248FBF703FE08BD00BF78250020B8
:105DB00008B503460B4A126842B10A4A1068034408
:105DC0006A46934206D8074A136008BD054A064949
:105DD0001160F2E706F02CF80C2303604FF0FF305F
:105DE000F3E700BF4C020020C82C00200F4B1A68BC
:105DF00042F001021A6059680D4A0A405A601A6856
:105E000022F0847222F480321A601A6822F480220E
:105E10001A605A6822F4FE025A604FF41F029A6018
:105E2000044B4FF000629A60704700BF00100240C0
:105E30000000FFF800ED00E0BFF34F8F0549CA688E
:105E400002F4E062044B1343CB60BFF34F8F00BFFB
:105E5000FDE700BF00ED00E00400FA0500238B42DF
:105E60000DD230B4C55CD45CA54206D10133DBB29F
:105E70008B42F7D3012030BC70470020FBE70120A4
:105E80007047000070B5012804D0831EDBB2012BDF
:105E900043D970BD4F4B1B7833B34F4B1B884F4AD0
:105EA0001288934202D34C4B00211980531E4C4957
:105EB000CB5C082B1CD0494B1C88474B1888A04250
:105EC000E7D2211A464D89B2284402F025FB631E11
:105ED000EB5C0D2B01D00A2B03D10221414802F0CB
:105EE0001BFB3D4B1C80D4E73B4B00221A80D0E7C4
:105EF000012A03D8394B00221A80DCE7023A374BDB
:105F00001A800321384802F007FB334B1B88002B13
:105F1000D1D0013B304A1380CDE7032820D00123A4
:105F2000324C94F80422F2B11D462B4A32F8131079
:105F3000B4F80421914203D32749002021F813002B
:105F4000531E23449B7A082B12D0B4F80461224BD1
:105F500033F81530B34223D3204603F0B9FB98E75A
:105F60000223234CDDE71C4A002122F8131090E79E
:105F7000012A03D80023A4F80431E6E7023AA4F882
:105F8000042103221849204603F0D6FB124B33F8B4
:105F90001530002BD9D0013B0F4A22F81530D4E739
:105FA000F21A0833E11892B20231204603F0C4FB22
:105FB000731E23449B7A0D2B05D00A2B03D0064B6E
:105FC00023F81560C8E702220649204603F0B4FB17
:105FD000F5E700BF8504002054020020900E002049
:105FE000B80A002054C9000824C30008840C00200B
:105FF000B412002070B504460D46174B1B78022BD7
:1060000012D0164B93F8053223B1144B93F8043297
:10601000022B0CD0124B93F8053223B1104B93F89E
:106020000432022B0DD070BD03F06EFCE9E70B4E7D
:106030002A462146304603F07FFB304603F048FBFA
:10604000E8E7074E2A462146304603F075FB304606
:1060500003F03EFBE7E700BF85040020840C00202E
:10606000B412002038B50446154B1B78022B12D011
:10607000144B93F8053223B1124B93F80432022BE0
:106080000CD0114B93F8053223B10F4B93F8043227
:10609000022B0CD038BD03F05DFCE9E7094D214629
:1060A000284603F075FB284603F012FBE9E7064D8E
:1060B0002146284603F06CFB284603F009FBE9E77C
:1060C00085040020840C0020B412002038B5054659
:1060D000012804D9022D1BD0ADB900240CE0174BC8
:1060E000D988174803F010FCF4E7154B195D1548E3
:1060F00003F00AFB0134A4B2104BDB88A342F4D8AE
:10610000104803F0E5FA032D16D08DB9002408E0FD
:106110000024F1E70A4B195D0B4803F0F5FA01344E
:10612000A4B2064BDB88A342F4D8074803F0D0FAA8
:10613000024B0022DA8038BD0024F2E7540200202E
:10614000B8190020840C0020B4120020054BDB8815
:10615000B3F5967F04D2591C024AD180024AD0542A
:10616000704700BF54020020B819002030B4C1B9F4
:1061700003787BB1144BDA88B2F5967F0AD2531CB0
:106180009BB21149CB8010F8014B10498C54B3F5E8
:10619000967FEDD90C4BDB880C4A0021D15430BCE2
:1061A00070470D460023AB42F4D2074AD288B2F5BD
:1061B000967FEFD2541C0449CC8010F8014B034960
:1061C0008C5401339BB2EEE754020020B819002032
:1061D00010B5041E1FDB4D4B9C4220DC4C4B9C42F7
:1061E0002DDC42F20F739C423DDCB4F57A7F4EDA2F
:1061F000632C61DC092C74DC464B83FB0423E01721
:10620000C0EBA30000EB80004300E01A3030C0B2C6
:10621000FFF79CFF10BD002CB8BF6442DBE703F121
:10622000864303F5492303F6444383FB0423E01725
:10623000C0EBA3403030C0B2FFF788FFCEE736484E
:1062400080FB0430E317C3EBA043344A02FB134343
:10625000334A82FB0312D817C0EB62303030C0B231
:10626000FFF774FFBDE72E4880FB0430E317C3EB54
:1062700060332C4A02FB13432B4A82FB0312D817CC
:10628000C0EB22303030C0B2FFF760FFADE72648E8
:1062900080FB0430E317C3EB203342F2107202FBA1
:1062A0001343224A82FB0312D817C0EBA2103030EE
:1062B000C0B2FFF74BFF9BE71C4880FB0430E3179D
:1062C000C3EBA0134FF47A7202FB1343184A82FB0C
:1062D0000312D817C0EB62103030C0B2FFF736FFA0
:1062E00088E7134880FB0430E317C3EB6013642294
:1062F00002FB1343074A82FB0312D817C0EBA2002C
:106300003030C0B2FFF722FF76E700BF3F420F00F8
:106310009F8601006766666683DE1B4340420F006E
:1063200089B5F814A0860100AD8BDB68D34D6210EF
:106330001F85EB512DE9F04F89B09DF8488072B16F
:1063400014461F460E460546B44A0421FFF786FD53
:1063500058B3012C06D0022C0FD0032C19D009B051
:10636000BDE8F08F0021AE48FFF700FF0120FFF7E6
:10637000ADFEAC4B00221A70F1E70021AA48FFF7EE
:10638000F5FE0220FFF7A2FEA84B002283F80422AC
:10639000E5E70021A648FFF7E9FE0320FFF796FE98
:1063A000A44B002283F80422D9E7A34A06212846F9
:1063B000FFF754FDC0B9A14A07212846FFF74EFD5B
:1063C000002849D0012C30D0022C39D0032CC6D162
:1063D00000219B48FFF7CAFE0320FFF777FE954B8D
:1063E000022283F80422BAE700219648FFF7BEFE96
:1063F000012C0BD0022C10D0032CB0D10320FFF7BE
:1064000065FE8C4B012283F80422A8E70120FFF7E8
:106410005DFE844B01221A70A1E70220FFF756FEB1
:10642000824B012283F8042299E700218648FFF776
:106430009DFE0120FFF74AFE7A4B02221A708EE77A
:1064400000218248FFF792FE0220FFF73FFE774BC4
:10645000022283F8042282E7B8F1000F01D1002F55
:1064600051D0B8F1020F53D0B8F1010F7FF477AFDC
:10647000774A04212846FFF7F1FC002840F071819B
:10648000744A07212846FFF7E9FC002840F05882AB
:10649000714A06212846FFF7E1FC002840F05982A6
:1064A0006E4A04212846FFF7D9FC002840F05382A9
:1064B0006B4A08212846FFF7D1FC8046002840F0AF
:1064C0004E82684A05212846FFF7C8FC0746002887
:1064D00040F04982644A04212846FFF7BFFC804609
:1064E000002840F09385614A04212846FFF7B6FC56
:1064F0000746002800F0B98600230493ADF8143055
:10650000434600F073BE3146284603F06FF826E795
:10651000012FA9D14E4A04212846FFF79FFC0028ED
:1065200037D14C4A07212846FFF798FC00285ED156
:10653000494A06212846FFF791FC002860D14C4AC1
:1065400007212846FFF78AFC002800F0AF80ED798C
:10655000303DEDB2072D59D805EB45139A00454B58
:1065600013445B6833B105EB45129300414AD35C99
:10657000002B47D100214048FFF7F8FD2846FFF7E0
:1065800027FE00213D48FFF7F1FD2046FFF79EFD65
:10659000E5E600213A48FFF7E9FD00213948FFF719
:1065A000E5FD00213848FFF7E1FD2046FFF78EFDAD
:1065B00000213648FFF7DAFD00213548FFF7D6FD08
:1065C0002046FFF783FD00213248FFF7CFFD002171
:1065D0003148FFF7CBFD00213048FFF7C7FD002110
:1065E0002F48FFF7C3FD2046FFF770FDB7E60021F7
:1065F0002C4B1868FFF7BAFD2046FFF767FDAEE6A3
:10660000FFF71AFC2846FDF7B3FDA8E6002126484F
:10661000FFF7ACFD2046FFF759FDA0E628C30008B0
:1066200030C30008850400204CC30008840C0020FF
:106630006CC30008B41200208CC3000818C4000802
:1066400064C4000894C3000820C4000840C40008C3
:1066500088C4000880C6000888C6000818D0000852
:1066600020D000082CD0000890D20008C0D200082A
:1066700090C60008940E002098C60008A0C6000826
:1066800090C40008B8C40008D8C4000824C5000895
:1066900090C50008E8C5000808C600082CC6000818
:1066A0004CC6000818010020D4C60008C34A0321C4
:1066B0002846FFF7D3FB00284BD00435C04A0321FE
:1066C0002846FFF7CBFBD8B9BE4A04212846FFF77E
:1066D000C5FB00BBBC4A03212846FFF7BFFB28BB14
:1066E000BA4A04212846FFF7B9FB50B30021B84845
:1066F000FFF73CFD2046FFF7E9FC02F00FFC2EE619
:106700000021B448FFF732FD2046FFF7DFFC0120EF
:1067100002F036FC23E60021AF48FFF727FD2046B4
:10672000FFF7D4FC022002F02BFC18E60021AB4856
:10673000FFF71CFD2046FFF7C9FC032002F020FCF8
:106740000DE60021A648FFF711FD2046FFF7BEFC2D
:1067500005E60021A348FFF709FD2046FFF7B6FC38
:10676000FDE50021A048FFF701FD2046FFF7AEFC44
:1067700000219E48FFF7FAFC2046FFF7A7FC002106
:106780009B48FFF7F3FC2046FFF7A0FC0021994847
:10679000FFF7ECFC2046FFF799FC00219648FFF735
:1067A000E5FC2046FFF792FC00219448FFF7DEFC51
:1067B0002046FFF78BFC00219148FFF7D7FC2046CD
:1067C000FFF784FC00218F48FFF7D0FC2046FFF73D
:1067D0007DFC00218C48FFF7C9FC2046FFF776FCC2
:1067E00000218A48FFF7C2FC2046FFF76FFC00211A
:1067F0008748FFF7BBFC2046FFF768FC002185486F
:10680000FFF7B4FC2046FFF761FC00218248FFF748
:10681000ADFC2046FFF75AFC00218048FFF7A6FC9C
:106820002046FFF753FC00217D48FFF79FFC2046E0
:10683000FFF74CFC00217B48FFF798FC2046FFF750
:1068400045FC00217848FFF791FC2046FFF73EFC0D
:1068500000217648FFF78AFC2046FFF737FC00212D
:106860007348FFF783FC2046FFF730FC0021714896
:10687000FFF77CFC2046FFF729FC00216E48FFF75C
:1068800075FC2046FFF722FC00216C48FFF76EFCE8
:106890002046FFF71BFC00216948FFF767FC2046F4
:1068A000FFF714FC00216748FFF760FC2046FFF764
:1068B0000DFC00216448FFF759FC2046FFF706FC59
:1068C00000216248FFF752FC2046FFF7FFFB002142
:1068D0005F48FFF74BFC2046FFF7F8FB00215D48BF
:1068E000FFF744FC2046FFF7F1FB00215A48FFF771
:1068F0003DFC2046FFF7EAFB00215848FFF736FC35
:106900002046FFF7E3FB00215548FFF72FFC204608
:10691000FFF7DCFB00215348FFF728FC2046FFF778
:10692000D5FB00215048FFF721FC2046FFF7CEFBA6
:1069300000214E48FFF71AFC2046FFF7C7FB0EE583
:1069400000214B4B1868FFF711FC2046FFF7BEFBF8
:1069500005E5FFF771FAFDF7B7FFFFF76DFAFDF7F1
:1069600073FFFFF769FA00214248FFF7FFFB454636
:1069700001E00135EDB2052D07D83F4B585D4028A9
:10698000F7D04008FFF7E2FBF3E72D20FFF7DEFB2F
:106990003A4B1878FFF71CFC00213948FFF7E6FB5B
:1069A000454601E00135EDB2052D6DD8354B585DFA
:1069B0004028F7D04008FFF7C9FBF3E700C70008FD
:1069C00004C7000838C7000870C70008B4C700082B
:1069D000BCC7000808C7000840C7000874C7000803
:1069E000E0C7000804C8000834C800085CC80008F4
:1069F0008CC80008B4C80008E8C80008B8C400087B
:106A00002CC6000828C9000858C900087CC900081D
:106A100098C90008C4C90008F4C9000820CA0008C1
:106A20004CCA000888CA0008D8CA000814CB00085D
:106A300050CB0008A4CB0008F0CB000840CC0008E5
:106A400074CC0008ACCC0008ECCC000840CD0008A9
:106A500094CD0008F8CD000858CE0008B0CE00084C
:106A6000FCCE000834CF000890CF0008D4CF000837
:106A70001801002034D00008240100204502002025
:106A800040D000081C0100200021C448FFF76EFB25
:106A9000C34D2888FFF79CFB0021C248FFF766FB27
:106AA0006888FFF795FB0021BF48FFF75FFBA888C8
:106AB000FFF78EFB0021BD48FFF758FBBC4B586821
:106AC000FFF786FB0021BB48FFF750FBBA4B586825
:106AD000FFF77EFB0021B948FFF748FBB84B1B7856
:106AE00013F0010F15D00021B648FFF73FFB00213E
:106AF000B548FFF73BFBB24B1B7813F0020F0DD0EC
:106B00000021B248FFF732FB2046FFF7DFFA474685
:106B10006DE00021AE48FFF729FBE8E70021AD4812
:106B2000FFF724FBF0E70021AB48FFF71FFB79E0FC
:106B30000135EDB2052D0CD806EB46139A00A74B94
:106B400013442B4493F871002028F1D0FFF7FEFA8C
:106B5000EEE72D20FFF7FAFA730133449A009F4DB8
:106B6000154495F87700FFF733FB95F8783033B389
:106B70002C20FFF7EBFA072501E00135EDB20C2DD3
:106B80000CD806EB46139A00944B13442B4493F80D
:106B900071002028F1D0FFF7D9FAEEE72D20FFF79A
:106BA000D5FA06EB46139A008C4B134493F87E00FB
:106BB000FFF70EFB03E000218948FFF7D7FA2046D4
:106BC000FFF784FA2C20FFF7C1FA2020FFF7BEFA66
:106BD00006EB4616B3000833804818440021043001
:106BE000FFF7C4FA2046FFF771FA0137FFB2072F0B
:106BF0003BD800217B48FFF7B9FA07F13000C0B25B
:106C0000FFF7A4FA00217848FFF7B0FA3E4607EBF9
:106C100047129300714AD35C002B84D00021734843
:106C2000FFF7A4FA730133449A006C4D1544686869
:106C30006F4BA3FB0030C009FFF7CAFA00216D4873
:106C4000FFF794FAA8686C4BA3FB00304009FFF7EC
:106C5000BFFA2C20FFF77AFA2020FFF777FA95F891
:106C60007130002BA7D0454664E700216348FFF749
:106C70007DFA634B93F83E3013F0010F08D00021EA
:106C80006048FFF773FA2046FFF720FA474632E0E4
:106C900000215D48FFF76AFAF5E70135EDB2042DF2
:106CA00037D806EB46035A00554B1344585D00286D
:106CB000F3D04008FFF74AFAEFE74546EFE7002137
:106CC0005248FFF753FA33E000215148FFF74EFADC
:106CD00047E000214F48FFF749FA494B93F8CE307F
:106CE00043FA06F616F0010F4ED000214A48FFF78E
:106CF0003DFA0137FFB2032F4BD800214748FFF779
:106D000035FA3E4607EB470253003D4AD35C002B61
:106D1000D3D100213448FFF729FA394B93F83D309D
:106D2000334113F0010FCAD000213D48FFF71EFA8E
:106D3000334D05EB060999F83400FFF749FA0021B5
:106D40003848FFF713FA99F83800FFF741FA95F839
:106D50003C30334113F0010FB6D000213248FFF729
:106D600005FA274B93F83F30334113F0010FB0D1B0
:106D7000234B93F84030334113F0010FADD0002185
:106D80002A48FFF7F3F9A8E700212948FFF7EEF9B1
:106D9000AFE72046FFF79AF9474679E050D0000860
:106DA0009404002064D0000874D0000888D0000843
:106DB000840C00209CD00008B4120020B0D0000841
:106DC000F8050020C0D00008C8D00008E0D00008B6
:106DD000C4D00008E4D0000800D10008940E0020C0
:106DE00014D10008E8D0000898D00008F4D00008BA
:106DF000F11976050CD10008898888881CD1000813
:106E0000B40B00202CD1000834D1000850D1000868
:106E100070D1000880D10008A0D100083CD1000842
:106E200044D100085CD1000864D1000890D100086A
:106E3000ACD100080135EDB2052D38D806EB46037C
:106E40005A00C34B1344585D4028F3D04008FFF765
:106E50007DF9EFE74546EFE70021BE48FFF786F9E9
:106E60003CE00021BC48FFF781F942E00021BB482B
:106E7000FFF77CF9B64B93F8CE3043FA06F616F0DE
:106E8000010F49D00021B648FFF770F90137FFB272
:106E9000032F46D80021B348FFF768F9B9463E1DD5
:106EA00006EB46025300AA4AD35C002BD2D12D2018
:106EB000FFF74CF9A64DA94499F83000FFF788F97F
:106EC0000021A948FFF752F995F83D30334113F0FE
:106ED000010FC1D00021A548FFF748F99C4B93F85A
:106EE0003C30334113F0010FBBD00021A048FFF725
:106EF0003DF9974B93F83F30334113F0010FB5D173
:106F0000934B93F84030334113F0010FB2D000217E
:106F10009848FFF72BF9ADE700219748FFF726F9CE
:106F2000B4E72046FFF7D2F800219448FFF71EF996
:106F3000874D95F84100FFF74BF900219048FFF786
:106F400015F995F8CF3013F0010F09D000218D48C5
:106F5000FFF70CF900218C48FFF708F9434606E0DB
:106F600000218A48FFF702F9F4E70133DBB2132B63
:106F70000CD8C3EBC301764A0A4492F84220002A97
:106F8000F3D008F101085FFA88F8EEE7B8F1090FCD
:106F90002ED97F4DA5FB0835ED0805F13000C0B2B4
:106FA000FFF7D4F805EB85056B00A8EB030303F1AD
:106FB0003000C0B2FFF7CAF800217648FFF7D6F8D4
:106FC000754B1878D0B900217448FFF7CFF800212D
:106FD0007348FFF7CBF8734B1B78012B11D00021BE
:106FE0007148FFF7C3F82046FFF770F8FFF7B7B90D
:106FF00008F13000C0B2FFF7A9F8DDE7FFF7E8F8C5
:10700000E5E700216948FFF7B1F8ECE7002168489F
:10701000FFF7ACF83E467FE00132D2B2052A0ED827
:10702000C5EBC50C4A496144114491F84210FF294F
:10703000F2D04FF0010EEFE7BE461A46EEE7BEF182
:10704000000F07D0421C08A908443F2100F8101C7B
:10705000D0B238E0431C08AA10442A2200F8102CB1
:10706000D8B2C5EBC5053A4B1D4495F84830FF2B07
:1070700039D0002B43D0421CD5B22D2108AA02449E
:1070800002F8101C092B40F299800230C0B2404A2D
:10709000A2FB0312D20802F130010DF1200C65446D
:1070A00005F8101C02EB820251005B1A3033624675
:1070B000024402F8103C22E0411C0DF1200C604417
:1070C00000F8102CC8B20133DBB2052BC9D8C5EBD0
:1070D000C5011F4A0A441A4492F84220FF2AABD045
:1070E000202AE9D1EFE7431CDBB208AA10442D2285
:1070F00000F8102C08AA13442A2203F8102C0021AF
:1071000004A8FFF733F800212A48FFF72FF820469C
:10711000FEF7DCFF0136F6B2132E3FF620A9354606
:107120003046FFF755F800212348FFF71FF8C6EB5C
:10713000C602074B134493F84230002B44D000237F
:1071400004930593ADF818303B463846BDE700BFC1
:10715000B40B0020C4D10008CCD1000880D10008B5
:10716000A0D100083CD1000898D00008BCD100088C
:1071700074D1000890D10008ACD10008D8D1000823
:1071800000D200081CD2000834D2000828D200081F
:10719000CDCCCCCC4CD200084402002070D20008E8
:1071A0007CD200083C02002034D100082CD1000819
:1071B00098D2000854C90008B4D20008303308AA95
:1071C0002A4402F8103C9AE70021A648FEF7CEFFB9
:1071D00099E7002B42D041462FE0062B27D05200E2
:1071E00008A9084400F8102C0133DBB2062B12D892
:1071F00018465A1DAA5C0D2AEBD00A2AE9D0A2F142
:107200003001C9B20929E8D9A2F14101C9B219294D
:10721000E3D9012100E0414679B109B30021924848
:10722000FEF7A4FF2046FEF751FFFFF798B80121B3
:10723000F2E708F101085FFA88F8B8F1050FECD819
:107240008A4B402203F8082008AB434413F8103C53
:10725000002BEED0854A02F80830EAE70121DCE78E
:1072600000218348FEF782FFDCE7824A042128469A
:10727000FEF7F4FD804600284CD000230493ADF8BF
:1072800014303B460CE0002B3DD039462DE0062B58
:1072900027D0520008A8014401F8102C0133DBB2BA
:1072A000062B12D819465A1DAA5C0D2AEBD00A2AC1
:1072B000E9D0A2F13000C0B20928E8D9A2F141001A
:1072C000C0B21928E3D9012100E0394669B1E1B122
:1072D00000216948FEF74AFF2046FEF7F7FEFFF758
:1072E0003EB80121F2E70137FFB2052FEFD8634B1B
:1072F0004022DA5508AB3B4413F8103C002BF2D087
:107300005E4AD355EFE70121E1E700215848FEF737
:107310002DFFE1E75A4A04212846FEF79FFD074664
:10732000002842D00023ADF810308DF812304346CB
:10733000022B1DD819465A1DAA5C0D2A0FD00A2A05
:107340000DD0A2F13000C0B209280CD8022B0DD00C
:1073500008A8014401F8102C0133DBB2E8E753B967
:107360004FF0010810E04FF0010801E04FF0010874
:10737000B8F1000F08D1002104A8FDF767F8C0B2EA
:107380000F2804D83F4B1870B8F1000F08D0002127
:107390003D48FEF7EBFE2046FEF798FEFEF7DFBF06
:1073A00000213348FEF7E2FEF5E7384A0721284678
:1073B000FEF754FD8046002840D0002304938DF84A
:1073C00014303B46042B1BD8194603F10802AA5C73
:1073D0000D2A0FD00A2A0DD0A2F13000C0B2092820
:1073E0000BD8042B0BD008A8014401F8102C013352
:1073F000DBB2E7E72BB9012711E0012700E0012705
:107400006FB9002104A8FDF721F880B2A0F1320382
:107410009BB240F6C412934202D81D4B188047B16C
:1074200000211C48FEF7A2FE2046FEF74FFEFEF7A5
:1074300096BF00210E48FEF799FEF5E7164A062191
:107440002846FEF70BFD0746002864D0002304936E
:107450008DF81430434627E0002B3AD14FF0010855
:1074600045E000BFB8D20008C8D2000824010020BF
:10747000E0D20008E8D20008F0D200081C01002089
:1074800008D300084502002010D3000824D30008C8
:10749000940400202CD3000844D3000808A8014419
:1074A00001F8102C0133DBB2042B0FD81946DA1D7A
:1074B000AA5C0D2AD0D00A2ACED0A2F13000C0B2E8
:1074C000092820D8042BE9D14FF00108B8F1000FAA
:1074D0000DD1002104A8FCF7B9FF80B2A0F10A0386
:1074E0009BB240F6EC12934204D8B44B5880B8F1EA
:1074F000000F0BD00021B248FEF738FE2046FEF701
:10750000E5FDFEF72CBF4FF00108DFE70021AD4895
:10751000FEF72CFEF2E7AC4A05212846FEF79EFC5A
:10752000804600283FD0002304938DF814303B465A
:10753000042B18D819469A1DAA5C0D2A0FD00A2AC6
:107540000DD0A2F13000C0B209280BD8042B23D0F3
:1075500008A8014401F8102C0133DBB2E8E71BB99D
:1075600001270FE001276FB9002104A8FCF76EFF87
:1075700080B2A0F164039BB240F69212934202D80B
:107580008E4B988057B100219048FEF7EFFD2046C2
:10759000FEF79CFDFEF7E3BE0127E4E700218948E2
:1075A000FEF7E4FDF3E78A4A07212846FEF756FC7A
:1075B00038B9884A07212846FEF750FC07460028BC
:1075C0004AD000230493CDF813304346062B1BD832
:1075D000194603F10802AA5C0D2A0FD00A2A0DD021
:1075E000A2F13000C0B209280CD8062B29D008A877
:1075F000014401F8102C0133DBB2E7E73BB94FF04F
:10760000010812E04FF00108B8F1000F0DD1002180
:1076100004A8FCF71BFFA0F596626F4B9A4207D8AF
:10762000AB78312B10D16D4B5860B8F1000F0ED0F4
:1076300000216B48FEF79AFD2046FEF747FDFEF756
:107640008EBE4FF00108DFE7664B5860EDE7002182
:107650005C48FEF78BFDEFE7634A06212846FEF7FC
:10766000FDFB002800F0C88195F80780A8F13008DC
:107670005FFA88F8B8F1070F06D900215B48FEF7DA
:1076800075FD2046FEF722FD6B7A6F2B0ED1AA7A8C
:107690006E2A0BD1842303FB08F8554B012203F813
:1076A000082000214748FEF761FD25E06F2B0DD132
:1076B000AA7A662A0AD1EA7A662A07D1842303FBCA
:1076C00008F84B4B002203F80820EAE7692B02D1A7
:1076D000AA7A762A04D0642B4FD1AA7A6C2A4CD18C
:1076E000002304933B46032B0BD99FB1012FD8D124
:1076F00000214048FEF73AFD2046FEF7E7FCFEF782
:107700002EBE194603F10C02AA5C0D2A01D00A2AEA
:1077100015D183B3002104A8FCF798FEB0F5347F9F
:10772000E6D86B7A692B1CD141F2707202FB00F231
:107730002F49842303FB0818C8F80420D6E7A2F1D8
:107740003000C0B2092808D8032B08D008A801448B
:1077500001F8102C0133DBB2C5E70127C5E701278B
:10776000C3E73C2202FB00F22149842303FB0818F3
:10777000C8F80820BAE70127B8E7642B57D1AA7ADE
:10778000612A54D1EA7A742A51D12A7B612A4ED1D6
:10779000AB1913F8013C0D2B01D00A2B2ED1F3B2FB
:1077A0000F3BDBB2632B38D900211348FEF7DEFC18
:1077B0002046FEF78BFCFEF7D2BD00BF94040020EC
:1077C0004CD30008E0D2000860D3000868D300085A
:1077D00080D3000888D3000850BD0100840C00202D
:1077E00090D30008B4120020A8D30008B0D300083A
:1077F000940E0020F0D30008CCD30008F3B20E3B67
:10780000DBB2CFE707F10E02A95CB348842202FB8A
:1078100008023A4411730137FFB2BB42F2D8AE4AB4
:10782000842303FB0828474400233B7339E7702B6C
:107830007FF45EAFAB7A612B7FF45AAFEB7A742B97
:107840007FF456AF2B7B682B7FF452AFAB1913F844
:10785000023C0D2B01D00A2B1BD1F0B21038C0B264
:10786000042825D1AB7B6E2B22D1EB7B6F2B1FD154
:107870002B7C6E2B1CD16B7C652B19D10D2F0CD959
:1078800000219648FEF772FC2046FEF71FFCFEF72B
:1078900066BDF0B20F38C0B2E2E78F4A842303FB23
:1078A00008233B44002283F871200137FFB2E5E74B
:1078B00000B901270023049305930693ADF81C300B
:1078C000002F7FD0002F00F0948000218448FEF725
:1078D0004DFC2046FEF7FAFBFEF741BDBCF12C0F34
:1078E00048D0BCF10D0F45D0BCF10A0F42D00127A2
:1078F000E8E70131C9B20DF1200EF4444FF0200E3B
:107900000CF810EC8C46072938D94FF00D0EF445D1
:10791000EFDB0131C9B20DF1200EF4440CF8103C3C
:107920000A2B2ED90232D2B20132D2B29042C9D938
:10793000062E4BD802F10E03EB5C2D2B24D102F165
:107940000F03EB5C303BDBB2092B41D802F1100C8A
:1079500015F80CC0ACF1300E5FFA8EFEBEF1090FC7
:10796000BCD803EB830E4FEA4E03DBB26344DBB2B9
:10797000303BDBB20F2BC5D90127A3E74FF0060E32
:10798000C5E70132D2B2CFE72C2B19D0A3F1300CCE
:107990005FFA8CFCBCF1090F06D9A3F1410C5FFA28
:1079A0008CFCBCF1190F15D80136F6B201F1010CAF
:1079B0000DF1200E714401F8103C5FFA8CF1B3E731
:1079C0003E46B1E73A4639463E46AFE7012779E7FA
:1079D000012777E7012775E708AB3B4413F8102C24
:1079E0003D49842303FB08133B4483F8712001378E
:1079F000FFB20D2FF0D954E63A4A04212846FEF78B
:107A00002DFA0746002800F02E842B79202B12D166
:107A10006A796F2A0FD1AA796E2A0CD1324A92F86C
:107A20003E3043F0010382F83E3000212B48FEF740
:107A30009DFB00F013BC202B10D16A796F2A0DD169
:107A4000AA79662A0AD1EA79662A07D1264B93F8E1
:107A50003E206FF3000283F83E20E6E795F80580AC
:107A6000A8F130085FFA88F8B8F1090F00F23E82F9
:107A7000202B40F03B82B8F1070F08D900211B48AA
:107A8000FEF774FB2046FEF721FBFEF768BC05F10C
:107A90000709174A02214846FEF7E0F950B10123D1
:107AA00003FA08F8104A92F83D3043EA080382F8D6
:107AB0003D30BAE70F4A03214846FEF7CFF90746A3
:107AC000D0B1012303FA08F8074A92F83D3023EABF
:107AD000080382F83D30A8E7940E0020E0D20008A9
:107AE000DCD3000804D40008B40B00200CD4000838
:107AF000ACD3000828D40008B44A06214846FEF753
:107B0000ADF98246002800F0D380002302938DF85F
:107B10000C30B8F1030F5AD9AB1913F8023C0D2BF6
:107B200001D00A2B60D1F2B2103AD2B2002A5FD053
:107B3000394600230493ADF81430002900F09C80EE
:107B400000297CD1052940F29F80A8F10408A04BB0
:107B5000434483F8307068E7194603F10D02AA5CCC
:107B60000D2A01D00A2A10D1002B36D03B46042F13
:107B700023D808AA3A4412F8181C9548062202FB9A
:107B80000802D1550137FFB2F1E7A2F13000C0B2CF
:107B9000092804D9A2F14100C0B2192819D8052B2F
:107BA00019D0520008A8014401F8182C0133DBB2A7
:107BB000052BD1D93B46002BD9D083B10021854874
:107BC000FEF7D4FA2046FEF781FAFEF7C8BB3B4623
:107BD000EEE70123EFE70123EDE70123EDE70021C5
:107BE0007D48FEF7C3FAEDE7F2B20E3AD2B29DE756
:107BF00001219EE7062B41D81E4603F10D00285CAB
:107C00002D2825D10E33EF5C303FFFB2092F16D857
:107C100006F10F03EB5CA3F13002D2B2092A0AD8B5
:107C200007EB87077A00D7B21F44FFB2303FFFB29D
:107C30000F2F04D884E70D2BFAD00A2BF8D000219F
:107C40006448FEF793FA2046FEF740FAFEF787BB3A
:107C5000A0F13007FFB2092F04D9A0F14107FFB20C
:107C6000192F0ED80133DBB208AF3E4406F8100CD2
:107C70009A42BFD80F4663E70B46F9E70F4601214A
:107C80005EE70F4601215BE7514A062303FB082309
:107C900040225A5408AB0B4413F8103C2BB15B0044
:107CA0004B48062202FB080253540131C9B249E78E
:107CB0004A4A04214846FEF7D1F830B9484A04211F
:107CC0004846FEF7CBF800283AD0B8F1030F37D872
:107CD0002B7B0D2B03D00A2B01D04FF0010AEA7A3F
:107CE000A2F13003DBB2092B01D94FF0010AE97987
:107CF0006D2905D1313AD2B2062A01D94FF0010AD5
:107D0000722901D1072B02D8BAF1000F08D0002147
:107D10003448FEF72BFA2046FEF7D8F9FEF71FBBD2
:107D20006D2908D12A4A904488F8343000212A4825
:107D3000FEF71CFAEFE7264A904488F83830F5E75A
:107D4000294A05214846FEF789F830B32B7B6F2B73
:107D50000DD16A7B6E2A0AD1012303FA08F81C4A66
:107D600092F83C3043EA080382F83C305DE66F2B22
:107D700040F070826B7B662B40F06C82AB7B662B95
:107D800040F06882012303FA08F8114A92F83C3067
:107D900023EA080382F83C3047E6144A07214846A4
:107DA000FEF75CF8002839D0AB7B6F2B20D1EA7B43
:107DB0006E2A1DD1012303FA08F8054A92F8CE3045
:107DC00043EA080382F8CE302FE600BF2CD4000827
:107DD000B40B002034D40008E0D2000848D40008D6
:107DE00050D4000858D400086CD4000874D400089B
:107DF0006F2B40F02F82EB7B662B40F02B822B7C8D
:107E0000662B40F02782012303FA08F8B94A92F85A
:107E1000CE3023EA080382F8CE3006E6B64A0821BF
:107E20004846FEF71BF860B3EB7B6F2B13D12A7C1F
:107E30006E2A10D1012303FA08F35BB2AD4A92F81F
:107E40003F10194382F83F1092F8401021EA0303D3
:107E500082F84030E9E56F2B40F0FC812B7C662BEB
:107E600040F0F8816B7C662B40F0F481012303FA2B
:107E700008F8A04A92F83F3023EA080382F83F301E
:107E8000D3E59E4A07214846FDF7E8FF00283FF466
:107E9000CCADAB7B6F2B13D1EA7B6E2A10D10123C3
:107EA00003FA08F35BB2934A92F84010194382F840
:107EB000401092F83F1021EA030382F83F30B4E506
:107EC0006F2B40F0C781EB7B662B40F0C3812B7C8E
:107ED000662B40F0BF81012303FA08F8854A92F827
:107EE000403023EA080382F840309EE505F1050999
:107EF000834A07214846FDF7B1FF0746F0B10C352C
:107F0000804A05212846FDF7A9FF38B1794A92F841
:107F1000CF3043F0010382F8CF3086E57A4A05215D
:107F20002846FDF79BFF002800F09481714B93F8E1
:107F3000CF206FF3000283F8CF2076E5734A052146
:107F40004846FDF78BFF804600283ED0002304936F
:107F50003B46032B0AD997B197B300216C48FEF733
:107F600005F92046FEF7B2F8FEF7F9B9194603F114
:107F70000A02AA5C0D2A01D00A2A0DD1F3B1002110
:107F800004A8FCF763FA83B2053B9BB2FA2BE4D852
:107F9000584B83F84100DFE7A2F13000C0B2092856
:107FA00008D8032B08D008A8014401F8102C01338D
:107FB000DBB2CEE70127CEE70127CCE70127CBE7ED
:107FC00000215448FEF7D2F8CBE7534A0521484632
:107FD000FDF744FF002800F03D81AF7A303FFFB24B
:107FE000092F4CD947464FF00109EB7AA3F1300233
:107FF000D2B2092A0AD8B9F1000F07D107EB8707D7
:108000007A00D7B21F44FFB2303FFFB2132F01D91D
:108010004FF00109092F34D84FF00C0A05EB0A0381
:1080200001933E4A04211846FDF718FF83460028B5
:1080300000F0F180AB1913F8023C0D2B01D00A2B94
:1080400022D1A6EB0A03DBB2073BDBB20BB94FF040
:10805000010900220492CDF81320B9F1000F00F0BD
:10806000AE804146B9F1000F00F0B88000212C48E5
:10807000FEF77CF82046FEF729F8FEF770B9C146F6
:10808000B3E74FF00D0AC9E7A6EB0A03DBB2053BE5
:10809000DBB2DBE7013B1B1A022B43D1B31D434488
:1080A000E85CA0F13003DBB2092B1DD89DF8163037
:1080B0000344303BDBB28DF81630A2F13003DBB263
:1080C000092B14D89DF8163002EB820250000344AD
:1080D0002033DBB28DF816309DF81630DBB20F2B53
:1080E000C0D94FF00109BDE74FF00109E5E74FF0B6
:1080F0000109F1E7B40B00207CD4000888D4000803
:1081000074D4000890D4000898D40008A0D40008C3
:10811000A8D40008E0D20008C4D40008CCD40008D9
:10812000D4D40008A2F13003DBB2092B4AD89DF861
:1081300016301344303BDBB28DF8163092E73F2AFD
:108140001DD108AA1044FF2200F8102C08F10108E4
:108150005FFA88F8434585D956460AF1040240463D
:108160004244AA5C2D2AEAD1721D4244AA5C2A2A02
:1081700001D03F2A8ED1FF238DF8163072E72A2ACC
:108180000BD1414606E008AA0A44FF2002F8100C71
:108190000131C9B20529F6D9D8E7A2F13006F6B205
:1081A000092E04D9A2F14106F6B2192E04D808AE60
:1081B000304400F8102CC9E74FF00109C6E74946E2
:1081C000C846C7E74FF001094CE708AB43442022FB
:1081D00003F8102C08F101085FFA88F801EB080396
:1081E000052BF2DD4B46062B07D9B9F1000F18D14C
:1081F00000218148FDF7BAFF17E008AA1A4412F8D7
:10820000101CC7EBC7007D4A02441A4482F8421092
:108210000133DBB2E7E77A4A06210198FDF71EFE3B
:10822000A0B900217748FDF7A1FF2046FDF74EFFDA
:10823000FEF795B8C7EBC702704B13445B440022AE
:1082400083F842200BF101035FFA83FBBBF1060FB9
:10825000F0D9CAE700216C48FDF788FF2046FDF7FA
:1082600035FFFEF77CB8694A0A212846FDF7F6FD7E
:10827000002838D0002304933B46032B0AD997B13A
:1082800067B300216248FDF771FF2046FDF71EFF2E
:10829000FEF765B8194603F10A02AA5C0D2A01D05F
:1082A0000A2A07D1C3B1002104A8FCF7CFF8594B23
:1082B0001870E5E7A2F13000C0B2092808D8032BF6
:1082C00008D008A8014401F8102C0133DBB2D4E730
:1082D0000127D4E70127D2E70127D1E7002146484B
:1082E000FDF744FFD1E74C4A04212846FDF7B6FDCF
:1082F00028B30435494A02212846FDF7AFFD48B1AD
:10830000474A137843F00103137000213A48FDF700
:108310002DFF09E0434A03212846FDF79FFD40B9A0
:1083200000213848FDF722FF2046FDF7CFFEFEF77B
:1083300016B83B4B1A786FF300021A70E5E73A4A19
:1083400005212846FDF78AFD28B30535334A022169
:108350002846FDF783FD48B1314A137843F0020304
:10836000137000212448FDF701FF09E02D4A032185
:108370002846FDF773FD40B900212248FDF7F6FEBF
:108380002046FDF7A3FEFDF7EABF254B1A786FF3F1
:1083900041021A70E5E7254A08212846FDF75EFDEF
:1083A00008B308351D4A02212846FDF757FD38B1AC
:1083B0001F4B01221A7000210F48FDF7D7FE09E07C
:1083C000184A03212846FDF749FD40B900210D4810
:1083D000FDF7CCFE2046FDF779FEFDF7C0BF144B3C
:1083E00000221A70E7E700211248FDF7BFFE204681
:1083F000FDF76CFEFDF7B3BFE0D20008B40B002020
:10840000E8D40008F0D40008F0D3000808D500082C
:1084100014D500084402002030D50008ACD3000871
:10842000F805002028D4000838D5000840D50008F9
:108430003C02002004C8000808B500220F4910487B
:10844000FAF72EFE70B90F490D48FAF740FE60B9F1
:108450000D490B48FAF7DCFD50B90948FAF73EFE22
:1084600048B908BDFDF74AFCEDE7FDF747FCEFE72B
:10847000FDF744FCF1E7FDF741FCF2E77401002051
:10848000E41A0020E00000203001002000207047A6
:108490000020704770B504460D46114E0146304627
:1084A000FAF7C5FD3046FAF7E2FD00232A68934249
:1084B00014D20C4801884A1C92B20280E65C0A4839
:1084C0004654FA2A05D0094A012111700B449BB287
:1084D000ECE7044B00221A80022000E0002070BD6F
:1084E000E41A0020900E0020B80A00208404002026
:1084F00010B5064C002206492046FAF790FD0549C2
:108500002046FAF794FD002010BD00BFE41A0020B9
:1085100090210020A81D002038B5124B93F89C3202
:10852000032B01D0012038BD0E4BD3F8B852D5F83B
:108530001432012B01D90120F5E70023D5F81442AC
:108540002CB10133084CA342F8D90220EBE70A46CC
:108550000146044C2046FAF762FD2046FAF76DFD0D
:10856000E1E700BFE41A0020905F010018B1022883
:1085700003D00220704700207047012070470000A0
:1085800002680E4B9A4200D0704700B583B003F5E5
:10859000DA33DA6942F40002DA61DB6903F40003DA
:1085A0000193019B002211461420F8F7A1FE14202C
:1085B000F8F7D2FE03B05DF804FB00BF005C00409A
:1085C00008B500F50C71D0F86802FAF7A0FD08BDF7
:1085D00008B500EB4113D3F83C21D0F86802FAF754
:1085E000C3FD08BD08B500EB4113DA6BD0F8680293
:1085F000FAF703FE08BD08B5D0F86802FAF7A5FE41
:1086000008BD10B504468368022B01D0FDF776FB48
:108610000121D4F86802FAF781FED4F86802FAF76B
:1086200055FE10BD10B50446D0F86802FAF779FE81
:10863000A36923B1024A136943F00603136110BD15
:1086400000ED00E008B5D0F86802FAF773FE08BD47
:1086500010B504461D48C0F86842C4F8C0021C4B5F
:108660000360082343600223836000238361C361A6
:108670000362F8F795FE30BB182300221146D4F8A8
:10868000C002F9F7BBFA582300228021D4F8C002B7
:10869000F9F7B4FAC02300228121D4F8C002F9F717
:1086A000ADFA4FF4887300220121D4F8C002F9F723
:1086B000A5FA4FF4807300228221D4F8C002F9F7A2
:1086C0009DFA002010BDFDF719FBD5E778250020A5
:1086D000005C004008B5D0F8C002F8F7DBFEFFF7F9
:1086E00045FF08BD10B51C4613462246D0F8C0020F
:1086F000F8F7FBFEFFF73AFF10BD08B5D0F8C0024F
:10870000F8F72BFFFFF732FF08BD08B5D0F8C0021D
:10871000F9F706FAFFF72AFF08BD08B5D0F8C0023E
:10872000F9F735FAFFF722FF08BDD0F8C03211F093
:10873000800F06D101F07F0103EB411191F82A016E
:10874000704701F07F0103EB411191F82A00704757
:1087500008B5D0F8C002F8F7B4FEFFF707FF08BD70
:1087600008B5D0F8C002F8F74CFFFFF7FFFE08BDD0
:1087700008B5D0F8C002F8F71EFFFFF7F7FE08BDF6
:1087800008B5D0F8C002F8F735FF08BD00487047BB
:108790005C0200207047704712230B80004870472E
:1087A0004001002004230B80004870475401002042
:1087B0000023934216D230B40BE0373401F8134053
:1087C00000015C00013400250D550133DBB29342FA
:1087D00006D2040F092CF0D8303401F81340EFE72B
:1087E00030BC70477047000038B50B4B1868043335
:1087F0001C6804331B68C01800D138BD074D08221F
:1088000005F11A01FFF7D4FF042205F12A012046E1
:10881000FFF7CEFFF1E700BFE8F7FF1F40010020A0
:1088200008B51A230B80FFF7DFFF014808BD00BF22
:108830005801002008B50A4628B105490548FBF74C
:10884000BFF8034808BD02490248FBF7B9F8F8E74A
:10885000E42700204CD5000810B5044C0A462146F8
:108860000348FBF7ADF8204610BD00BFE427002009
:1088700054D5000808B50A4628B105490548FBF754
:108880009FF8034808BD02490248FBF799F8F8E74A
:10889000E42700204CD5000808B50A4628B1054950
:1088A0000548FBF78DF8034808BD02490248FBF76D
:1088B00087F8F8E7E42700204CD5000848B9094BB1
:1088C0004FF400521A61A3F580634FF400121A614D
:1088D0007047044B4FF000521A61A3F580632022C9
:1088E0001A617047001001402DE9F04F83B00A462D
:1088F000431003FB03F3D1E93845E61845EBE37772
:10890000C1E93867D1F8E8300133C1F8E8300D78B3
:10891000022D4BD0072308E0591E02EB4104B4F9A5
:10892000044002EB43039C80CBB2002BF4D1908037
:1089300000200BE05900984C0C44B4F9104011444D
:10894000B1F9041001FB04000133DBB2072B0BD893
:10895000002DEFD1904931F9131002EB4304B4F923
:10896000044004FB0100EFE792F85430C0130433D5
:1089700002EB8303586092F854E00EF1010EDEF131
:1089800000030EF0070E03F0070358BFC3F1000EFB
:108990005FFA8EFE82F854E000230026002730465E
:1089A000394634463D46CDE9006740E091F8543001
:1089B000043301EB83035860DDE70EEB030C0CF08E
:1089C000070C0CF1040C02EB8C0CDCF804C0DFF893
:1089D000D0A103F11E0B5AF82BB00CFB0BFBDDE909
:1089E000008918EB0B0849EBEB79CDE9008903F11D
:1089F0002E0B5AF82BB00CFB0BFB14EB0B0445EBC6
:108A0000EB7503F1160B5AF82BB00CFB0BFB10EBBC
:108A10000B0041EBEB7103F1260B5AF82BA00CFB7A
:108A20000AFC16EB0C0647EBEC770133DBB2072BA5
:108A3000C3D94FEA103848EA01580B1308FB03F377
:108A4000A8FB088909EB4309300B40EA07503B13A8
:108A500000FB03F3A0FB000101EB430110EB080A4C
:108A600041EB090BDDE90001060B46EA01560B1349
:108A700006FB03F3A6FB060101EB4301260B46EAC6
:108A800005562B1306FB03F3A6FB066707EB43070C
:108A900010EB060841EB0709D2F8F43003F100535C
:108AA000C2F8F430D94508BFD04534BF01240024B2
:108AB00092F8F850A5420DD003F10053013B374D19
:108AC000AB421CD892F8F930073382F8F930002312
:108AD000C2F8F43082F8F84092F8F930642B02D9E9
:108AE000642382F8F93092F8F9301E2B0FD992F8EE
:108AF000D83043F0010382F8D8300E231CE092F8FE
:108B0000F930002BE3D0013B82F8F930DFE792F82F
:108B1000D8306FF3000382F8D830EEE703F1FF3C62
:108B200003F10A0402EBC40430CC0B3302EBC303A1
:108B3000C3E900455FFA8CF3002BEFD1BAEB0800D4
:108B40006BEB0901C2E916010024002518E0124967
:108B500001EB4301B1F92000C11703F10B0602EB51
:108B6000C60C52F83670DCF8046000FB06F607FB12
:108B70000166A0FB0701314424184D410133DBB2EB
:108B80000E2BE4D9012C75F10003ACBF01200020AD
:108B900003B0BDE8F08F00BFD4C00008FEFFFF3F68
:108BA000E82A002020B9044B4FF400021A617047F4
:108BB000014B80221A617047000C01400000000048
:108BC00010B50C46D1F8EC20C1F8F02002F10051AC
:108BD000C4F8EC1063785B00DBB200F001000343E3
:108BE0006370002906DB637803F00303013B012B6C
:108BF00027D910BD002AF6DDA2785200D2B2A270A9
:108C000003F00703591FC9B2022901D9032B02D16E
:108C100042F00102A270A37803F00303032B00D0FB
:108C20003BB91B49611A18BF01210120FAF754FF13
:108C3000D9E71749611A18BF01210020FAF74CFF44
:108C4000D1E71348201A18BF0120FAF735FF022890
:108C50000CD0D4F8EC00F7F7CDFB00220D4BF7F762
:108C600033FCF7F7E1FEC4F8EC00C2E7D4F8EC00FF
:108C7000F7F7C0FB04A3D3E90023F7F725FCF7F7C8
:108C8000D3FEC4F8EC00B4E7AE47E17A14AEE73F98
:108C9000C02B00200000E03F014B1878704700BF58
:108CA0007C040020034B1B780BB900207047012087
:108CB000704700BFE82A002040B1094B0020002186
:108CC000C3E938010022C3F8E8207047054B0020B3
:108CD0000021C3E938010022C3F8E820704700BF33
:108CE000E8290020C02B002038B598B1134CD4E9F6
:108CF0003801F7F7D9FF0546D4F8E800F7F7C2FFC7
:108D000001462846F8F7CAF801F0ECF9F8F714FA2A
:108D100080B238BD0A4CD4E93801F7F7C5FF0546E3
:108D2000D4F8E800F7F7AEFF01462846F8F7B6F8A2
:108D300001F0D8F9F8F700FA80B2EAE7E829002054
:108D4000C02B0020684620F007018D4679B52C4BDA
:108D50001B6813F0200F03D1BDE8794085467047AA
:108D6000274A536843F020035360264BB3F844204E
:108D7000B3F846401444B3F848201444B3F84A30DA
:108D80001C446410A4F6FF7424B21F4D29462046EB
:108D9000FFF7AAFD29460028D4BF00200120FFF7D5
:108DA0000FFF1A4E31462046FFF79EFD3146002840
:108DB000D4BF00200120FFF703FF95F8D83013F04F
:108DC000010F16D196F8D83013F0010F11D10E4BC8
:108DD00093F8D83013F0010FBED10C4B93F8D83074
:108DE00013F0010FB8D10020094B1870FFF766FD92
:108DF000B2E70120064B1870FFF760FDACE700BF3B
:108E000000000240E82A0020C02B0020E8290020B2
:108E10007C040020684620F007018D4601B4194A01
:108E2000136923F001031361174A92F842300133AA
:108E3000DBB282F8423092F8423003F01F0382F82E
:108E40004230124B1B7813F0010F11D1104BDA682E
:108E500022F47042DA600C4A92F8421002EB4102AE
:108E60005188DA6842EA0132DA6001BC854670470F
:108E7000134692F8422003EB42035B889BB2054AFB
:108E80005363F2E7002C0140E82A0020F805002097
:108E9000000C014000080040684620F007018D46A4
:108EA00001B51B4A136923F001031361194B1B78A9
:108EB000BBB1184A92F84C30B3FA83F35B0982F8DD
:108EC0004C30144B93F84C30C3B9134A002353620F
:108ED000104B93F85230DBB2D362BDE801408546B7
:108EE0007047FAF747FF0028EBD10A4A92F84C3056
:108EF000B3FA83F35B0982F84C30E2E7064A0023B9
:108F00005362044B93F85330DBB2D362E5E700BF02
:108F100000040040E82A0020002C014008B5002091
:108F2000144B1870144A136823F00103136002F500
:108F30009432136823F0010313604FF080421368EA
:108F400043F0010313600D4B4FF00052C3F8802033
:108F5000BFF34F8FBFF36F8F4FF00072C3F88020C5
:108F6000BFF34F8FBFF36F8F4FF480521A60FFF73C
:108F700019FE08BDE82A00200004004000E100E0DE
:108F800010B50446244B1B78002B33D10120FFF78A
:108F900009FE214B1C70214B11229A620122DA60DA
:108FA0001A6842F001021A604FF08042136823F001
:108FB000010313601A4B4FF48052C3F88020BFF3B3
:108FC0004F8FBFF36F8F4FF000721A60012C14D0D7
:108FD000022C19D0134B47229A620121D9600E4A04
:108FE000B2F8542092B2DA6219600D4B4FF0005281
:108FF0001A6010BDFFF792FFC8E7074B93F8523095
:10900000DBB2064AD362F4E7034B93F85330DBB28A
:10901000024AD362EDE700BFE82A0020002C01409D
:1090200000E100E00004004008B50120FFF7BAFDB0
:10903000154A11239362D36843F00103D360134BA5
:1090400047219962D96841F00101D9601049B1F80E
:10905000541089B2D9620121196011604FF0804229
:10906000136823F0010313600A4B4FF48052C3F8D6
:109070008020BFF34F8FBFF36F8F4FF000721A60E5
:109080004FF000521A6008BD002C0140000400405F
:10909000E82A002000E100E008B54FF080421368A4
:1090A00043F00103136002F58062136823F00103AB
:1090B000136002F59432136823F0010313600D4B23
:1090C0004FF00072C3F88020BFF34F8FBFF36F8F54
:1090D0004FF00052C3F88020BFF34F8FBFF36F8F64
:1090E0004FF480521A600020FFF75CFD024B2C22E7
:1090F0005A6308BD00E100E00008004070B5AE4BC7
:109100009A6942F008029A619A6942F010029A61E3
:109110009A6942F004029A61DA6942F00102DA6166
:10912000DA6942F00202DA619A6942F400629A61F5
:109130009A6942F400729A615A6942F001025A61D6
:109140009E4A516841F400115160516821F4801128
:109150005160516821F440015160A2F5806251686C
:1091600089B25160516841F0085141F408115160D1
:109170009349086820F00C000860086820F003009C
:109180000860116841F000511160116821F08051B0
:109190001160116821F040411160116841F4001123
:1091A0001160116821F480111160116821F44001EF
:1091B00011605A6842F400425A605A6822F48042B0
:1091C0005A60A3F56C439A6842F002029A609A686A
:1091D00042F460229A60DA6A22F47002DA621A6952
:1091E00042F004021A615A6B22F01F025A639A6815
:1091F00042F001029A609A6842F008029A60714B4C
:109200009B6813F0080FFAD16E4A936843F0040389
:1092100093606C4B9B6813F0040FFAD1694B9A680A
:1092200042F480129A609A6842F480029A6003F5D0
:109230005C431C331A6842F480621A601A6822F494
:1092400000621A601A6842F480721A601A6822F486
:1092500000721A601A6842F0A2021A6004225A6070
:10926000594A9A60594ADA60196841F00101196057
:10927000574B4FF4805119604FF080431121996290
:10928000D96841F48071D9606720D862196841F0CB
:1092900001011960A2F144039073372283F853202F
:1092A0004FF45072A3F85420002443E02046F7F70F
:1092B000E9FC4849F7F73EFD4FF07851F7F73AFDE2
:1092C000054600F0FBFC4449F7F734FDF7F70EFFC5
:1092D000424E04F11E0346F82300284600F02AFD02
:1092E0003D49F7F727FDF7F701FF04F12E0346F894
:1092F00023003B492846F7F71DFD3A49F7F7CEFD15
:10930000054600F0DBFC3449F7F714FDF7F7EEFEF5
:1093100004F1160346F82300284600F00BFD2E4901
:10932000F7F708FDF7F7E2FE04F1260346F82300FD
:109330000134E4B2072CB9D900241BE02046F7F72A
:10934000A1FC2449F7F7F6FC4FF07451F7F7F2FC53
:1093500000F0F0FC2449F7F7EDFC4FF08241F7F7FD
:10936000E1FBF7F7E9FE80B21C4B03EB44035880A6
:109370000134E4B21F2C3DD81C4B1B7813F0010FB5
:10938000DCD02046F7F77EFC1249F7F7D3FC4FF00C
:109390007451F7F7CFFC00F0CDFC4FF07E51F7F79A
:1093A000C1FB1349F7F7C6FCF7F7C6FE80B20B4BBB
:1093B00003EB44035880DBE700100240001001403B
:1093C00000080140002401404C2401402C2B0020C7
:1093D00000E100E0F90FC94000F07F45E82A0020D5
:1093E00000800945000096440000E040F805002098
:1093F000000034421E4B1B7813F0020F31D01D4B7E
:1094000002221A701C4B01221A70194B1B7813F0A0
:10941000010F25D0194AD36943F00403D361184BD7
:109420001A6842F000621A601A6842F040721A60CC
:109430001A6822F080621A60A3F5823307229A62CA
:109440005A22DA629A6942F060029A611A6A42F01C
:1094500001021A622C225A631A6842F001021A6051
:1094600070BD044B02221A70034B00221A70CCE725
:10947000F8050020C02B0020E82900200010024041
:10948000000C01400A4B1B680A4AA2FB03235B093C
:10949000013BB3F1807F09D2074A5360074BF021AB
:1094A00083F823100023936007231360704700BFE5
:1094B0002C0100201F85EB5110E000E000ED00E0E2
:1094C00010B5044603681A6812F0200F26D01A68F7
:1094D00022F020021A6002685068B4F80431E118E2
:1094E00088720133A4F804313C4B9A4252D03C4B71
:1094F0009A4253D0B4F804213A4BA3FB02131B0940
:10950000FA2101FB1323A4F8043194F804322BB997
:10951000354B1B6803F5FA73C4F8083223681A68E0
:1095200012F0100F12D05A68B4F804218AB3A17A4D
:10953000C02937D0013A2244927A0D2A01D00A2A52
:1095400004D1012222720022C4F808221A6812F003
:10955000800F17D0B4F80022B4F802128A422BD040
:10956000511CA4F80012224492F806215A60B4F863
:1095700000221C4BA3FB02131B09FA2101FB13233E
:10958000A4F80032D4F808321BB1174A126893428B
:1095900019D910BD0220FCF775FCABE70320FCF7DE
:1095A00071FCA7E7511E2144897AC029C2D100214C
:1095B0002172C4F80812BDE700226272DA6822F054
:1095C0008002DA60DEE70021C4F80812A4F8041172
:1095D000FA2204F10A0002F065FCDAE700380140E3
:1095E00000440040D34D62108004002009294CD96A
:1095F0002DE9F0410E46054600242146274621E08C
:10960000022C1DD902291BD1DFF88880B8F8B434A8
:109610005A1CA8F8B4244344FF2283F85C2238463D
:10962000FCF7B0F8B8F8B424C2F51672331B023355
:109630009A422CDB032103E04B1EDBB2012B15D930
:109640000134A4B2B4421DD228192B5DC02BD7D04F
:10965000002BF1D1621EAB5CC02BEDD109B1032907
:10966000EAD10C4BB3F8B4740121E9E7094BB3F824
:10967000B424511CA3F8B4140178134483F85C1289
:109680000221DDE70020BDE8F081012070470020C5
:10969000F9E700BFFC050020684620F007018D4671
:1096A00001B50348FFF70CFFBDE801408546704750
:1096B000840C0020684620F007018D4601B5034860
:1096C000FFF7FEFEBDE8014085467047B41200205A
:1096D00090F805323BB1012343720268D36843F02E
:1096E0008003D3607047B0F80232A0F800327047B0
:1096F00000B583B002AB03F8040D01211846FEF754
:109700000BFF03B05DF804FB10B4437A012BFCD0CF
:10971000B0F80242631C9AB2044484F80611054B67
:10972000A3FB02131B09FA2101FB1323A0F8023249
:1097300010BC7047D34D621070B4164622B1437A04
:10974000012BFCD000221CE08B5D002BF7D00136F2
:10975000B6B2FA2EF8D1F2E7B0F802526B1C9CB206
:10976000A0F802428B5C054485F80631074BA3FB49
:1097700004531B09FA2505FB1343A0F802320132FA
:1097800092B2B242E8D370BC704700BFD34D6210B2
:1097900038B505460C1E23DB002CB8BF6442504B85
:1097A0009C4221DC4F4B9C422FDC42F20F739C42C7
:1097B00040DCB4F57A7F52DA632C66DC092C7ADC63
:1097C000494B83FB0423E117C1EBA30101EB8101AA
:1097D0004B00E11A3031C9B22846FFF795FF38BD7A
:1097E0002D21FFF791FFD7E703F1864303F54923C6
:1097F00003F6444383FB0423E117C1EBA34130315B
:10980000C9B22846FFF780FFCCE7384981FB043115
:10981000E317C3EBA143364A02FB1343354A82FBED
:109820000312D917C1EB62313031C9B22846FFF7B4
:109830006BFFBAE72F4981FB0431E317C3EB6133B8
:109840002D4A02FB13432D4A82FB0312D917C1EBA9
:1098500022313031C9B22846FFF756FFA9E7274920
:1098600081FB0431E317C3EB213342F2107202FB98
:109870001343234A82FB0312D917C1EBA2113031E3
:10988000C9B22846FFF740FF96E71D4981FB043126
:10989000E317C3EBA1134FF47A7202FB1343194A87
:1098A00082FB0312D917C1EB62113031C9B22846CD
:1098B000FFF72AFF82E7134981FB0431E317C3EB6B
:1098C0006113642202FB1343074A82FB0312D91778
:1098D000C1EBA2013031C9B22846FFF715FF6FE78F
:1098E0003F420F009F8601006766666683DE1B436A
:1098F00040420F0089B5F814A0860100AD8BDB68EB
:10990000D34D62101F85EB512DE9F04180460F4683
:1099100011B9F7F78BFC87B23E4600242546AF42CB
:1099200015D9272E0DD904EB8403D80028214044F3
:10993000FEF7F2FD0134E4B2283EB6B22835ADB2EE
:10994000EDE7791B89B208EB0500FEF7E5FDBDE800
:10995000F081000010B5041E22DB002CB8BF644269
:109960004C4B9C4220DC4C4B9C422DDC42F20F7352
:109970009C423DDCB4F57A7F4EDA632C61DC092C25
:1099800074DC464B83FB0423E017C0EBA30000EB21
:1099900080004300E01A3030C0B2FFF7A9FE10BDCE
:1099A0002D20FFF7A5FED8E703F1864303F54923F1
:1099B00003F6444383FB0423E017C0EBA34030309D
:1099C000C0B2FFF795FECEE7354880FB0430E317C1
:1099D000C3EBA043334A02FB1343334A82FB031217
:1099E000D817C0EB62303030C0B2FFF781FEBDE760
:1099F0002D4880FB0430E317C3EB60332B4A02FB96
:109A000013432B4A82FB0312D817C0EB22303030AD
:109A1000C0B2FFF76DFEADE7254880FB0430E317C9
:109A2000C3EB203342F2107202FB1343214A82FB44
:109A30000312D817C0EBA2103030C0B2FFF758FEA7
:109A40009BE71C4880FB0430E317C3EBA0134FF4E3
:109A50007A7202FB1343184A82FB0312D817C0EB39
:109A600062103030C0B2FFF743FE88E7124880FB37
:109A70000430E317C3EB6013642202FB1343074A6D
:109A800082FB0312D817C0EBA2003030C0B2FFF740
:109A90002FFE76E73F420F009F86010067666666ED
:109AA00083DE1B4340420F0089B5F814A0860100F5
:109AB000AD8BDB68D34D62101F85EB5170B504464A
:109AC000016042600223037200254572A0F8045130
:109AD000A0F80052A0F8025280F8045280F8055213
:109AE000C0F80852FA26324629460A3002F0DAF95E
:109AF0003246294604F5837002F0D4F970BD0000A7
:109B000003684A4A934203D0494A934246D0704779
:109B100002F55842936943F480439361454B5A6878
:109B200042F020025A605A6822F040025A605A6895
:109B300042F080025A605A6842F480625A605A6861
:109B400022F400625A6042683B4B1B68B3FBF2F39D
:109B5000364A936089B1D36843F4005343F03C0321
:109B6000D360364B202283F8252371B15A6000312F
:109B700018BF012180F8051270472C4AD36823F4DE
:109B8000005323F03C03D360EBE72C4B2022C3F8B7
:109B90008420BFF34F8FBFF36F8FE8E702F5E63203
:109BA000D36943F40033D361224B1A6842F4007244
:109BB0001A601A6822F480621A601A6842F400621D
:109BC0001A601A6842F480421A601A6822F400424D
:109BD0001A6043685A00184B1B68B3FBF2F3144A2F
:109BE000936091B1D36843F4005343F03C03D360D6
:109BF000124B202283F8262379B140225A6000318B
:109C000018BF012180F8051281E7094AD36823F4BF
:109C1000005323F03C03D360EAE7084B4022C3F82B
:109C20008420BFF34F8FBFF36F8FE8E70038014008
:109C300000440040000801402C01002000E100E049
:109C4000064B45F255521A6005225A6040F6FF72E3
:109C50009A604CF6CC421A60704700BF003000405A
:109C6000024B4AF6AA221A60704700BF003000403B
:109C7000002103E00B4B5B58435004310A480B4B67
:109C800042189A42F6D30A4A02E0002342F8043B03
:109C9000084B9A42F9D3FCF7A9F802F0CFF8FBF78A
:109CA000DBFE704760D9000800000020F8010020AA
:109CB000F8010020C42C0020FEE7000000B51C4A7B
:109CC00020F00043934283B018DDB3F1FF4F05DB72
:109CD0000146F6F725FF03B05DF804FB694601F085
:109CE00087F800F00302012A0ED0022A18D092B1A0
:109CF00001220199009801F067FEECE7002101F0D4
:109D00003DFA03B05DF804FB0199009801F05CFE98
:109D100000F10040DFE70199009801F02FFADAE73F
:109D20000199009801F02AFA00F10040D3E700BF42
:109D3000D80F493F00B51D4A20F00043934283B03D
:109D400019DDB3F1FF4F05DB0146F6F7E9FE03B07D
:109D50005DF804FB694601F04BF800F003000128B0
:109D600010D0022819D090B10199009801F006FA9C
:109D700000F10040EBE70022002101F025FE03B0D6
:109D80005DF804FB0199009801F0F8F9DFE7012282
:109D90000199009801F018FED9E701220199009875
:109DA00001F012FE00F10040D1E700BFD80F493F9B
:109DB0002DE9F04F8DB006460F4614461D4600F0C3
:109DC000E3F9DFF81493CDE9000199F90080B8F1C7
:109DD000FF3F36D022462B4620462946F6F70EFE98
:109DE000834670BB32463B4630463946F6F706FEA0
:109DF0008246002840F0AD803046394600220023DC
:109E0000F6F7CAFD10B30022002320462946F6F7D4
:109E1000C3FD8346002869D0012200200021A94B00
:109E2000CDF828A0CDE90467CDE90645CDE90801C4
:109E3000CDE90223B8F1000F42D00023A24CCDE9B6
:109E40000034DDE900010DB0BDE8F08FDDE900016F
:109E500001F034FE8046002800F09880DDE9000122
:109E60004FF0000A4FF0000B52465B46F6F794FDA8
:109E70000028E6D03046394601F020FE0028E0D028
:109E80002046294601F01AFE0028DAD004200021DD
:109E900099F900308B4A022BCDE90467CDE90645DC
:109EA000CDE908AB02900A91039204D002A801F018
:109EB0000BFE002842D101F0BBFF222303603DE0EE
:109EC00002A801F001FE002800F0B3800A9B002BDD
:109ED0003AD001F0ADFFDDE90834CDE900340A9B4A
:109EE0000360DDE900010DB0BDE8F08F2046294692
:109EF00001F0E4FD0028A4D00022002320462946DA
:109F0000F6F754FD00289CD001216E4A99F90030E3
:109F1000CDF828B0CDE90467CDE90645CDE90212B8
:109F2000002B00F08B8000206849022BCDE908014E
:109F300040F0888001F07CFF212303600A9B1BB165
:109F400001F076FF0A9B0360DDE90834CDE90034B7
:109F500077E70022002320462946F6F71DFD00285A
:109F60003FF46FAF01200022574B5649B8F1020F62
:109F7000CDF828B0CDE90467CDE906450290CDE9DA
:109F8000082303919CD1CDE900235AE73046394696
:109F900001F094FD00283FF461AF2046294601F00E
:109FA0008DFD00283FF45AAFDDE900231046194625
:109FB000F6F724FD99F900A0002868D10323DFF803
:109FC00004C10A902946204602930022404BCDE965
:109FD0000645CDE90467CDF80CC0F6F775FA0446DE
:109FE0000D46BAF1000F34D14FF0604ADFF8ECB003
:109FF0000022002330463946CDE908ABF6F7D6FCFF
:10A0000000283FF453AF2046294601F065FD224663
:10A010002B46F6F7C1FC002836D14FF060422D4B9D
:10A0200099F900A0CDE90823BAF1020F3FF443AF3C
:10A030003CE701F0FDFE2123036047E700230024F5
:10A04000CDE9083402A801F03FFD00287FF476AF87
:10A0500070E74FF0000BDFF888C000220023304685
:10A060003946CDE908BCF6F7A1FC0028DCD0204633
:10A07000294601F031FD22462B46F6F78DFC18B932
:10A080000022124BCDE9082399F900A0CCE7012268
:10A090000C4BCDF82880CDE90467CDE90645CDE924
:10A0A0000223BAF1000FC9D000220023104619463E
:10A0B000F6F734FBBAF1020FCDE908013FF43AAFED
:10A0C000C0E700BF68D500080000F03F0000F0FFC7
:10A0D0000000E03FFFFFEFC791010020FFFFEF47C7
:10A0E0000000F07FF0B58BB0044600F0F3FF234B87
:10A0F000064693F900506B1C0AD021462046F6F71D
:10A10000DFFF074620B900212046F6F7B1FF10B95E
:10A1100030460BB0F0BD0122194B2046CDE900239B
:10A120000897F6F779F90022CDE90401CDE902019B
:10A130000023ADB110461946F6F7F0FA022DCDE92D
:10A1400006010FD101F074FE21230360089B7BB947
:10A15000DDE90601F6F790FC064630460BB0F0BD8F
:10A16000CDE90623684601F0AFFC0028EED1E9E70F
:10A1700001F05EFE089B0360EAE700BF910100204A
:10A180006CD50008000000002DE9F04F23F00045D9
:10A1900055EA020493B00DD0794E21F00044B44248
:10A1A0000F4682460FDD04F1404404F5801454EA62
:10A1B0000A035BD10023734CCDE90034DDE90001D3
:10A1C00013B0BDE8F08F984694464ED0B542EADC15
:10A1D0006B4EB54266D0002F8B468146CDE90223F7
:10A1E00064DB0026BCF1000F0ED1654B9D4246D0CA
:10A1F000644B9D4200F09780B8F1804F00F0B28030
:10A20000614B984500F0D2834846594601F052FC14
:10A21000CDE90001BAF1000F06D1002C60D0594BF6
:10A2200027F040429A425BD0FF0F013F56EA0703F6
:10A2300000F08280554B9D4240F3B08003F10473DF
:10A240009D4240F34E84524B9C4240F38280B8F1D1
:10A25000000F40F3828048A3D3E90023104619463B
:10A26000F6F732F9CDE90001A8E728B1494813B063
:10A27000BDE8F04F01F02ABCA542F7DCA8E704F1E5
:10A28000404303F5801353EA0A0393D0404B9C42AA
:10A2900040F39683B8F1000F5FDBDDE90234CDE9CE
:10A2A00000348BE7BCF1000F95D07CE73A4B9D4220
:10A2B00037DCA3F154739D4293DD2B15A3F2FF33DA
:10A2C000142B40F3ED83C3F134032CFA03F202FAAA
:10A2D00003F3634585D102F00102C2F1020681E772
:10A2E000B8F1000F07DADDE9002300202549F6F771
:10A2F00015FACDE90001002FBFF660AF04F140442C
:10A3000004F5801454EA060300F04984012E7FF41A
:10A3100055AFDDE90045224605F10043CDE90023B4
:10A320004CE702265EE7B8F1000FC0F255834846BD
:10A330005946CDE9000141E74A4648465B46594641
:10A34000F5F70AFF02460B46F6F7E8F9CDE90001FA
:10A3500034E7B8F1000FFFF67EAF00230024CDE90B
:10A3600000342BE74A4648465B465946F6F7ACF8B8
:10A37000CDE9000122E700BF9C7500883CE4377EF0
:10A380000000F07F0000F03F0000E03F0000E041EF
:10A39000FFFFEF3F7CC60008FFFF3F43B4F5801F7F
:10A3A00080F29C83DDE900010022D14BF6F78CF8A6
:10A3B0006FF0340C0C46CDE900012315CD4AC4F3EF
:10A3C0001304A3F2FF3344F07F5503EB0C019442D6
:10A3D0000D9145F4401540F37383C74B9C4240F305
:10A3E0000084002300240022CDE90A34CDE9103492
:10A3F0000024C24B0131CDE906230D91A5F580154E
:10A40000DDE906ABDDE9000152465B4629468046A0
:10A41000F5F7A2FE5246CDE908015B4640462946C3
:10A42000CDE906ABF5F79AFE02460B460020B3498C
:10A43000F6F774F90A4601461346CDE90E120246B4
:10A44000DDE90801F6F740F80A4683469446002302
:10A4500001460020CDE900BC00936B1043F000538F
:10A4600003F50023CDE90412DDE900AB1919A94673
:10A4700004460D4602460B4650465946F6F724F868
:10A4800002460B46DDE90801F5F766FEDDE9062325
:10A49000CDE9080120462946F5F75EFE02460B4647
:10A4A00040464946F5F758FE52465B46F6F70CF82B
:10A4B00002460B46DDE90801F5F74EFEDDE90E2305
:10A4C000F6F702F8DDE90445CDE9060122462B4600
:10A4D00020462946F5F7F8FF73A3D3E90023044685
:10A4E0000D46F5F7F1FF72A3D3E90023F5F736FE29
:10A4F00022462B46F5F7E8FF6FA3D3E90023F5F7D3
:10A500002DFE22462B46F5F7DFFF6DA3D3E900238E
:10A51000F5F724FE22462B46F5F7D6FF6AA3D3E9CA
:10A520000023F5F71BFE22462B46F5F7CDFF68A367
:10A53000D3E90023F5F712FE2246804689462B46D2
:10A5400020462946F5F7C0FF02460B4640464946DD
:10A55000F5F7BAFF04460D46DDE9040152465B46B5
:10A56000F5F7FCFDDDE90623F5F7AEFF22462B46A5
:10A57000F5F7F4FD5246804689465B4650465946FB
:10A58000F5F7A2FF00225E4BCDE90801F5F7E6FDE5
:10A5900042464B46F5F7E2FD00980D4604462B4631
:10A5A000224650465946F5F78FFF002282468B46D9
:10A5B000534B20462946F5F7CFFDDDE90823F5F793
:10A5C000CBFD02460B4640464946F5F7C5FDDDE9A1
:10A5D0000423F5F779FF224680468946DDE9060126
:10A5E0002B46F5F771FF02460B4640464946F5F704
:10A5F000B5FD8046894602460B4650465946F5F75A
:10A60000ADFD35A3D3E9002300980D460446F5F7C8
:10A610005BFF5246CDE904015B4620462946F5F72B
:10A620009BFD02460B4640464946F5F795FD2CA397
:10A63000D3E90023F5F748FF2BA3D3E90023804695
:10A64000894620462946F5F73FFF02460B4640461D
:10A650004946F5F783FDDDE91023F5F77FFD8046D8
:10A660000D988946F5F7C6FE82468B46DDE9040162
:10A6700042464B46F5F772FDDDE90A23F5F76EFD1C
:10A6800052465B46F5F76AFD009852465B46044623
:10A690000D46F5F761FDDDE90A23F5F75DFDDDE91E
:10A6A00004232FE0AFF30080EF4E454A287ECA3FD7
:10A6B00065DBC9934A86CD3F01411DA96074D13F36
:10A6C0004D268F515555D53FFFAB6FDBB66DDB3F48
:10A6D000033333333333E33F000000E009C7EE3F79
:10A6E000FD033ADC09C7EE3FF5015B14E02F3EBEE7
:10A6F000000040438E98030079B60B000000F03F45
:10A7000000000840F5F728FD0B4602464946404642
:10A71000F5F722FD0022013E56EA070314BFDA4B8B
:10A72000DA4B8B46CDE90423DDE9021200230E4605
:10A730001746CDE900670093DDE9006782463B4696
:10A74000084611463246F5F707FD22462B46F5F737
:10A75000BBFEDDE902238046894650465946F5F79F
:10A76000B3FE02460B4640464946F5F7F7FC8046E5
:10A77000894632463B4620462946CDE90289F5F70F
:10A78000A3FE0B46024606460F4640464946F5F7ED
:10A79000E5FCBF4B044699420D468A4640F32681AC
:10A7A00001F13F4303F5E003034340F0FE81A2A320
:10A7B000D3E90023DDE90201F5F7D0FC32468046FB
:10A7C00089463B4620462946F5F7C6FC02460B461D
:10A7D00040464946F6F708F9002840F0E681A846C9
:10A7E0004FF4801300204FEA2852A2F2FE321341A8
:10A7F0005344C3F30A52A74DA2F2FF321541C3F3EB
:10A80000130423EA0501C2F1140B44F48014BAF1D5
:10A81000000F02460B4644FA0BFB30463946B8BFE0
:10A82000CBF1000BF5F798FC06460F46DDE9020177
:10A8300032463B46F5F792FC0D464FEA0B5A002490
:10A840007FA3D3E9002320462946F5F73DFE324693
:10A85000804689463B4620462946F5F77DFC024660
:10A860000B46DDE90201F5F777FC77A3D3E9002376
:10A87000F5F72AFE76A3D3E9002306460F462046C5
:10A880002946F5F721FE02460B4630463946F5F7D4
:10A8900065FC06460F4602460B4640464946F5F71C
:10A8A0005DFC42464B4604460D46F5F755FC024614
:10A8B0000B4630463946F5F74FFC2246804689461E
:10A8C0002B4620462946F5F7FFFD63A3D3E9002375
:10A8D00006460F46F5F7F8FD61A3D3E90023F5F727
:10A8E0003BFC32463B46F5F7EFFD5FA3D3E900237F
:10A8F000F5F734FC32463B46F5F7E6FD5CA3D3E9B9
:10A900000023F5F729FC32463B46F5F7DDFD5AA357
:10A91000D3E90023F5F722FC32463B46F5F7D4FD98
:10A9200002460B4620462946F5F716FC06460F461A
:10A9300002460B4620462946F5F7C6FD0022CDE922
:10A9400000014FF0804330463946F5F705FC0246DA
:10A950000B46DDE90001F5F7E1FE424606460F46EB
:10A960004B4620462946F5F7AFFD42464B46F5F7E4
:10A97000F5FB02460B4630463946F5F7EDFB22461D
:10A980002B46F5F7E9FB02460B4600203E49F5F75A
:10A99000E3FB8A44BAF5801FC0F235815146DDE9F8
:10A9A0000423F5F791FDCDE9000107E4002FFFF640
:10A9B0002BAC4846594613B0BDE8F04F00F056B9ED
:10A9C000B8F1000FBFF6C9ACDDE90234009304F121
:10A9D00000430193FFF7F2BB4A465B4600202A4939
:10A9E000F5F79CFECDE90001FFF7E8BB2A4B21F00B
:10A9F0000048984540F3E980284B0B4403430AD1B3
:10AA000032463B46F5F7A8FBDDE90223F5F7E2FF06
:10AA100000283FF4E5AE1AA3D3E90023DDE90401E1
:10AA2000F5F752FD16A3D3E90023F5F74DFDCDE967
:10AA30000001FFF7C3BB00BFFE822B654715973CA3
:10AA400000000000432EE63FEF39FAFE422EE63FBB
:10AA5000396CA80C615C20BED0A4BE726937663E1A
:10AA6000F16BD2C541BDBB3E2CDE25AF6A56113F0E
:10AA700093BDBE166CC1663F3E5555555555C53FF5
:10AA800059F3F8C21F6EA5010000F03F0000F0BFAF
:10AA9000FFFF8F40FFFF0F00FFCB904000346F3F60
:10AAA000BCF1000F40F09A80C3F1140345FA03F2A1
:10AAB00002FA03F3AB4200F0AA806646FFF798BBA8
:10AAC000002300241A462346CDE90A23CDE91023AA
:10AAD0000022614B0024CDE9062391E44FF0000CE5
:10AAE0006BE45E4B9C427FF734AC5B4B9C423FF780
:10AAF000AEABDDE900010022574BF5F72DFB48A373
:10AB0000D3E9002304460D46F5F7DEFC46A3D3E95E
:10AB1000002382468B4620462946F5F7D5FC0022C5
:10AB2000CDE900014E4B20462946F5F7CDFC024603
:10AB30000B463FA1D1E90001F5F70EFB22462B465B
:10AB4000F5F7C2FC02460B4600204649F5F704FB28
:10AB50002246804689462B4620462946F5F7B4FC16
:10AB600002460B4640464946F5F7AEFC32A3D3E910
:10AB70000023F5F7A9FC02460B46DDE90001F5F7D5
:10AB8000EBFA02460B468046894650465946F5F791
:10AB9000E5FA00200D46044652465B46B2E5DDE983
:10ABA000002310461946FFF7CBBB25A3D3E90023AA
:10ABB000DDE90401F5F788FC21A3D3E90023F5F7CB
:10ABC00083FCCDE90001FFF7F9BA264B98453FF722
:10ABD00007AEDDE900239246934630E60026FFF7F4
:10ABE00013BB19A3D3E90023CDE90A2318A3D3E9A2
:10ABF0000023CDE9102300221B4B4FF48024CDE924
:10AC00000623FFF7FDBB5A4600F0F2FFC7E602F04D
:10AC10000102C2F10206FFF7EBBA00BFAFF30080FA
:10AC2000000000604715F73F44DF5DF80BAE543E6F
:10AC3000555555555555D53FFE822B654715F73F60
:10AC40009C7500883CE4377E0000004003B8E23F7A
:10AC500006D0CF43EBFD4C3E0000F03FFEFFEF3F40
:10AC60000000D03F0000E03F0000F83F5F4A2DE9C0
:10AC7000F0418A430D46074600F0948000290B46B8
:10AC80000446064654DD0F1500F0A780C3F31303F6
:10AC9000A7F2FF3743F48013F20FF80702EB4303E8
:10ACA0004FEA460503D5ED0F05EB4303B50000263B
:10ACB0001622B4464FF400117F100CEB01009842AD
:10ACC0004FEAD5744FEA450503DC1B1A00EB010C73
:10ACD0000E44013A04EB43034FEA5101EDD1104613
:10ACE000964620244FF0004209E052D05B00013C20
:10ACF00003EBD5734FEA52024FEA450537D063455F
:10AD000002EB0E01F1DD002901EB020E0ADBE04649
:10AD1000A3EB0C03A94288BF03F1FF33C4466D1AAD
:10AD20001044E3E7BEF1000FF1DB0CF10108EFE79F
:10AD300021F00042024329D0002945D10146CA0A28
:10AD4000153B4905002AFAD012F4801001D048E0E2
:10AD500030465200D40200F10106F9D5C6F12004B4
:10AD600001FA06F6E1401F1A41EA02038EE72B437F
:10AD700024D14408731003F17F53F20703F5001345
:10AD800048BF44F0004403EB075127463846BDE86E
:10AD9000F081A942AAD8002901EB020EC2DB984635
:10ADA0000023BBE702460B46F5F78EFB3A462B46DF
:10ADB000F5F7D4F907463846BDE8F081411C16BFC7
:10ADC000421C01365408D5E70246F5F7C5F902469C
:10ADD0000B46F5F7A3FC0746D8E71A4621463B4643
:10ADE000B2E70E4620244FF0FF30BBE70000F07FB3
:10ADF0002DE9F04FAA4A20F00044944289B06FDD5B
:10AE0000A84A064694420D461CDC002824F00F0494
:10AE1000A5496DDDF5F784FEA44B06469C4200F083
:10AE2000E980A349F5F77CFE014630462960F5F735
:10AE300077FE9F49F5F774FE01276860384609B030
:10AE4000BDE8F08F9B4A944268DDB4F1FF4F80F279
:10AE5000CA80E715863FA4EBC7542046F6F746F9AB
:10AE6000F5F714FF0346204619460593F5F758FEFB
:10AE70004FF08741F5F75EFF8046F6F737F9F5F7B3
:10AE800005FF0446404621460694F5F749FE4FF07B
:10AE90008741F5F74FFF00210790F6F7DFF800280C
:10AEA00000F0DB8020460021F6F7D8F8002814BF18
:10AEB00001230223022080493A46CDE900012946B8
:10AEC00005A800F01FFA002E07460DDAD5E9002389
:10AED00002F1004203F1004347422A606B6003E045
:10AEE0000022002708604A60384609B0BDE8F08FAC
:10AEF000F5F718FE6D4B06469C4200F09B806C49AE
:10AF0000F5F710FE014630462960F5F709FE68495D
:10AF1000F5F708FE4FF0FF376860E5E700F0DAFE6E
:10AF200066498046F5F706FF4FF07C51F5F7FAFDCC
:10AF3000F6F7DCF80746F5F7A9FE5B498346F5F717
:10AF4000F9FE01464046F5F7EBFD59498146584662
:10AF5000F5F7F0FE1F2F8246014648465CDDF5F707
:10AF6000DFFD8046E215C8F3C753D31A082B5EDD18
:10AF7000534958460392F5F7DDFE804601464846A0
:10AF8000F5F7CEFD014604464846F5F7C9FD4146B2
:10AF9000F5F7C6FD80464B495846F5F7CBFE4146CE
:10AFA000F5F7BEFD014682462046F5F7B9FD039A46
:10AFB000C0F3C753D21A192A804650DCA146286034
:10AFC00041464846F5F7ACFD5146F5F7A9FD002E80
:10AFD000686089DA08F1004800F10040C5F8008097
:10AFE00068607F4280E70146F5F79AFD00276860B8
:10AFF000286079E73249F5F793FD32490446F5F7C1
:10B000008FFD014620462960F5F78AFD2D49F5F7A9
:10B0100087FD0127686067E7F5F782FD2A4B7A1EF6
:10B0200053F8223024F0FF029A4280469AD0C5F8A5
:10B030000080C5E72249F5F775FD22490446F5F77A
:10B0400071FD014620462960F5F76AFD1D49F5F7B7
:10B0500069FD4FF0FF37686046E703232AE71B4985
:10B060005846F5F767FE804601462046F5F758FD3D
:10B07000014681462046F5F753FD4146F5F750FD60
:10B08000044613495846F5F755FE2146F5F748FDA5
:10B09000014682464846F5F743FD8046C7E700BFB4
:10B0A000D80F493FE3CB1640800FC93FD00FC93FAF
:10B0B00043443537800F4943F4D5000884F9223FD3
:10B0C0000044353708A3852E74D5000800A3852ECB
:10B0D00032318D2420F00042B2F1FF4FF8B5044622
:10B0E0003AD2C2B3002803463DDBB2F5000F4FEA67
:10B0F000E0500AD214F4000201D03BE00A465B00A3
:10B100001C0202F10101F9D5801A0026C3F31603CF
:10B110007F3843F40002C1074FEA42034FF019049D
:10B1200048BF930031464FF0807247108D189D4202
:10B1300002DC5B1BA9181644013C4FEA43034FEAAB
:10B140005202F3D113B1013626F00106701000F15E
:10B150007C5000EBC750F8BD0146F5F7EBFD2146EA
:10B16000F5F7E0FCF8BD0146F5F7DAFC0146F5F726
:10B1700095FEF8BD4FF0FF32C6E700BF2DE9F8435A
:10B1800020F00045B5F1485F06460F4649DAF5F76D
:10B19000ADFF002800F0998031463046F5F7CAFD32
:10B1A00004464E49F5F7C6FD4D49F5F7BBFC21466F
:10B1B000F5F7C0FD4B49F5F7B3FC2146F5F7BAFDAD
:10B1C0004949F5F7AFFC2146F5F7B4FD4749F5F7D6
:10B1D000A7FC2146F5F7AEFD4549F5F7A3FC21464E
:10B1E000F5F7A8FD80464FF07C512046F5F7A2FD0B
:10B1F000414605462046F5F79DFD39460446304652
:10B20000F5F798FD01462046F5F78AFC01462846E9
:10B21000F5F786FC01464FF07E50F5F781FCBDE85E
:10B22000F8830146F5F786FD04462C49F5F782FDC3
:10B230002B49F5F777FC2146F5F77CFD2949F5F711
:10B240006FFC2146F5F776FD2749F5F76BFC2146A3
:10B25000F5F770FD2549F5F763FC2146F5F76AFD22
:10B260002349F5F75FFC2146F5F764FD214B804645
:10B270009D42B8DD204B9D422BDC05F17F452946E0
:10B280004FF07E50F5F74CFC81464FF07C51204644
:10B29000F5F750FD2946F5F743FC414605462046A3
:10B2A000F5F748FD394604463046F5F743FD0146BB
:10B2B0002046F5F735FC01462846F5F731FC0146F6
:10B2C0004846F5F72DFCBDE8F8834FF07E50BDE809
:10B2D000F883DFF82C90094DD7E700BF4ED747AD74
:10B2E000F6740F317CF29334010DD037610BB63A0E
:10B2F000ABAA2A3D9999993E0000483F0000903E34
:10B300000000383F2DE9F04F1C46DDB00B91611E67
:10B31000019107936699C74B064653F82130049371
:10B32000D31E48BF131DDB1023EAE3714B1CA2EBB5
:10B33000C3030593049A019B0991CF1AD31818D41B
:10B340003B4400255C1C0DF18008DDF89C9108E071
:10B3500059F82700F5F79AFC0137A74248F8040B83
:10B3600007D0002FF4DA28460137A74248F8040B2B
:10B37000F7D1049B002BC0F2FD824FF00009079B20
:10B38000321F9B000499D518039220AA89000693C6
:10B39000D61849AB029103EB010848AF019B002B83
:10B3A000C0F29F81B246CB46039C5AF8041D54F864
:10B3B000040FF5F7BFFC01465846F5F7B3FBAC4266
:10B3C0008346F2D147F804BB474506F10406E5D1B0
:10B3D00006990398029A01440D460DF1300AA2F134
:10B3E000080353440A930BAB1344049C0893A30033
:10B3F0005CAA0293002C134453F850BC22DD57463C
:10B400000DF5907808EB84064FF06E515846F5F72D
:10B4100091FCF5F76BFEF5F739FC4FF0874181465B
:10B42000F5F788FC01465846F5F77AFBF5F75EFE1E
:10B4300056F8041D47F8040B4846F5F773FB4645DC
:10B440008346E1D1059F5846394600F08BFC4FF00A
:10B4500078510646F5F76EFC00F040FC4FF0824153
:10B46000F5F768FC01463046F5F75AFB0646F5F756
:10B470003DFE8346F5F70AFC01463046F5F750FBE2
:10B48000002F064640F3CF80611E5AF82130C7F1E5
:10B49000080843FA08F202FA08F8A3EB0803C7F118
:10B4A00007084AF82130934443FA08F8B8F1000F2E
:10B4B00029DD002C0BF1010B40F34582DAF8007016
:10B4C000002F40F09780012C0AD05146012251F8FC
:10B4D000047F531C002F40F08F809C421A46F6D107
:10B4E000059B002B0BDD012B00F09781022B06D171
:10B4F000621E5AF8223003F03F034AF82230B8F1B6
:10B50000020F00F0D78000213046F5F7A7FD002894
:10B5100000F0A180049B671EBB420FDC002204F1F7
:10B520008043013B08980AEB830353F804198342D4
:10B5300042EA0102F9D1002A40F0DC80049B013B81
:10B540005AF82330002B40F0C9804FF001080A9BC5
:10B5500053F8042908F10108002AF9D008EB040384
:10B5600004F101099945069339DC099A079909EB19
:10B57000020602EB030B06F18046679B013E03EBDC
:10B58000860648AB03EB8909679B0C4403EB8B03EE
:10B5900020A901EB8404029356F8040FF5F776FB1B
:10B5A0002746019B47F8040B002B1ADBDDF80CB093
:10B5B0004FF00008043C01E054F804095BF8041F54
:10B5C000F5F7B8FB01464046F5F7ACFAAB458046C7
:10B5D000F2D1029B49F8048B9E423C46DCD1069C8A
:10B5E00005E74FF00008029B49F8048B9E423C4659
:10B5F000D2D1F4E701230022C7F580779C424AF8B4
:10B6000022700EDD02995AF82320514489460AEB34
:10B61000830300E01A68C2F1FF0243F8042B4B4594
:10B62000F8D101275CE707D1631E5AF823304FEAAF
:10B6300023283BE738D900084FF07C51F5F72CFD63
:10B64000002840F07981804600213046F5F706FD5C
:10B6500000287FF45FAF059B30465942CDF8088043
:10B6600000F080FB4FF087410546F5F715FD0028F7
:10B6700000F06B814FF06E512846F5F75BFBF5F754
:10B6800035FDF5F703FB4FF087410646F5F752FB12
:10B6900001462846F5F744FAF5F728FD4AF8240054
:10B6A0003046F5F723FD059B671C083305934AF8E0
:10B6B000270033E031464FF07E50F5F731FA064669
:10B6C000002F3FF420AF05994FF07E5000F04AFB69
:10B6D00001463046F5F724FA064614E74FF0010814
:10B6E0003CE7CB4647F804BB474506F104067FF428
:10B6F00055AE6DE6059A5AF82730083ACDF808801D
:10B7000005925BB907F18043013B0AEB830353F8D1
:10B710000419013F083A0029F9D0059205994FF024
:10B720007E5000F01FFB002F0446C0F22C814FF02A
:10B730006E564FEA870848AA08F10403904406931E
:10B740000AEB030908F1040559F8040DF5F79EFA10
:10B750002146F5F7EFFA314645F8040D2046F5F796
:10B76000E9FAD1450446EFD134AB00269A467A1C5B
:10B77000DDF810900393A8F104080192CDF814B0FD
:10B780000497B9F1000FC0F2D5808D4DC3468D48A6
:10B790000027002403E0B4420DDC55F8040F5BF8E9
:10B7A000041FF5F7C7FA01463846F5F7BBF901342F
:10B7B000A1450746EFDA019B01369E424AF8047B19
:10B7C000A8F10408DDD1DDE9047B669B032B1FD8BB
:10B7D000DFE803F09A87872B029B0020002B40F0C4
:10B7E000BB800B9B014618603498F5F799F9002F40
:10B7F0000CDD012434AD013455F8041FF5F792F93E
:10B80000A742F8DA029B002B40F0B1800B9B5860F6
:10B810000BF007005DB0BDE8F08F621E5AF82230D1
:10B8200003F07F034AF8223069E6002F40F3C58019
:10B83000BD005CAB2B4453F8A08C34AB9A46039309
:10B840005C1954F8049C41464846F5F76BF90646E6
:10B8500001464846F5F764F94146F5F763F920607B
:10B8600044F8046DA245B046EBD1012F40F3A5800A
:10B87000039B35AF5E1934465CAB1D4455F8A08C74
:10B8800054F8049C41464846F5F74CF905460146F4
:10B890004846F5F745F94146F5F744F9206044F884
:10B8A000045DA742A846EBD10020039D043608356D
:10B8B00056F8041DF5F736F9B542F9D10299349AD4
:10B8C000359B29B102F1004203F1004300F1004031
:10B8D0000B9988600BF007000A604B605DB0BDE813
:10B8E000F08F002FFFF678AF002034AD05EB870412
:10B8F000043454F8041DF5F715F9A542F9D1029B5B
:10B90000002B3FF46EAF27E0069B00201C46039DF2
:10B910002C4454F8041DF5F705F9A542F9D1029B12
:10B920000BB100F100400B9B18600BF007005DB0FD
:10B93000BDE8F08F00273EE7002C0BF1010B33DD53
:10B940004FF00208BAE50027CAE52846F5F7CEFB16
:10B9500027464AF82400E1E60B9A00F1004301462D
:10B9600013603498F5F7DCF8002F3FF742AF00F191
:10B9700000404BE7331F0393079B9B000693049BF8
:10B980009B00029324E5669B032B3FF641AF01A287
:10B9900052F823F0A5B90008E3B80008E3B800089E
:10B9A0002BB800080020BAE731464FF07E50F5F77B
:10B9B000B7F84FF002080646A5E500207EE700BF75
:10B9C0000CD900080000C93F2DE9F84320F00043DE
:10B9D000B3F1485F04460F46904603DAF5F786FB5D
:10B9E000002858D021462046F5F7A4F9054601461F
:10B9F0002046F5F79FF9294906462846F5F79AF9B2
:10BA00002749F5F78DF82946F5F794F92549F5F713
:10BA100089F82946F5F78EF92349F5F781F8294683
:10BA2000F5F788F92149F5F77DF88146B8F1000F5F
:10BA300022D04FF07C513846F5F77CF949468046D4
:10BA40003046F5F777F901464046F5F769F829469B
:10BA5000F5F770F93946F5F763F8154905463046AC
:10BA6000F5F768F901462846F5F75CF801462046E7
:10BA7000F5F756F8BDE8F88301462846F5F75AF978
:10BA80000B49F5F74DF83146F5F754F92146F5F72E
:10BA900049F8BDE8F8832046BDE8F883D3C92E2FC6
:10BAA000342FD7321BEF3836010D50398988083CC6
:10BAB000ABAA2A3E21F000431946704741F00041ED
:10BAC00001F58010C00F7047002070470020014929
:10BAD000704700BF0000F87F2DE9F041C1F30A571D
:10BAE000A7F2FF35132D82B002460B460C464FEAF3
:10BAF000D178064632DC002D4DDB3B49294103EA73
:10BB00000100104325D049080B4052EA03060BD030
:10BB10004FF48023132D0CBF4FF00046002624EA7B
:10BB2000010143FA05F40C433049234601EBC808F0
:10BB3000D8E90045324620462946F4F70FFBCDE907
:10BB40000001DDE9000122462B46F4F705FB024621
:10BB50000B461046194602B0BDE8F081332D07DDD3
:10BB6000B5F5806FF5D1F4F7F9FA02460B46F0E728
:10BB70004FF0FF31A7F21347F9400842E9D04908D6
:10BB80000842D1D04FF0804320EA010143FA07F781
:10BB900041EA0706C8E721F000410143D9D0C3F3C9
:10BBA00013031E4373423343640C1B0B640403F4FE
:10BBB000002343EA04010B460C4901EBC801D1E91B
:10BBC000004520462946F4F7C9FACDE90001DDE930
:10BBD000000122462B46F4F7BFFA21F0004102464D
:10BBE00041EAC873B5E700BFFFFF0F0048D900085E
:10BBF000F8B5C1F30A5304460D460E4617460BBB73
:10BC0000034621F0004633431BD02F4B0022F4F7AC
:10BC10005BFC2E4B04469F420D4637DB0E46C1F3BC
:10BC20000A53363B40F2FE723B4493421ADC002B2F
:10BC300011DD26F0FF4626F4E00646EA03552046CD
:10BC40002946F8BD40F2FF729342EBD102460B4603
:10BC5000F4F784FAF8BD13F1350F1DDA4CF25033C6
:10BC60009F420CDD14A1D1E9000122462B4600F0D1
:10BC7000D1F811A3D3E90023F4F726FCF8BD22463E
:10BC80000FA1D1E900012B4600F0C4F80CA3D3E9C1
:10BC90000023F4F719FCF8BD26F0FF4626F4E00671
:10BCA000363346EA0355204629460022084BF4F76E
:10BCB0000BFCF8BDAFF300809C7500883CE4377E38
:10BCC00059F3F8C21F6EA50100005043B03CFFFFBE
:10BCD0000000903C20F00040704700BF2DE9F0418B
:10BCE00020F00047FC0D7F3C162C054618DC002C8C
:10BCF000804620DB184F2741384214D01749F4F70B
:10BD000011FF0021F5F7D2F968B1002D04DA4FF4E4
:10BD1000000343FA04F4A04428EA0700BDE8F081D8
:10BD2000B7F1FF4F02D22846BDE8F0810146F4F793
:10BD3000F9FEBDE8F0810949F4F7F4FE0021F5F7BA
:10BD4000B5F90028EFD0002D01DB0020ECE7002F33
:10BD5000E9D00348E8E700BFFFFF7F00CAF249715E
:10BD6000000080BF10B50C4630F00041034610D0F3
:10BD7000B1F1FF4F0ED2B1F5000F0FD30246C80D3F
:10BD80002044FE281EDC002824DD22F0FF4242EA87
:10BD9000C05010BD0146F4F7C5FE10BD4FF09841EC
:10BDA000F4F7C8FF184A0346944207DB0246C0F383
:10BDB000C7501938E4E7154800F034F81349F4F790
:10BDC000B9FF10BD1946124800F02CF81049F4F7DD
:10BDD000B1FF10BD10F1160F0BDA4CF25032944245
:10BDE0001946E8DD0A4800F01DF80949F4F7A2FFFA
:10BDF00010BD22F0FF42193042EAC0504FF04C51C2
:10BE0000F4F798FF10BD00BFB03CFFFF6042A20DE9
:10BE1000CAF2497103F0004321F0004242EA0301F3
:10BE2000704700BF01F0004120F000400843704718
:10BE3000014B1868704700BF9401002070B50025C1
:10BE40000C4E0D4CA41BA410A54209D100F01EF904
:10BE500000250A4E0A4CA41BA410A54205D170BDB2
:10BE600056F8253098470135EEE756F825309847C3
:10BE70000135F2E758D9000858D9000858D9000808
:10BE80005CD90008024B0146186800F05FB800BF9B
:10BE900094010020024B0146186800F00BB800BF67
:10BEA0009401002003460244934200D1704703F8F6
:10BEB000011BF9E738B50546002943D051F8043C89
:10BEC0000C1F002BB8BFE41800F0DEF81E4A136800
:10BED000104633B9636014602846BDE8384000F06E
:10BEE000D4B8A3420BD921686218934201BF1A68E3
:10BEF0005B685218226063600460EDE713465A687D
:10BF00000AB1A242FAD919685818A0420BD1206888
:10BF10000144581882421960DED110685268014409
:10BF200019605A60D8E702D90C232B60D4E7206847
:10BF300021188A4201BF11685268091821606260A5
:10BF40005C60C9E738BD00BF8804002070B5CD1C17
:10BF500025F0030508350C2D38BF0C25002D0646AD
:10BF600001DBA94203D90C233360002070BD00F02F
:10BF70008BF8214A1468214691B9204C23681BB9DB
:10BF8000304600F071F820602946304600F06CF829
:10BF9000431C24D10C233046336000F076F8E4E7EC
:10BFA0000B685B1B18D40B2B0FD90B60CC18CD5032
:10BFB000304600F06AF804F10B00231D20F0070062
:10BFC000C31AD3D05A42E250D0E74B688C4216BF16
:10BFD000636013600C46EBE70C464968CCE7C41C71
:10BFE00024F00304A04205D0211A304600F03CF8AA
:10BFF0000130CFD02560DBE7880400208C040020CE
:10C0000038B5134B1C68A36B7BB91820FFF73AFFB8
:10C01000104A114BA063C0E90023104B012283603A
:10C020000B2383810023C0E90423A16B0C480A6918
:10C030004B6950430B4C04FB0300A2FB0423034455
:10C04000541C43F10005C1E9044525F0004038BD0A
:10C05000940100200E33CDAB34126DE6ECDE05000A
:10C060002DF451582D7F954C38B50023054C0546CD
:10C0700008462360F9F79CFE431C02D1236803B1F4
:10C080002B6038BDC02C002070477047F8B500BF4A
:10C09000F8BC08BC9E467047F8B500BFF8BC08BCA9
:04C0A0009E46704701
:10C0A80002030405060708090A0B0C0D0E0F1010F1
:10C0B800010200000000000000000000010203046B
:10C0C800060708090000000001020304D80296CB05
:10C0D800D6FD254CD6FD96CBD8023808EFD69AD592
:10C0E80075254C5D75259AD5EFD691FC10E8AAE820
:10C0F80039F61D108731A052E46ACB73E46AA05266
:10C1080087311D1039F6AAE810E800002841582E9A
:10C11800323529205472616E736D697474696E6763
:10C1280020626561636F6E200000000056502D4448
:10C1380069676920762E20312E322E350D0A546813
:10C1480065206F70656E2D736F75726365207374EB
:10C15800616E64616C6F6E65204150525320646952
:10C16800676970656174657220636F6E74726F6C55
:10C178006C657220616E64204B49535320544E43C2
:10C188000D0A00004469676970656174656420661A
:10C1980072616D652072656365697665642C2064DB
:10C1A800726F7070696E67206F6C64206672616D63
:10C1B800652066726F6D20766973636F75732D6481
:10C1C800656C6179206275666665720D0A0000000B
:10C1D800536176696E67206672616D6520666F725D
:10C1E80020766973636F75732D64656C617920645B
:10C1F80069676970656174696E670D0A00000000FF
:10C208002841582E32352920446967697065617460
:10C21800696E67206672616D653A20002841582E64
:10C22800323529205472616E736D697474696E6752
:10C2380020766973636F75732D64656C61796564C5
:10C24800206672616D653A20000000000D0A496E93
:10C25800707574206C6576656C20746F6F206869E2
:10C2680067682120506C6561736520726564756329
:10C278006520736F206D6F73742073746174696FB8
:10C288006E73206172652061726F756E642035303F
:10C298002D3730252E0D0A000D0A496E7075742051
:10C2A8006C6576656C20746F6F206C6F77212050F9
:10C2B8006C6561736520696E63726561736520736F
:10C2C8006F206D6F73742073746174696F6E73205F
:10C2D8006172652061726F756E642035302D37305C
:10C2E800252E0D0A000000002841582E323529203D
:10C2F8004672616D65207265636569766564205B69
:10C30800000000005D2C207369676E616C206C650D
:10C3180076656C2000000000253A200008200800FF
:10C328006B6973730000000055534220737769747A
:10C338006368656420746F204B495353206D6F64A4
:10C34800650D0A005541525431207377697463684A
:10C35800656420746F204B495353206D6F64650DDD
:10C368000A0000005541525432207377697463689B
:10C37800656420746F204B495353206D6F64650DBD
:10C388000A000000636F6E6669670000537769747E
:10C398006368656420746F20636F6E666967757281
:10C3A8006174696F6E206D6F64650D0A4D6F7374EB
:10C3B8002073657474696E67732077696C6C207478
:10C3C800616B652065666665637420696D6D696477
:10C3D800696174656C792C206275740D0A72656DDB
:10C3E800656D62657220746F20736176652074686C
:10C3F8006520636F6E66696775726174696F6E2018
:10C408007573696E67202273617665220D0A0000D4
:10C418006D6F6E69746F720055534220737769743B
:10C428006368656420746F206D6F6E69746F722025
:10C438006D6F64650D0A00005541525431207377C1
:10C4480069746368656420746F206D6F6E69746FBA
:10C4580072206D6F64650D0A00000000554152544A
:10C468003220737769746368656420746F206D6F18
:10C478006E69746F72206D6F64650D0A00000000AC
:10C4880068656C70000000000D0A436F6D6D616E89
:10C498007320617661696C61626C6520696E206DDC
:10C4A8006F6E69746F72206D6F64653A0D0A0000D3
:10C4B80068656C70202D2073686F777320746869C5
:10C4C800732068656C7020706167650D0A00000054
:10C4D80063616C207B6C6F777C686967687C616CD2
:10C4E800747C73746F707D202D207472616E736D0F
:10C4F8006974732F73746F7073207472616E736DC7
:10C5080069747465722063616C6962726174696FC1
:10C518006E207061747465726E0D0A00096C6F7715
:10C52800202D207472616E736D697473204D4152B1
:10C538004B20746F6E652C2068696768202D207405
:10C5480072616E736D697473205350414345207452
:10C558006F6E652C20616C74202D207472616E736F
:10C568006D69747320616C7465726E6174696E674D
:10C5780020746F6E657320286E756C6C20627974F8
:10C588006573290D0A000000626561636F6E203CC7
:10C59800626561636F6E5F6E756D6265723E202DB8
:10C5A80020696D6D6564696174656C792074726168
:10C5B8006E736D6974732073656C6563746564204C
:10C5C800626561636F6E20286E756D6265722066A4
:10C5D800726F6D203020746F2037290D0A0000001B
:10C5E8006B697373202D2073776974636865732092
:10C5F800746F204B495353206D6F64650D0A00001A
:10C60800636F6E666967202D207377697463686548
:10C618007320746F20636F6E666967206D6F646541
:10C628000D0A00007265626F6F74202D20726562BA
:10C638006F6F747320746865206465766963650D2F
:10C648000A00000076657273696F6E202D2073688A
:10C658006F77732066756C6C206669726D7761728E
:10C66800652076657273696F6E20696E666F0D0A54
:10C678000D0A0D0A0000000076657273696F6E007E
:10C688007265626F6F740000626561636F6E20008F
:10C69800426561636F6E2000206E6F7420656E6165
:10C6A800626C65642E2043616E6E6F7420747261D3
:10C6B8006E736D69742064697361626C656420626D
:10C6C8006561636F6E732E0D0A0000004265616339
:10C6D8006F6E206E756D626572206D757374206261
:10C6E800652077697468696E20302D372072616E15
:10C6F80067650D0A0000000063616C006C6F7700CD
:10C708005374617274696E67206C6F7720746F6EF2
:10C71800652063616C6962726174696F6E207472FE
:10C72800616E736D697373696F6E0D0A00000000A6
:10C7380068696768000000005374617274696E6705
:10C74800206869676820746F6E652063616C696230
:10C75800726174696F6E207472616E736D69737340
:10C76800696F6E0D0A000000616C74005374617289
:10C7780074696E6720616C7465726E6174696E6746
:10C7880020746F6E65732063616C6962726174698D
:10C798006F6E207061747465726E207472616E734E
:10C7A8006D697373696F6E0D0A00000073746F70A2
:10C7B8000000000053746F7070696E672063616CCD
:10C7C8006962726174696F6E207472616E736D69EB
:10C7D8007373696F6E0D0A0055736167653A20635C
:10C7E800616C207B6C6F777C686967687C616C74AE
:10C7F8007C73746F707D0D0A00000000556E6B6EBF
:10C808006F776E20636F6D6D616E642E20466F7258
:10C8180020636F6D6D616E64206C69737420747928
:10C828007065202268656C70220D0A000D0A436F3E
:10C838006D6D616E647320617661696C61626C65AF
:10C8480020696E20636F6E666967206D6F64653A54
:10C858000D0A00007072696E74202D207072696E66
:10C86800747320616C6C20636F6E666967757261A2
:10C8780074696F6E20706172616D65746572730D95
:10C888000A0000006C697374202D207072696E7440
:10C89800732063616C6C7369676E2066696C74657C
:10C8A80072206C6973740D0A00000000736176656C
:10C8B800202D20736176657320636F6E66696775D6
:10C8C800726174696F6E20616E64207265626F6F49
:10C8D800747320746865206465766963650D0A0061
:10C8E8006572617365616C6C202D2065726173657A
:10C8F8007320616C6C20636F6E6669677572617412
:10C90800696F6E7320616E64207265626F6F7473F5
:10C9180020746865206465766963650D0A00000007
:10C9280076657273696F6E202D2073686F77732038
:10C9380066756C6C206669726D77617265207665C4
:10C948007273696F6E20696E666F0D0A0D0A0000BA
:10C9580063616C6C203C63616C6C7369676E3E202C
:10C968002D20736574732063616C6C7369676E0D39
:10C978000A00000073736964203C302D31353E2075
:10C988002D207365747320535349440D0A00000029
:10C9980064657374203C616464726573733E202D12
:10C9A80020736574732064657374696E6174696F4C
:10C9B8006E20616464726573730D0A00747864652F
:10C9C8006C6179203C35302D323535303E202D20B4
:10C9D8007365747320545844656C61792074696D6B
:10C9E8006520286D73290D0A0000000074787461B1
:10C9F800696C203C31302D323535303E202D207386
:10CA08006574732054585461696C2074696D65208D
:10CA1800286D73290D0A00007175696574203C3111
:10CA280030302D323535303E202D2073657473201B
:10CA380071756965742074696D6520286D73290D99
:10CA48000A000000727331626175642F727332627A
:10CA5800617564203C313230302D3131353230301F
:10CA68003E202D20736574732055415254312F5543
:10CA7800415254322062617564726174650D0A0016
:10CA880070776D205B6F6E2F6F66665D202D206559
:10CA98006E61626C65732F64697361626C65732083
:10CAA80050574D2E2049662050574D206973206FEE
:10CAB80066662C205232522077696C6C20626520A1
:10CAC8007573656420696E73746561640D0A00008E
:10CAD800666C6174205B6F6E2F6F66665D202D201B
:10CAE80073657420746F20226F6E22206966206639
:10CAF8006C617420617564696F20696E707574204B
:10CB0800697320757365640D0A00000062656163CE
:10CB18006F6E203C302D373E205B6F6E2F6F666640
:10CB28005D202D20656E61626C65732F6469736189
:10CB3800626C6573207370656369666965642062F9
:10CB48006561636F6E0D0A00626561636F6E203CFC
:10CB5800302D373E205B69762F646C5D203C302D8C
:10CB68003732303E202D207365747320696E7465EA
:10CB78007276616C2F64656C617920666F722074BF
:10CB880068652073706563696669656420626561BC
:10CB9800636F6E20286D696E290D0A0062656163F6
:10CBA8006F6E203C302D373E2070617468203C65E4
:10CBB8006C312C5B656C325D3E2F6E6F6E65202D7F
:10CBC8002073657473207061746820666F722074B6
:10CBD800686520737065636966696564206265616C
:10CBE800636F6E0D0A000000626561636F6E203C22
:10CBF800302D373E2064617461203C646174613E6D
:10CC0800202D207365747320696E666F726D617470
:10CC1800696F6E206669656C6420666F722074683F
:10CC28006520737065636966696564206265616320
:10CC38006F6E0D0A0000000064696769205B6F6E03
:10CC48002F6F66665D202D20656E61626C65732F9F
:10CC580064697361626C65732077686F6C652064C2
:10CC68006967697065617465720D0A00646967694E
:10CC7800203C302D373E205B6F6E2F6F66665D203F
:10CC88002D20656E61626C65732F64697361626CD7
:10CC980065732073706563696669656420736C6F7A
:10CCA800740D0A0064696769203C302D373E2061A5
:10CCB8006C696173203C616C6961733E202D20733F
:10CCC80065747320616C69617320666F7220746883
:10CCD800652073706563696669656420736C6F7439
:10CCE8000D0A000064696769203C302D333E205BE3
:10CCF8006D61782F7265705D203C302F312D373E85
:10CD0800202D2073657473206D6178696D756D2FA2
:10CD18007265706C6163656D656E74204E20666F18
:10CD2800722074686520737065636966696564203C
:10CD3800736C6F740D0A000064696769203C302DBC
:10CD4800373E2074726163205B6F6E2F6F66665D7D
:10CD5800202D20656E61626C65732F646973616252
:10CD68006C6573207061636B6574207472616369AC
:10CD78006E6720666F7220746865207370656369DA
:10CD88006669656420736C6F740D0A00646967696D
:10CD9800203C302D373E20766973636F7573205BB6
:10CDA8006F6E2F6F66665D202D20656E61626C6503
:10CDB800732F64697361626C657320766973636F3E
:10CDC80075732D64656C6179206469676970656144
:10CDD80074696E6720666F72207468652073706569
:10CDE80063696669656420736C6F740D0A000000DE
:10CDF80064696769203C302D373E20646972656339
:10CE080074205B6F6E2F6F66665D202D20656E61E6
:10CE1800626C65732F64697361626C657320646901
:10CE2800726563742D6F6E6C7920646967697065CB
:10CE38006174696E6720666F72207468652073700C
:10CE48006563696669656420736C6F740D0A000018
:10CE580064696769203C302D373E2066696C7465CB
:10CE680072205B6F6E2F6F66665D202D20656E6188
:10CE7800626C65732F64697361626C65732070619D
:10CE8800636B65742066696C746572696E67206689
:10CE98006F7220746865207370656369666965647C
:10CEA80020736C6F740D0A00646967692066696C89
:10CEB800746572205B626C61636B2F776869746557
:10CEC8005D202D20736574732066696C74657269C2
:10CED8006E67207479706520746F20626C61636B73
:10CEE8006C6973742F77686974656C6973740D0A5B
:10CEF80000000000646967692064757065203C352E
:10CF08002D3235353E202D207365747320616E7483
:10CF1800692D64757065206275666665722074692E
:10CF28006D65202873290D0A00000000646967698F
:10CF3800206C697374203C302D31393E205B736559
:10CF480074203C63616C6C3E2F72656D6F76655D15
:10CF5800202D20736574732F636C65617273207361
:10CF680070656369666965642063616C6C73696781
:10CF78006E20736C6F7420696E2066696C746572BC
:10CF8800206C6973740D0A006175746F726573653E
:10CF980074203C302D3235353E202D207365747356
:10CFA800206175746F2D726573657420696E746580
:10CFB8007276616C20286829202D203020746F201B
:10CFC80064697361626C650D0A0000006D6F6E6BB9
:10CFD800697373205B6F6E2F6F66665D202D2073FB
:10CFE800656E64206F776E20616E6420646967697E
:10CFF800706561746564206672616D657320746F15
:10D00800204B49535320706F7274730D0A0000004F
:10D0180073617665000000006572617365616C6C10
:10D02800000000007072696E7400000043616C6C4F
:10D038007369676E3A2000000D0A44657374696E5F
:10D048006174696F6E3A20000D0A545844656C612A
:10D058007920286D73293A20000000000D0A5458E1
:10D068005461696C20286D73293A20000D0A5175A6
:10D078006965742074696D6520286D73293A2000EC
:10D088000D0A5541525431206261756472617465AC
:10D098003A2000000D0A55415254322062617564ED
:10D0A800726174653A2000000D0A44414320747986
:10D0B80070653A200000000050574D00523252006F
:10D0C8000D0A466C617420617564696F20696E7021
:10D0D80075743A2000000000796573006E6F0000D7
:10D0E8000D0A426561636F6E200000004F6E2C20B0
:10D0F80049763A20000000004F66662C2049763AAF
:10D10800200000002C20446C3A2000006E6F207034
:10D11800617468000D0A44696769706561746572B5
:10D128003A2000004F6E0D0A000000004F66660DA1
:10D138000A000000416C6961732000004F6E2C20CA
:10D148006D61783A200000004F66662C206D61788A
:10D158003A2000002C207265703A20002C2074724E
:10D16800616365642C2000002C20756E7472616305
:10D1780065642C2000000000766973636F75732D59
:10D1880064656C61792C20006469726563742D6F25
:10D198006E6C792C2000000066696C746572656499
:10D1A8000D0A0000756E66696C74657265640D0A17
:10D1B800000000004F6E2C20000000004F66662C17
:10D1C80020000000756E7472616365642C20000095
:10D1D800416E74692D6475706C6963617465206251
:10D1E800756666657220686F6C642074696D652069
:10D1F8002873293A200000000D0A43616C6C73699A
:10D20800676E2066696C74657220747970653A205F
:10D218000000000077686974656C6973740D0A0012
:10D22800626C61636B6C6973740D0A0043616C6CAA
:10D238007369676E2066696C746572206C697374B3
:10D248003A20000020656E74726965730D0A417595
:10D25800746F2D7265736574206576657279202800
:10D2680068293A200000000064697361626C656493
:10D27800000000000D0A4B495353206D6F6E69740E
:10D288006F723A20000000006C697374000000009F
:10D2980043616C6C7369676E2066696C7465722093
:10D2A8006C6973743A200D0A000000002E200000FB
:10D2B800656D70747900000063616C6C000000009B
:10D2C800496E636F72726563742063616C6C736915
:10D2D800676E210D0A0000004F4B0D0A0000000088
:10D2E8006465737400000000496E636F7272656351
:10D2F800742061646472657373210D0A0000000074
:10D308007373696400000000496E636F727265632D
:10D31800742053534944210D0A0000007478646551
:10D328006C617900496E636F72726563742054583A
:10D3380044656C6179210D0A0000000074787461FD
:10D34800696C0000496E636F72726563742054588B
:10D358005461696C210D0A007175696574000000DB
:10D36800496E636F727265637420717569657420A4
:10D3780074696D65210D0A0072733162617564000C
:10D388007273326261756400496E636F72726563AD
:10D3980074206261756472617465210D0A00000071
:10D3A800626561636F6E0000496E636F72726563D8
:10D3B8007420626561636F6E206E756D6265720DB3
:10D3C8000A0000004461746120746F6F206C6F6EF6
:10D3D800670D0A00496E636F72726563742070612D
:10D3E8007468210D0A000000496E636F72726563EC
:10D3F8007420636F6D6D616E640D0A0064696769FE
:10D4080000000000496E636F727265637420616C7E
:10D41800696173206E756D6265720D0A0000000007
:10D428006F666600616C696173200000496E636F06
:10D43800727265637420616C696173210D0A000062
:10D448006D61782000000000726570200000000007
:10D45800496E636F72726563742076616C756521BD
:10D468000D0A0000747261632000000066696C7424
:10D4780065722000766973636F7573200000000081
:10D4880064697265637420007768697465000000D8
:10D49800626C61636B0000006475706520000000B9
:10D4A800496E636F727265637420616E74692D646E
:10D4B8007570652074696D65210D0A006C69737457
:10D4C800200000007365742000000000496E636F3F
:10D4D800727265637420666F726D6174210D0A0043
:10D4E80072656D6F76650000496E636F7272656371
:10D4F8007420636F6D6D616E64210D0A0000000079
:10D508006175746F7265736574200000496E636F8E
:10D5180072726563742074696D6520696E746572D2
:10D5280076616C210D0A000070776D200000000004
:10D53800666C6174200000006D6F6E6B69737320F8
:10D548000000000056502D446967690050696F74E7
:10D55800722057696C6B6F6E205351384C00000075
:10D56800706F77007371727466000000000FC93F16
:10D57800000F494000CB9640000FC9400053FB40C4
:10D5880000CB164100ED2F41000F494100316241A7
:10D5980000537B41003A8A4100CB9641005CA3418D
:10D5A80000EDAF41007EBC41000FC94100A0D5414C
:10D5B8000031E24100C2EE410053FB4100F2034258
:10D5C800003A0A420083104200CB164200141D4262
:10D5D800005C234200A5294200ED2F420036364266
:10D5E800007E3C4200C74242000F4942A2000000B0
:10D5F800F9000000830000006E0000004E000000EB
:10D60800440000001500000029000000FC00000094
:10D618002700000057000000D1000000F5000000BE
:10D6280034000000DD000000C0000000DB00000046
:10D638006200000095000000990000003C00000016
:10D64800430000009000000041000000FE000000C0
:10D658005100000063000000AB000000DE00000085
:10D66800BB000000C500000061000000B70000001A
:10D67800240000006E0000003A0000004200000094
:10D688004D000000D2000000E0000000060000008D
:10D69800490000002E000000EA0000000900000018
:10D6A800D1000000920000001C000000FE000000F5
:10D6B8001D000000EB0000001C000000B10000008D
:10D6C80029000000A70000003E000000E80000005C
:10D6D8008200000035000000F50000002E00000068
:10D6E800BB0000004400000084000000E9000000C6
:10D6F8009C0000007000000026000000B40000003C
:10D708005F0000007E0000004100000039000000BA
:10D7180091000000D60000003900000083000000DE
:10D728005300000039000000F40000009C000000D5
:10D73800840000005F0000008B000000BD000000B6
:10D74800F9000000280000003B0000001F00000056
:10D75800F800000097000000FF000000DE00000055
:10D7680005000000980000000F000000EF00000016
:10D778002F000000110000008B0000005A0000007C
:10D788000A0000006D0000001F0000006D0000008E
:10D79800360000007E000000CF00000027000000D7
:10D7A800CB00000009000000B70000004F00000097
:10D7B800460000003F000000660000009E000000D8
:10D7C8005F000000EA0000002D0000007500000066
:10D7D80027000000BA000000C7000000EB000000AE
:10D7E800E5000000F10000007B0000003D000000A3
:10D7F8000700000039000000F70000008A00000060
:10D808005200000092000000EA0000006B000000D7
:10D81800FB0000005F000000B10000001F000000D6
:10D828008D0000005D0000000800000056000000A8
:10D83800030000003000000046000000FC0000006B
:10D848007B0000006B000000AB000000F00000004F
:10D85800CF000000BC000000200000009A0000007B
:10D86800F4000000360000001D000000A9000000C0
:10D87800E300000091000000610000005E0000006D
:10D88800E60000001B000000080000006500000022
:10D8980099000000850000005F00000014000000EF
:10D8A800A000000068000000400000008D0000009B
:10D8B800FF000000D8000000800000004D000000BC
:10D8C800730000002700000031000000060000007F
:10D8D800060000001500000056000000CA00000005
:10D8E80073000000A8000000C900000060000000EC
:10D8F800E20000007B000000C00000008C00000077
:10D908006B0000000000C93F0000F0390000DA3762
:10D918000000A2330000842E0000502B0000C22714
:10D928000000D0220000C41F0000C61B00004417DE
:10D9380004000000070000000900000000000000CB
:10D94800000000000000304300000000000030C369
:04D95800350100088D
:04D95C0011010008AD
:10D96000010000001000000009024300020100C095
:10D970003209040000010202010005240010010523
:10D980002401000104240202052406000107058287
:10D990000308001009040100020A00000007050145
:10D9A0000240000007058102400000000902430018
:10D9B000020100C032090400000102020100052436
:10D9C00000100105240100010424020205240600C0
:10D9D000010705820308001009040100020A000083
:10D9E0000007050102000200070581020002000095
:10D9F00009074300020104C03209040000010202C9
:10DA00000100052400100105240100010424020284
:10DA1000052406000107058203080010090401001F
:10DA2000020A00000007050102400000070581020C
:10DA3000400000000A060002000000400100000053
:10DA4000672F0008252F00084B2E0008000000005B
:10DA5000772D0008FF2D0008D12D000800000000E0
:10DA60000000000000000000AD2D0008A12D0008FE
:10DA7000B92D0008C52D000834C1000882A09CAC57
:10DA8000606260009C608682989800000024F40028
:10DA9000F18400088D8400089184000895840008B2
:10DAA00012010002020200408304405700020102FA
:10DAB00003010000040309041A0300000000000031
:10DAC0000000000000000000000000000000000056
:10DAD0000000000099870008A58700085988000801
:10DAE0003588000821880008758800089988000892
:10DAF000020100009801002000000000000000006A
:10DB00000000000000000000000000000000000015
:10DB10000000000000000000000000000000000005
:10DB200000000000000000000000000000000000F5
:10DB300000000000000000000000000000000000E5
:10DB400000000000000000000000000000000000D5
:08DB50000000000000000000CD
:0400000508009C71E2
:00000001FF
